:100000000C949F2E0C94D02E0C94D02E0C94D02EA9
:100010000C94D02E0C94D02E0C94D02E0C94D02E68
:100020000C94D02E0D94154E0D94154E0D94154E26
:100030000C94D02E0C94D02E0C94D02E0C94D02E48
:100040000C94D02E0C945FB30C94D02E0C94D02E24
:100050000C94D02E0C94D02E0C9458AC0D94CB4D07
:100060000C94D02E0C94107D0C94DA7C0C94D02E31
:100070000C94D02E0C94D02E0C94D02E0C94D02E08
:100080000C94D02E0C94D02E0C94D02E0C94D02EF8
:100090000C94D02E0C94D02E0C94D02E0C94D02EE8
:1000A0000C94D02E0C94D02E0C94D02E0C94D02ED8
:1000B0000C94D02E0C94D02E0C94D02E0C94D02EC8
:1000C0000C94D02E0C94D02E0C94D02E0C94D02EB8
:1000D0000C94D02E0C94D02E0C94D02E0C94D02EA8
:1000E0000C94D02E084AD73B3BCE016E84BCBFFD9A
:1000F000C12F3D6C74319ABD56833DDA3D00C77FF8
:1001000011BED9E4BB4C3E916BAAAABE0000008090
:100110003F05A84CCDB2D44EB93836A9020C50B91F
:10012000918688083CA6AAAA2ABE000000803F004B
:100130000C94D0440C94C0500C943E4E0C94E54367
:100140000C940F420C94F1410C94D2410D94B302E3
:100150000D9448240C94784F0C94D6430C94C840CA
:100160000C94BD400D94544B0C9496EE0D94F811E4
:100170000C94F94C0C9404F00C94F3440D949F539C
:100180000C9473980C9484430C94C4410C940442D2
:100190000C941F410C9425F80C9439420C940DF8E2
:1001A0000D94AF4B0D94C3030C9495980C94BF4ED3
:1001B0000C945A4D0C94BB500C94D7410C94874E20
:1001C0000C94C1440C940AF10C94DC3F0C94D2EED4
:1001D0000D94C34B0D94E6110C944E4D0C94D24FDC
:1001E0000D9440240C940CEE0C9400F10D94F2113B
:1001F0000C9440980C94DF400D94AC150C949845E9
:100200000C9484F80C94CB4E0C9497500C941C5086
:100210000D9460240D9463120C94ED4F0C949DF199
:100220000D9499240C94364E0C94BD410D944917AD
:100230000C94B8F00C940A420D94CE110C949F7D4E
:100240000C9405F10C947DF20C9448410C94CE4032
:100250000D948E490D940A120C9429F00D944D12B0
:100260000C944E4E0C94F4430C949B940D945612A3
:100270000C9475430C94BB450C949B7D0C94664D7B
:100280000C9449450C94E8400C94474D0C94EE4472
:100290000D945B570D943B170D9492490C9419F2F1
:1002A0000D9447120C942F4D0D9476240C943B4DD5
:1002B0000C94D9F10C946D410C9480F10C94C941CB
:1002C0000C9487960D94F0060C9428500C94274EAD
:1002D0000C94D32E0D9436170C942F500D94784B0C
:1002E0000C94E3F20C94FBF00D9453120D945E4BBE
:1002F0000C9404500D9451230C9454410D946612A7
:100300000D945B490D94860E0D9410120C9467F0B9
:100310000C9458500C94F14E0C9442EE0C94AAEEAE
:100320000C94F04D0C94FEEF0C944B7D0C94F4EE79
:100330000C94D24D0C94823F0C94304F0C94AA40F4
:100340000C943B500C9433F30C9482EE0C94BC440C
:100350000C942D3F0C94B1400C9468D90C94A39844
:100360000C946E4E0C94803F0C94E2410C943442F9
:100370000D94C2080C947A500C94884F0D94334B12
:100380000C9438F00C947E3F0D945F490C946C4FA4
:100390000C941EEE0C94444F0C9465980C94F94305
:1003A0000C94774E0C94FB500D947A490C9440D3E6
:1003B0000D9444120D948C4B0C94B73F0C94AA4F9F
:1003C0000C9443410D94404B0C94C3400C942B442B
:1003D0000C9416EF0D9476490C944F410D945012E5
:1003E0000D9468490D94D50F0D944A120C94994FB1
:1003F0000C9445F80C94BEF00C9435F80C94BA4F5C
:100400000C9423F20C945D440D94CD4B0C94767DAA
:100410000D9462490C94A37D0C948F440C943D413F
:100420000D94A54B0C9467410D9453490C9458EED0
:100430000C9474450C94CEFD0C94A7410C94E14DA2
:100440000C94D22E0D94E0110C9458440C9421423B
:100450000D94B94B0D949B4B0D94131B0C94BF4DF5
:100460000D9440170D948D490C9483400C94AD4429
:100470000D943B120C9462410C946D430D94161232
:100480000D945E120D9431170C946EEE0C9447F699
:100490000C941DF80D946C490D94FE010C948F4D35
:1004A0000C94FF4D0C94B2F00C94F04C0C9401F0B1
:1004B0000D94B2530C946A510C9411F00C94AF50FB
:1004C0000C9449440C9461F00D946B580D944D4973
:1004D0000D944A4B0C94AD410C94977D0C94DAF03A
:1004E0000D9457490C94B53F0C945D410C94184EF3
:1004F0000C94ECF50D9450230C94E6EE0C94A35060
:100500000C94DA3F0C94DE4F0C947EF10D9404129F
:100510000D94A8530C94064F0C945ED50C94324164
:100520000D94CA0C0C943A440C9410500C949B41BA
:100530000D94EC110C94DC4E0D945E4A0C9408EF73
:100540000C94F2400C948A440C9410990C9440F250
:100550000C94BAF90C94BEEE0C948C7D0C949441DE
:100560000D9472490C94DF440C946C440D9438053E
:100570000C944BFB0D9488490C945E980C94AF43FB
:100580000C9469500C941A420C9424F10C945B3F27
:100590000C94E89A0D94824B0C941C4D0D94CB0056
:1005A0000C942DF80C9419300C94BD430C9401500C
:1005B0000C941B4F0C94A74E0C945E4E0C947B44F1
:1005C0000C9426420C946C980D94664B0C9464F138
:1005D0000D94C8110C94A1F80C94724D0C94D34056
:1005E0000C94A74D0C9491430D9459120C94DCFC7F
:1005F0000C9402460C94DC410C94F74F0C94937DC0
:100600000C94584F0C94ED400C943AD70C94B8418C
:100610000C94C7430C94094E0C94C64F0C94B93FEC
:100620000D949F180C94114D0C9436510C9431F08C
:100630000C94D74E0C94774D0C94F8400D949A532B
:100640000C9421F00C9417440C94DA400C94A043C1
:100650000D9484490C948B500D9495530C94BAF1DD
:100660000C9453500C943A980C94974E0C94E94C7B
:100670000C94054D0C94C4F00C94ED9A0C94B34E6C
:100680000C9486F00C94DE3F0C94C4940D94BB241F
:100690000D9416000C9411EE0C9447500C949E444B
:1006A0000C9415420C9415F80C94593F0C94B241DB
:1006B0000C94B1980C94E14C0C9426410C94384164
:1006C0000C94F8410C94A97D0C9405F80C94DE452B
:1006D0000D94D4110D9492150C94D94C0C94FDF7F3
:1006E0000C941E450C94E34F0D9480490C940844DF
:1006F0000D94DA110C94BCF10C942F420C94847D6F
:100700000C94F29A0C940FF20C9419F00C94E6FEEF
:100710000C943DF80D940B1F0C94234D0D946E4BCF
:100720000C9476F20D943B4B0C9459960D94FE115B
:100730000C9465F00D9460120C9426440D94C449F9
:100740000C947D434E414E494E495459494E46CD35
:10075000CCCC3D0AD7233C17B7D13877CC2B329578
:1007600095E6241FB14F0A000020410000C8420056
:10077000401C4620BCBE4CCA1B0E5AAEC59D7443DD
:100780004F4D4D554E49434154494F4E00445259E7
:1007900052554E004552524F525300494E464F005B
:1007A0004543484F004572726F72207772697469D1
:1007B0006E6720746F20454550524F4D210A0062EC
:1007C0007573793A2070617573656420666F722065
:1007D000696E7075740A00627573793A207061757C
:1007E00073656420666F7220757365720A006275A6
:1007F00073793A2070726F63657373696E670A006C
:100800006D41290A0020647269766572206F7665F1
:100810007274656D7065726174757265207761724E
:100820006E696E67212028003A200020637572727D
:10083000656E742064656372656173656420746FAE
:1008400020006D41290A0020647269766572206F6C
:1008500076657274656D7065726174757265207706
:1008600061726E696E67212028003A20002063754E
:100870007272656E7420646563726561736564206D
:10088000746F20006D41290A0020647269766572D8
:10089000206F76657274656D7065726174757265CE
:1008A000207761726E696E67212028003A2000204F
:1008B00063757272656E74206465637265617365D9
:1008C0006420746F20006D41290A002064726976EB
:1008D0006572206F76657274656D7065726174758E
:1008E0007265207761726E696E67212028003A2058
:1008F000002063757272656E742064656372656151
:1009000073656420746F20004B494C4C2063617503
:10091000736564206279204B494C4C206275747475
:100920006F6E2F70696E0A004B494C4C20636175E5
:1009300073656420627920746F6F206D7563682021
:10094000696E6163746976652074696D65202D2018
:1009500063757272656E7420636F6D6D616E643A5B
:100960002000506C6561736520726573657400507A
:1009700052494E5445522048414C54454400706FF2
:100980007765726F6666004B494C4C45442E2000DB
:100990005072696E7465722068616C7465642E2093
:1009A0006B696C6C28292063616C6C6564210A009A
:1009B0006563686F3A004572726F723A0066616CE7
:1009C0007365007472756500486F74656E64207499
:1009D0006F6F20636F6C640A0050726573732062DE
:1009E0007574746F6E20286F72204D313038292055
:1009F000746F20726573756D650A00496E73657258
:100A0000742066696C616D656E7420616E6420701F
:100A10007265737320627574746F6E20286F722014
:100A20004D313038290A0050726573732062757435
:100A3000746F6E20286F72204D3130382920746F0A
:100A40002068656174206E6F7A7A6C650A00706147
:100A500075736564004D3630303A20546F6F2063F3
:100A60006F6C6400486F74656E6420746F6F2063F0
:100A70006F6C640A00726573756D656400496E730E
:100A80006572742066696C616D656E7420616E6458
:100A900020707265737320627574746F6E20286F96
:100AA00072204D313038290A0025753A25303275CB
:100AB00000253032753A25303275002575642025C1
:100AC0003032753A2530327500447269766572208D
:100AD0006572726F7200636F696C2073686F7274F5
:100AE00020636972637569740A006F766572746554
:100AF0006D70657261747572650A00206472697642
:100B00006572206572726F722064657465637465C6
:100B1000643A20307800303D2E33323500313D2E9E
:100B20003138006D6178002F3331002F3331002FC1
:100B3000333100303D2E33323500313D2E31380017
:100B40006D6178002F3331002F3331002F333100A6
:100B5000303D2E33323500313D2E3138006D617815
:100B6000002F3331002F3331002F333100303D2E31
:100B700033323500313D2E3138006D6178002F332E
:100B800031002F3331002F333100092042616420BE
:100B9000726573706F6E7365210009204261642075
:100BA000726573706F6E7365210009204261642065
:100BB000726573706F6E7365210009204261642055
:100BC000726573706F6E7365210044726976657229
:100BD000207265676973746572733A0A006F7409ED
:100BE000006F7470770900733267610900733267B0
:100BF0006209006F6C6109006F6C620900737473A5
:100C00007409006673616374697665090073675FD0
:100C1000726573756C7409007374616C6C677561CF
:100C2000726409004452565354415455530053744E
:100C3000616C6C67756172642074687273002D73E7
:100C4000746172740900687973746572657369738D
:100C50000A2D656E640900626C616E6B2074696DAB
:100C600065006F66662074696D6509004F542070D9
:100C700072657761726E206861730A6265656E20C5
:100C8000747269676765726564004F54207072659D
:100C90007761726E005B6D6D2F735D090070776D0B
:100CA0000A7468726573686F6C64090074737465A4
:100CB0007009006D73746570730900737465616CFD
:100CC000746843686F70007673656E7365090050D1
:100CD000574D207363616C650043532061637475E5
:100CE000616C0900486F6C642063757272656E7484
:100CF0000052756E2063757272656E74004D4158B6
:100D00002063757272656E7400524D532063757264
:100D100072656E74005365742063757272656E74CB
:100D200000456E61626C6564090009004C4F570014
:100D300048494748004F4B004572726F723A204154
:100D40006C6C200020636F6E6E656374696F6E2E2D
:100D50002E2E200054657374696E6720004C4F5727
:100D60000048494748004F4B004572726F723A2065
:100D7000416C6C200020636F6E6E656374696F6EEA
:100D80002E2E2E200054657374696E6720004C4F20
:100D9000570048494748004F4B004572726F723AFE
:100DA00020416C6C200020636F6E6E656374696F08
:100DB0006E2E2E2E200054657374696E6720004CD1
:100DC0004F570048494748004F4B004572726F72B9
:100DD0003A20416C6C200020636F6E6E656374690D
:100DE0006F6E2E2E2E200054657374696E6720007E
:100DF000544D4320434F4E4E454354494F4E20459A
:100E000052524F52000A0A426564204C6576656C66
:100E100020436F7272656374696F6E204D617472E6
:100E200069783A00202B000A436F7272656374651B
:100E30006420426564204865696768742076732E73
:100E40002042656420546F706F6C6F67793A0A00B6
:100E5000202B000A42656420486569676874205445
:100E60006F706F6772617068793A0A2020202B2DAD
:100E70002D2D204241434B202D2D2B0A2020207C5C
:100E800020202020202020202020207C0A204C20F0
:100E90007C20202020282B29202020207C20520A62
:100EA0002045207C20202020202020202020207C65
:100EB00020490A2046207C20282D29204E20282B3E
:100EC00029207C20470A2054207C2020202020201C
:100ED00020202020207C20480A2020207C20202048
:100EE00020282D29202020207C20540A2020207C0E
:100EF00020202020202020202020207C0A202020AC
:100F00004F2D2D2046524F4E54202D2D2B0A202898
:100F1000302C30290A003474682070726F626520AA
:100F2000706F696E742C2064697374616E636520E0
:100F300066726F6D20706C616E653A2000202844E7
:100F4000525952554E2900473239204175746F204D
:100F5000426564204C6576656C696E67003F2028A9
:100F60004C2C522C462C4229206F7574206F662021
:100F7000626F756E64732E0A003F50726F62652057
:100F8000706F696E74732028592920697320696D08
:100F9000706C61757369626C652028322D32292E60
:100FA0000A003F50726F626520706F696E74732023
:100FB00028582920697320696D706C6175736962A6
:100FC0006C652028322D32292E0A003F28562965CB
:100FD00072626F7365206C6576656C206973206939
:100FE0006D706C61757369626C652028302D3429D1
:100FF0002E0A0020284E6F7420796574206D65617B
:101000007375726564290020204176657261676599
:10101000206D65617375726564206261636B6C61DC
:10102000736820286D6D293A002020536D6F6F740E
:1010300068696E6720286D6D293A202020202020C5
:10104000202020202020202020202053002020426B
:1010500061636B6C6173682044697374616E63656E
:1010600020286D6D293A20202020202020200020DB
:101070002846312E30203D2066756C6C2C20463081
:101080002E30203D206E6F6E65290A002020436FB0
:101090007272656374696F6E20416D6F756E742F27
:1010A000466164652D6F75743A202020202046002B
:1010B0006163746976653A0A00696E004261636B28
:1010C0006C61736820436F7272656374696F6E2020
:1010D000004D6163726F20746F6F206C6F6E672EAE
:1010E0000A0047323800617869733A70776D5F7330
:1010F00063616C652F637572725F7363616C652FDA
:101100006D6563685F6C6F61647C666C6167737C3E
:101110007761726E636F756E740A004452565F5346
:101120005441545553090050574D5F5343414C456A
:10113000090050574D434F4E460900434F4F4C4313
:101140004F4E46090043484F50434F4E4609005406
:101150004849474809090054434F4F4C544852539B
:1011600009005450574D54485253090054535445A4
:101170005009090054504F574552444F574E0900EB
:10118000494F494E09090047535441540909004940
:10119000484F4C445F4952554E090047434F4E4615
:1011A00009090009007370726561644379636C65B5
:1011B00000737465616C746843686F7000206472BA
:1011C00069766572206D6F64653A090073707265A7
:1011D00061644379636C6500737465616C74684322
:1011E000686F700020647269766572206D6F646547
:1011F0003A09007370726561644379636C650073CA
:101200007465616C746843686F70002064726976FD
:101210006572206D6F64653A090073707265616470
:101220004379636C6500737465616C746843686FBF
:10123000700020647269766572206D6F64653A098A
:101240000020737465616C746843686F70206D6111
:10125000782073706565643A200020737465616C52
:10126000746843686F70206D617820737065656481
:101270003A200020737465616C746843686F702055
:101280006D61782073706565643A20002073746521
:10129000616C746843686F70206D6178207370654D
:1012A00065643A200020496E76616C696420657837
:1012B000747275646572200020746F6F206C6F6E9D
:1012C0006720657874727573696F6E2070726576C9
:1012D000656E7465640A0020636F6C6420657874C1
:1012E000727573696F6E2070726576656E74656471
:1012F0000A00536C6565702E2E2E004D313137205B
:10130000486F7420456E642048656174696E672E6D
:101310002E2E0A4D31303420533137302054300ACC
:10132000473238204F310A473120593235205A315F
:10133000302046353030300A4D3131372052657714
:101340006970696E67206E6F7A7A6C650A54300A2C
:101350004731205831313520593137342046353026
:1013600030300A4D31303920523137302054300A74
:101370004731205A310A473120583131352059310F
:1013800037342046343030300A4731205834352045
:10139000593137342046343030300A473120583103
:1013A000313520593137342046343030300A473116
:1013B0002058343520593137342046343030300A03
:1013C00047312058313135205931373420463430B7
:1013D00030300A47312058343520593137342046CF
:1013E000343030300A4731205831313520593137C7
:1013F000342046343030300A4731205834352059B3
:101400003137342046343030300A473120583131BA
:101410003520593137342046343030300A473120B6
:1014200058343520593137342046343030300A476B
:10143000312058313135205931373420463430305D
:10144000300A47312058343520593137342046345A
:101450003030300A4731205A31350A4D313036208C
:1014600053323535200A47302058302059300A4D44
:1014700031303920523136302054300A4D31303736
:101480000A004D31303420533137302054300A4D6A
:10149000313137204C6576656C696E672058204184
:1014A0007869730A4732380A47302058313530207E
:1014B00046393939390A4730205A352046363030D6
:1014C000300A4739310A4D3231312053300A4D3418
:1014D00030300A4D393036205A3630300A47302005
:1014E0005A2D313520463530300A4730205A3520C4
:1014F000463530300A4739300A4D3430300A4D39DC
:101500003036205A3936300A4D3231312053310AC3
:101510004732380A4D313137204C6576656C696E3B
:101520006720646F6E652E0A4731320A4D313039BB
:1015300020523136300A4D3131372050726F626996
:101540006E67206265640070726F62655F726577B6
:10155000697065004175746F6C6576656C206661B5
:10156000696C6564004D31313720426564206C65DB
:1015700076656C696E67206661696C65642E0A47E2
:1015800030205A31300A47302045300A4D33303050
:101590002050323520533838300A4D333030205007
:1015A00035302053300A4D333030205032352053FF
:1015B0003838300A4D333030205035302053300A1F
:1015C0004D3330302050323520533838300A4734CC
:1015D0002053310070726F62655F6661696C65648B
:1015E000004D3131372050726F626520737563632F
:1015F00065737366756C0A00205A3A200020593AC8
:10160000200042656420583A2000436C69636B20D7
:10161000746F20726573756D652E2E2E004E6F20CF
:101620006D6F76652E00456E642066696C65206C72
:101630006973740A00426567696E2066696C65208B
:101640006C6973740A00286E6F2066696C652900E6
:1016500043757272656E742066696C653A2000533A
:1016600044207072696E74696E67206279746520B7
:10167000004E6F74205344207072696E74696E67F7
:101680000A002E0A0044656C6574696F6E206661FD
:10169000696C65642C2046696C653A200046696C6B
:1016A000652064656C657465643A005072696E7497
:1016B0002074696D653A200050726F7465637465BB
:1016C000642050696E0A0025311D402924301C45D4
:1016D00027232F1B0A0743222B1A42043803FF3605
:1016E0000408060600010A53746174733A204669BF
:1016F0006C616D656E7420757365643A20002C20F2
:101700004C6F6E67657374206A6F623A2000546F85
:1017100074616C2074696D653A2000537461747350
:101720003A20002C204661696C65643A20002C2028
:1017300046696E69736865643A20005072696E7418
:10174000733A200053746174733A2000486F7465D3
:101750006E6420436F6F6C696E672E2E2E00486F8B
:1017600074656E642048656174696E672E2E2E0064
:101770006F666600A0079B0794078D077F074445A7
:101780004255473A004D3131332053006F6B004CC6
:10179000756C7A426F74204D696E692032204F4615
:1017A000462E004348414D4245525F54454D5045F9
:1017B000524154555245004D4F54494F4E5F4D4F85
:1017C00044455300544845524D414C5F50524F548C
:1017D000454354494F4E004155544F5245504F5286
:1017E000545F53445F5354415455530050524F4D2E
:1017F00050545F535550504F525400454D45524739
:10180000454E43595F504152534552004341534561
:101810005F4C494748545F4252494748544E4553EC
:101820005300544F47474C455F4C49474854530079
:10183000534F4654574152455F504F57455200420F
:1018400055494C445F50455243454E54004C455613
:10185000454C494E475F44415441005A5F50524FF6
:101860004245004155544F4C4556454C0050524955
:101870004E545F4A4F420050524F47524553530017
:101880004155544F5245504F52545F54454D5000AE
:10189000564F4C554D455452494300454550524FC3
:1018A0004D0042494E4152595F46494C455F5452A2
:1018B000414E534645520053455249414C5F584FA3
:1018C0004E5F584F4646004649524D574152455F7C
:1018D0004E414D453A4D61726C696E202046495229
:1018E0004D574152455F56455253494F4E3A322E5D
:1018F000302E302E31343420455854525544455200
:101900005F545950453A4D31373520534F55524366
:10191000455F434F44455F55524C3A687474707349
:101920003A2F2F636F64652E616C6570686F626A11
:10193000656374732E636F6D2F6469666675736972
:101940006F6E2F4D41524C494E2050524F544F43D1
:101950004F4C5F56455253494F4E3A312E30204D31
:10196000414348494E455F545950453A4C756C7A4D
:10197000426F74204D696E6920322045585452558B
:101980004445525F434F554E543A312055554944D2
:101990003A65353530323431312D643436642D3486
:1019A0003231642D626133612D61323031323664FF
:1019B00037393330660A002F2F20004D313435205F
:1019C000533C696E6465783E206F7574206F6620A5
:1019D00072616E67652028302D31290A002054007D
:1019E000205200416363656C65726174696F6E3A81
:1019F000205000205A00205900580020204D6178C6
:101A00003A2000205A00205900580020204D696ECD
:101A10003A2000536F667420656E6473746F707340
:101A20003A200020466C6F773A200050726F626552
:101A3000205A204F66667365743A200020643A008D
:101A400020693A0020703A00496E76616C69642022
:101A500065787472756465720A0020643A002069C2
:101A60003A0020703A0064697300656E0043290AE9
:101A70000061626C656420286D696E2074656D700C
:101A80002000436F6C642065787472756465732000
:101A900061726520004F4646004F4E00426564204B
:101AA0004C6576656C696E6720004661696C65649B
:101AB00020746F20656E61626C6520426564204C05
:101AC0006576656C696E670A00426564204C6576D0
:101AD000656C20436F7272656374696F6E204D612F
:101AE000747269783A00454550524F4D204F4B0A69
:101AF000003F5A206F7574206F662072616E6765B3
:101B000020282D3220746F2035290A0050726F6210
:101B100065205A204F66667365743A20003F4B205B
:101B200076616C7565206F7574206F662072616ECA
:101B300067652028302D3130292E0A0041647661F6
:101B40006E6365204B3D0020647269766572206388
:101B5000757272656E743A200020647269766572DF
:101B60002063757272656E743A2000206472697623
:101B700065722063757272656E743A20002064721B
:101B8000697665722063757272656E743A20002002
:101B900074656D70657261747572652070726577B9
:101BA00061726E207472696767657265643A2000BD
:101BB0002074656D706572617475726520707265F0
:101BC0007761726E207472696767657265643A2026
:101BD000002074656D706572617475726520707235
:101BE000657761726E207472696767657265643AC1
:101BF00020002074656D7065726174757265207067
:101C000072657761726E2074726967676572656468
:101C10003A2000207072657761726E20666C616791
:101C200020636C65617265640A002070726577617B
:101C3000726E20666C616720636C65617265640A10
:101C400000207072657761726E20666C6167206338
:101C50006C65617265640A00207072657761726EEE
:101C600020666C616720636C65617265640A0020A0
:101C7000686F6D696E672073656E736974697669E4
:101C800074793A200020686F6D696E672073656E05
:101C900073697469766974793A2000496E76616C6B
:101CA00069642065787472756465720A00436170B6
:101CB0003A0047322F4733206261642070617261BD
:101CC0006D65746572730A00220A00656E71756530
:101CD0007565696E672022002042002050006F6BFE
:101CE00000526573656E643A200053544F5050455E
:101CF000442E20005072696E7465722073746F7088
:101D00007065642064756520746F206572726F72EF
:101D1000732E2046697820746865206572726F7230
:101D200020616E6420757365204D39393920746FD8
:101D300020726573746172742E202854656D70650D
:101D40007261747572652069732072657365742E93
:101D50002053657420697420616674657220726511
:101D60007374617274696E67290A004E6F2043684C
:101D700065636B73756D2077697468206C696E6537
:101D8000206E756D6265722C204C617374204C69F5
:101D90006E653A20004E6F20436865636B73756D06
:101DA0002077697468206C696E65206E756D626558
:101DB000722C204C617374204C696E653A2000636C
:101DC0006865636B73756D206D69736D61746368AD
:101DD0002C204C617374204C696E653A20004C696C
:101DE0006E65204E756D626572206973206E6F742A
:101DF000204C617374204C696E65204E756D626570
:101E0000722B312C204C617374204C696E653A2022
:101E1000004D313130004D33310053442072656143
:101E200064206572726F720A00446F6E6520707272
:101E3000696E74696E672066696C650A002569734E
:101E40000025696D20256973002569682025696D65
:101E50002025697300256964202569682025696D3E
:101E60002025697300256979202569642025696822
:101E70002025696D202569730020573A004265646A
:101E800020636F6F6C696E672E2E2E004265642092
:101E900068656174696E672E2E2E0023646566691D
:101EA0006E652044454641554C545F0000626564B0
:101EB000004B6420004B6920004B702000504944C7
:101EC000204175746F74756E652066696E697368FC
:101ED0006564212050757420746865206C6173748A
:101EE000204B702C204B6920616E64204B64206372
:101EF0006F6E7374616E74732066726F6D206265AD
:101F00006C6F7720696E746F20436F6E66696775BA
:101F1000726174696F6E2E680A00504944204175E1
:101F2000746F74756E65206661696C6564212074D8
:101F3000696D656F75740A00486F74656E6420542E
:101F40004845524D414C2052554E4157415900424F
:101F5000454420544845524D414C2052554E41571E
:101F6000415900546865726D616C2052756E6177DD
:101F7000617900486F74656E642048656174696EAC
:101F800067206661696C656400426564206865610C
:101F900074696E67206661696C6564004865617488
:101FA000696E67206661696C656400504944204130
:101FB00075746F74756E65206661696C6564212047
:101FC00054656D706572617475726520746F6F20F1
:101FD000686967680A00204B643A2000204B693A20
:101FE0002000204B703A20000A20436C6173736913
:101FF0006320504944200A002054753A2000204BA9
:10200000753A2000206D61783A2000206D696E3AA3
:10201000200020643A200020626961733A20005059
:102020004944204175746F74756E652073746172D4
:10203000740A00504944204175746F74756E6520B0
:102040006661696C6564212054656D7065726174A8
:1020500075726520746F6F20686967680A0050495F
:1020600044204175746F74756E65206661696C6596
:102070006421204261642065787472756465722001
:102080006E756D6265720A004572723A20757466EB
:102090003820666F6E74206E6F7420696E69746983
:1020A000616C697A65642E004572723A20757466B7
:1020B0003820666F6E74206E6F7420696E69746963
:1020C000616C697A65642E003048483025336400BD
:1020D0002534640025202000252000202020200019
:1020E0004572723A207574663820666F6E74206E81
:1020F0006F7420696E697469616C697A65642E0019
:102100001FFFFFFFFFFFFF600000000001FF400016
:1021100000000000FF8000000000007F83CF00006F
:102120000C303F87FF80000C301F867980000C0048
:102130000F8C30C7838C30E78C30CFC7CC31F38C19
:1021400030DCECEC33B98C30D86C6C33198C30D07B
:102150006C0C33198C30D86C0C33198C30DC6C0E51
:102160003B198C30CF7C079F198C30C77C038F19AB
:1021700040000000000002600000000000061FFF99
:10218000FFFFFFFFF8486F74656E6400486F746569
:102190006E64005A005A0059005900580058005403
:1021A0004D43206472697665727300590059005876
:1021B000005800544D432064726976657273004F75
:1021C0006666004F6E00486F74656E64004F666609
:1021D000004F6E005A004F6666004F6E0059004F68
:1021E0006666004F6E005800544D43206472697655
:1021F00065727300537465616C746843686F702016
:10220000656E61626C6564005374657070696E67B9
:10221000206D6F64650053656E736F726C657373C8
:1022200020686F6D696E6700487962726964207416
:1022300068726573686F6C640044726976657220B9
:1022400063757272656E7400436F6E74726F6C00AA
:1022500042616279737465702058004261627973DB
:1022600074657020590050726F6265205A204F6665
:1022700066736574004261627973746570205900F9
:102280004261627973746570205800466C6F770004
:10229000466C6F770046616E20737065656400461A
:1022A000616E207370656564004265640042656418
:1022B000004E6F7A7A6C65004E6F7A7A6C650053C7
:1022C00070656564005370656564004D61696E00FA
:1022D0000000007E006000600060F87ECC60CC6092
:1022E000CC60F860CC00CC00CC00CC00000000003A
:1022F00000000000000000000000000000000000DE
:10230000000000000000FE7FFE7F0660000000006D
:1023100000000000F00FF81FF81FF81FF00FF00F7B
:10232000F81FF81FF81FE007C0038001000000003D
:102330000000FE7F0E702664724E7A5E324C82413F
:10234000324C7A5E724E26640E70FE7F00000000F2
:102350000000FE7F0E70C663C24382411A58BA5D08
:102360001A588241C243C6630E70FE7F000000000F
:1023700000008808880810112022202210118808E7
:10238000880810110000000000000000000000009C
:102390000000202210118808880810112022202215
:1023A000101188080000000000000000000000007C
:1023B000436172642072656D6F766564004361727B
:1023C0006420696E736572746564004D696E69207E
:1023D000322072656164792E005072696E74696E84
:1023E000672E2E2E005072696E74207061757365B1
:1023F000640063616E63656C005072696E74206185
:10240000626F727465640000002C43000034430066
:10241000003743000010C10000A0C00000000029E8
:102420000A002062797465733B2063726320005355
:10243000657474696E67732053746F7265642028C5
:1024400000454550524F4D206461746173697A654F
:10245000206572726F722E0A00290A002062797458
:1024600065733B2063726320002073746F72656430
:102470002073657474696E67732072657472696520
:10248000766564202800202863616C63756C617434
:10249000656429210A0020213D2000454550524F06
:1024A0004D20435243206D69736D61746368202D24
:1024B000202873746F7265642920002053697A653F
:1024C0003A2000496E6465783A2000204D61726CB4
:1024D000696E3D563637290A00454550524F4D200A
:1024E00076657273696F6E206D69736D6174636870
:1024F0002028454550524F4D3D00454550524F4DC7
:1025000020496E697469616C697A65640A00486182
:102510007264636F6465642044656661756C7420E1
:1025200053657474696E6773204C6F616465640AE7
:10253000002823000028230000C8000000E8030052
:1025400000000096430000964300009643000020E0
:10255000420000C8420000C842000048430080CF4B
:10256000433A0A0020204D3930360020204D3931C1
:10257000330020204D3931340020204D36303320B7
:1025800000205300205A0020590020580020204DE0
:102590003432352046004261636B6C61736820639E
:1025A0006F6D70656E736174696F6E3A0A002055C5
:1025B000004C0046696C616D656E74206C6F6164DF
:1025C0002F756E6C6F6164206C656E677468733A0A
:1025D0000A0020204D393030204B004C696E656177
:1025E0007220416476616E63653A0A00543020457A
:1025F00000205A0020590020580020204D3536393F
:10260000205331004472697665722073746570706E
:10261000696E67206D6F64653A0A00205900205882
:10262000005374616C6C47756172642074687265E4
:1026300073686F6C643A0A00205430204500205AB9
:10264000002059002058004879627269642054685B
:10265000726573686F6C643A0A002054302045003C
:10266000205A00205900205800537465707065721C
:10267000206472697665722063757272656E743A51
:102680000A0020204D383531205A005A2D50726FE3
:102690006265204F6666736574002044002049001F
:1026A00020204D33303420500020440020490020A9
:1026B000204D3330312050005049442073657474EC
:1026C000696E67733A0A00204600204200204800E5
:1026D00020204D3134352053004D6174657269619D
:1026E0006C2068656174757020706172616D6574CD
:1026F0006572733A0A0020204D3432302053004175
:1027000075746F20426564204C6576656C696E67F0
:102710003A0A00204500205A002059002058002085
:10272000540020530020204D3230352042002045F7
:102730003C6D61785F655F6A65726B3E0020583C56
:102740006D61785F785F6A65726B3E20593C6D61A0
:10275000785F795F6A65726B3E205A3C6D61785F85
:102760007A5F6A65726B3E00416476616E63656490
:102770003A20423C6D696E5F7365676D656E745F8C
:1027800074696D655F75733E20533C6D696E5F665D
:10279000656564726174653E20543C6D696E5F745A
:1027A000726176656C5F66656564726174653E0032
:1027B00020540020520020204D323034205000415F
:1027C0006363656C65726174696F6E2028756E69EC
:1027D00074732F7332293A20503C7072696E745FA3
:1027E000616363656C3E20523C7265747261637410
:1027F0005F616363656C3E20543C74726176656C06
:102800005F616363656C3E0A00204500205A00202A
:10281000590020204D3230312058004D6178696DCB
:10282000756D20416363656C65726174696F6E20BC
:1028300028756E6974732F7332293A0A0020450097
:10284000205A0020590020204D3230332058004DAE
:102850006178696D756D2066656564726174657314
:102860002028756E6974732F73293A0A00537465B2
:1028700070732070657220756E69743A0A002020AA
:102880004D3134392043203B20556E6974732069E3
:102890006E2043656C736975730A0020286D6D297D
:1028A000002020473231202020203B20556E6974C3
:1028B0007320696E206D6D006F70656E0054524913
:1028C000474745524544003A20007A5F6D617800E1
:1028D0007A5F6D696E00795F6D617800785F6D6910
:1028E0006E005265706F7274696E6720656E6473F6
:1028F000746F70207374617475730A00205A3A0003
:1029000020593A0020436F756E7420583A002045D4
:102910003A00205A3A0020593A00583A00486F6D60
:1029200065202573257325732066697273740020F2
:1029300066697273740A00486F6D652000486F6D98
:10294000696E67206661696C656400000010C100F3
:102950000034430000374300004842000048420072
:102960000020425761726E696E673A20486F6D6948
:102970006E672042756D702044697669736F7220AE
:102980003C20310A000202040000000000000000A8
:102990000000004000003543000039430000374389
:1029A000FF010124F4D43050C38E20C2A24017820C
:1029B0008B7011127A910D816CD90AA861E108C758
:1029C000586607615143061E4B5D05C145A7041AB1
:1029D000411104093D9803713931034036DB02652A
:1029E000339102D4305402802E1D02632CEE017507
:1029F0002AC501B028A001102781018F2564012B71
:102A0000244B01E0223401AC211F018D200D0180F7
:102A10001FFC00841EED00971DDF00B81CD200E6ED
:102A20001BC600201BBC00641AB200B219A8000A21
:102A300019A0006A189900D117910040178B00B5B2
:102A400016840031167E00B31579003A157300C75D
:102A5000146F0058146A00EE136600881363002593
:102A6000135E00C7125B006C12570015125400C1B0
:102A700011510070114F0021114B00D61049008DEB
:102A80001047004610440002104200C00F40008072
:102A90000F3E00420F3C00060F3B00CB0E38009368
:102AA0000E37005C0E3500270E3400F30D3200C1E6
:102AB0000D3100900D3000600D2E00320D2D0005FF
:102AC0000D2C00D90C2B00AE0C2900850C29005CC4
:102AD0000C2700350C27000E0C2600E80B2400C440
:102AE0000B2400A00B23007D0B23005A0B2100397F
:102AF0000B2100180B2000F80A1F00D90A1E00BB8A
:102B00000A1E009D0A1D00800A1D00630A1C004762
:102B10000A1B002C0A1B00110A1A00F7091A00DD13
:102B2000091900C4091900AB091900920917007BA3
:102B3000091800630917004C091600360916002011
:102B40000916000A091500F5081500E0081400CC64
:102B5000081400B8081400A4081400900813007D9D
:102B60000812006B081300580812004608120034BF
:102B7000081100230811001208110001081100F0CB
:102B8000071000E0071000D0071000C0071000B0C9
:102B9000070F00A107100091070E0083070F0074B4
:102BA000070F0065070E0057070E0049070E003B90
:102BB000070D002E070E0020070D0013070D00065D
:102BC000070D00F9060C00ED060D00E0060C00D420
:102BD000060C00C8060C00BC060C00B0060C00A4D5
:102BE000060B0099060C008D060B0082060B007781
:102BF000060B006C060B0061060A0057060B004C22
:102C0000060A0042060A0038060A002E060A0024B8
:102C1000060A001A060A001006090007060A00FD47
:102C2000050900F4050900EB050900E2050900D9D2
:102C3000050900D0050900C7050900BE050900B552
:102C4000050800AD050800A50509009C05080094CD
:102C50000508008C050800840508007C0508007440
:102C60000508006C050700650508005D05070056AE
:102C70000508004E05070047050700400508003815
:102C8000050700310507002A050700230507001C7A
:102C9000050600160507000F0507000805060002D7
:102CA000050700FB040600F5040700EE040600E833
:102CB000040600E2040700DB040600D5040600CF8A
:102CC000040600C9040600C3040600BD040600B7DC
:102CD000040600B1040500AC040600A6040600A02A
:102CE0000405009B04060095040500900406008A74
:102CF00004050085040500800406007A04050075BB
:102D0000040500700405006B0405006604050061FD
:102D10000405005C04050057040500520405004D3D
:102D200004050048040500430405003E0404003A7D
:102D300004050035040500300404002C04050027B8
:102D4000040400230405001E0404001A04040016F1
:102D5000040500110404000D040400090405000426
:102D600004040000040400FC030400F8030400F45D
:102D7000030400F0030400EC030400E8030400E48F
:102D8000030400E0030400DC030400D8030400D4BF
:102D9000030400D0030400CC030400C8030300C5EF
:102DA00003030024F404D9201BC40C5C0E9804C453
:102DB000095F0265077101F405F900FB04B30048DF
:102DC000048700C10369005803550003034500BE92
:102DD000023A008402310053022A0029022500042D
:102DE000022000E4011C00C8011900AF011700987F
:102DF00001140084011300710110006101100051E1
:102E0000010E0043010D0036010B002B010B0020C9
:102E1000010B00150109000C01090003010800FB6A
:102E2000000800F3000800EB000700E4000600DEE5
:102E3000000600D8000600D2000600CC000500C73E
:102E4000000500C2000500BD000400B9000400B583
:102E5000000400B1000400AD000400A9000400A5B6
:102E6000000300A20003009F0004009B00030098E1
:102E70000003009500020093000300900003008D02
:102E80000002008B0003008800020086000200841C
:102E9000000300810002007F0002007D0002007B31
:102EA0000002007900020077000100760002007441
:102EB00000020072000100710002006F0002006D4C
:102EC0000001006C0002006A000100690002006756
:102ED000000100660001006500010064000200625C
:102EE00000010061000100600001005F0002005D60
:102EF0000001005C0001005B0001005A0001005964
:102F00000001005800010057000100560001005563
:102F10000001005400010053000000530001005262
:102F200000010051000100500001004F0001004E5F
:102F30000000004E0001004D0001004C0001004B5C
:102F40000000004B0001004A000100490001004858
:102F50000000004800010047000100460000004654
:102F6000000100450000004500010044000100434D
:102F70000000004300010042000000420001004147
:102F800000000041000100400001003F0000003F40
:102F90000001003E0000003E0001003D0000003D39
:102FA0000001003C0000003C0000003C0001003B30
:102FB0000000003B0001003A0000003A0001003927
:102FC000000000390001003800000038000000381F
:102FD0000001003700000037000100360000003615
:102FE000000000360001003500000035000000350B
:102FF0000001003400000034000000340001003300
:1030000000000033000000330001003200000032F5
:1030100000000032000100310000003100000031EA
:103020000001003000000030000000300001002FDF
:103030000000002F0000002F0000002F0001002ED4
:103040000000002E0000002E0001002D0000002DC9
:103050000000002D0000002D0001002C0000002CBD
:103060000000002C0000002C0001002B0000002BB1
:103070000000002B0000002B0001002A0000002AA5
:103080000000002A0000002A000100290000002999
:10309000000000290000002900000029000100288C
:1030A0000000002800000028000000280000002880
:1030B0000001002700000027000000270000002773
:1030C0000000002700010026000000260000002666
:1030D0000000002600000026000100250000002559
:1030E000000000250000002500000025000000254C
:1030F000000100240000002400000024000000243F
:103100000000002400010023000000230000002331
:103110000000002300000023000000230000002323
:103120000001002200000022000000220000002216
:103130000000002200000022000100210000002108
:1031400000000021000000210000002100000021FB
:1031500000000021000100200000002000000020ED
:1031600000000020000000200000002000000020DF
:10317000000000200001001F0000001F0000001FD1
:103180000000001F0000001F0000001F0000001FC3
:103190000001001E0000001E0000001E0000001EB6
:1031A000000000C23100001C260000F4190000D805
:1031B0000F0000EB080000C0040000750200004092
:1031C000010000626564002C2073797374656D20C2
:1031D00073746F7070656421204865617465725FF7
:1031E00049443A20004265642068656174696E67ED
:1031F000206661696C65640048656174696E67206A
:103200006661696C65640042454420544845524DEE
:10321000414C2052554E4157415900546865726DDA
:10322000616C2052756E6177617900486F74656ECC
:10323000642048656174696E67206661696C6564C5
:103240000048656174696E67206661696C65640039
:10325000486F74656E6420544845524D414C20526D
:10326000554E4157415900546865726D616C20524A
:10327000756E61776179001000AD0330016A01500D
:10328000022B0170030A019004F500B005E500D09F
:1032900006D800F007CE001009C500300ABE005065
:1032A0000BB700700CB100900DAB00B00EA600D0B3
:1032B0000FA200F0109D00101299003013950050DD
:1032C00014920070158E0090168B00B0178700D0F6
:1032D000188400F0198100101B7E00301C7B005008
:1032E0001D7900701E7600901F7300B0207000D012
:1032F000216E00F0226B001024690030256600501A
:103300002663007027610090285E00B0295C00D021
:103310002A5900F02B5600102D5400302E51005029
:103320002F4E0070304B0090314800B0324500D035
:10333000334200F0343E0010363B00303737005047
:1033400038330070392E00903A2900B03B2300D06A
:103350003C1B00F03D1100103F0100F03F00004811
:103360006F74656E64204572723A204D4158544521
:103370004D50004572723A204D415854454D5020F1
:10338000424544004D415854454D50207472696780
:10339000676572656400486F74656E64204572727B
:1033A0003A204D494E54454D50004572723A204DD9
:1033B000494E54454D5020424544004D494E5445D8
:1033C0004D502074726967676572656400202F0034
:1033D0002042403A0020403A0020573A007C3C3ED0
:1033E0005E2B3D3F2F5B5D3B2C2A225C0043616ED0
:1033F0006E6F74206F70656E2073756264697220E1
:103400000053442063617264206F6B0A006F706523
:103410006E526F6F74206661696C65640A00766F26
:103420006C756D652E696E6974206661696C656482
:103430000A00534420696E6974206661696C0A0051
:103440004D3234004D323320257300577269746950
:103450006E6720746F2066696C653A20002E0A0042
:103460006F70656E206661696C65642C2046696CBE
:10347000653A20002E0A006F70656E206661696CE7
:1034800065642C2046696C653A200046696C6520AD
:1034900073656C65637465640A002053697A653AE4
:1034A000200046696C65206F70656E65643A200087
:1034B000667265736800646F696E67002066696C88
:1034C000653A20004E6F772000454E442053554208
:1034D000524F5554494E450A002220706F73002206
:1034E00020706172656E743A2200535542524F55F6
:1034F00054494E452043414C4C20746172676574B9
:103500003A2200747279696E6720746F2063616C6F
:103510006C207375622D67636F64652066696C65E6
:1035200073207769746820746F6F206D616E7920E5
:103530006C6576656C732E204D4158206C65766500
:103540006C2069733A310A006F6F6F0000004741C9
:103550004D45204F56455200107CFEFEFE4440244F
:10356000800000318000002480444004000E000EE2
:10357000007FC0FFE0FFE0FFE0FFE01FC07FF0DD65
:10358000D8FFF87FF006000F001F8036C03FC0094B
:10359000001680294006000F001F8036C03FC0166D
:1035A0008020401080104008801FC037607FF05F8F
:1035B000D050500D80104048905FD077707FF01F42
:1035C000C0104020200F007FE0FFF0E670FFF019F0
:1035D0008036C0C0300F007FE0FFF0E670FFF019CA
:1035E0008036C019800A003B20454550524F4D207F
:1035F000496E6465783A20005570646174696E673D
:10360000207A6F666673657420696E204545505256
:103610004F4D3A200001FC0007FF000F07800E010C
:10362000C00001C00000E00800E01C00E03E00E037
:103630007F00E01C00E00E00E00E01C00783C00325
:10364000FF8000FE0000FE0003FF800783C00E0124
:10365000C00E00E01C00E07F00E03E00E01C00E047
:103660000800E00000E00001C00E01C00F07800765
:10367000FF0001FC000E000E000E000E000E000EFA
:10368000000E000E007FC03F801F000E00040004EB
:10369000000E001F003F807FC00E000E000E000EC7
:1036A000000E000E000E000E00FFFFFF7F80FFC027
:1036B000FFC0FFC07F807F80FFC0FFC0FFC03F0012
:1036C0001E000C0050726F6265205A204F666673B0
:1036D0006574004C6F6164206D6D004C6F616420F7
:1036E0006D6D00556E6C6F6164206D6D00556E6C74
:1036F0006F6164206D6D00416476616E6365204B7F
:1037000000416476616E6365204B00416476616EB2
:103710006365642053657474696E677300565472F0
:103720006176206D696E005654726176206D696E07
:1037300000566D696E00566D696E00566D61782099
:103740004500566D6178204500566D6178205A001D
:10375000566D6178205A00566D6178205900566D7B
:103760006178205900566D6178205800566D617857
:10377000205800416476616E6365642053657474FB
:10378000696E677300416D6178204500416D617815
:10379000204500416D6178205A00416D6178205AC2
:1037A00000416D6178205900416D617820590041D8
:1037B0006D6178205800416D6178205800412D746A
:1037C000726176656C00412D74726176656C0041A2
:1037D0002D7265747261637400412D72657472613B
:1037E000637400416363656C00416363656C004111
:1037F0006476616E6365642053657474696E677383
:103800000056652D6A65726B0056652D6A65726B90
:1038100000567A2D6A65726B00567A2D6A65726B56
:103820000056792D6A65726B0056792D6A65726B48
:103830000056782D6A65726B0056782D6A65726B3A
:1038400000416476616E6365642053657474696ECB
:103850006773004573746570732F6D6D00457374E5
:103860006570732F6D6D005A73746570732F6D6D75
:10387000005A73746570732F6D6D005973746570A1
:10388000732F6D6D005973746570732F6D6D0058D3
:1038900073746570732F6D6D005873746570732F3A
:1038A0006D6D00416476616E636564205365747468
:1038B000696E67730046696C616D656E7400544D86
:1038C000432064726976657273004261636B6C6158
:1038D00073680053746570732F6D6D004A65726B69
:1038E00000416363656C65726174696F6E00566553
:1038F0006C6F6369747900436F6E66696775726196
:1039000074696F6E00536D6F6F7468696E670053F2
:103910006D6F6F7468696E67005A005A00590059DC
:103920000058005800436F7272656374696F6E00CF
:10393000436F7272656374696F6E004D61696E00EA
:103940004C6F61642073657474696E6773005265AF
:1039500073746F7265206661696C7361666500538C
:10396000746F72652073657474696E67730050724A
:103970006F6265205A204F666673657400416476F5
:10398000616E6365642053657474696E6773004D7E
:1039900061696E004D37303220542564004D363059
:1039A0003020423020542564004D373032203B25F2
:1039B00064004D37303120542564004368616E67E0
:1039C000652066696C616D656E740050726568652E
:1039D000617420437573746F6D0050726568656122
:1039E0007420414253005072656865617420504CE8
:1039F00041005072656865617420437573746F6D22
:103A0000004261636B00456E642066696C616D65A0
:103A10006E74206368616E6765005075726765201B
:103A20006D6F726500004368616E67696E6720465E
:103A3000696C616D656E7400554E4C4F4144204673
:103A4000494C414D454E54004C4F41442046494C51
:103A5000414D454E540020204E6F7A7A6C653A20D5
:103A60000020005061726B696E672E2E2E00746FFD
:103A70002073746172740066696C616D656E742088
:103A80006368616E6765005761697420666F7200D4
:103A900066696C616D656E7420756E6C6F61640033
:103AA0005761697420666F7200506C6561736520A0
:103AB000776169742E2E2E004E6F7A7A6C652068BD
:103AC000656174696E6700746F2068656174206E4B
:103AD0006F7A7A6C650050726573732062757474C6
:103AE0006F6E00746F20636F6E74696E7565006130
:103AF0006E6420707265737320627574746F6E00EB
:103B0000496E736572742066696C616D656E7400D0
:103B100066696C616D656E74206C6F6164005761DD
:103B2000697420666F7200746F20726573756D65BD
:103B3000207072696E7400507265737320627574C0
:103B4000746F6E00506C6561736520776169742EC7
:103B5000000066696C616D656E74207075726765D2
:103B6000005761697420666F7200536E346B3300C6
:103B7000496E76616465727300427269636B6F753A
:103B800074004D61696E003E200045787472756462
:103B9000656420746F74616C3A00256C642E25692D
:103BA0006D003E20004C6F6E67657374206A6F6213
:103BB0002074696D653A003E2000546F74616C207A
:103BC0007072696E742074696D653A00436F6D7030
:103BD0006C657465643A20005072696E7420436F9E
:103BE000756E743A200047616D6573005072696E9E
:103BF000746572205374617473004669726D7761E5
:103C000072652056657273696F6E004D61696E0052
:103C10003F0053746F70207072696E74004261636C
:103C20006B0053746F70004D323520500A4D3234A2
:103C3000005072696E742070617573656400506124
:103C4000757365207072696E7400726573756D6549
:103C5000004D3234005072696E742066726F6D20B0
:103C60005344004368616E6765205344206361726A
:103C700064004D32310041626F7574205072696E7C
:103C8000746572004368616E67652066696C616D7A
:103C9000656E74004368616E67652066696C616D6E
:103CA000656E74004D36303020423000436F6E66D2
:103CB000696775726174696F6E0054656D706572C5
:103CC0006174757265004D6F76656D656E74005236
:103CD0006573756D65207072696E740054756E65DC
:103CE0000053746F70207072696E74005061757348
:103CF00065207072696E74004E6F205344206361BA
:103D0000726400496E666F2073637265656E004D64
:103D10006F76652058004D6F76652059004D6F769F
:103D200065205A0045787472756465722000457884
:103D300074727564657220004175746F20686F6DD0
:103D40006500473238004D6F7665205A004D6F761A
:103D5000652059004D6F76652058004D6F76656D72
:103D6000656E740044697361626C6520737465707C
:103D700070657273004D3834004175746F20686F40
:103D80006D6500473238004C6576656C20582061BF
:103D9000786973004D313137204C6576656C696EFA
:103DA00067205820417869730A4732380A47302023
:103DB000583135302046393939390A4730205A359B
:103DC0002046363030300A4739310A4D3231312001
:103DD00053300A4D3430300A4D393036205A36309F
:103DE000300A4730205A2D313520463530300A47C9
:103DF00030205A3520463530300A4739300A4D34A4
:103E000030300A4D393036205A3936300A4D323189
:103E1000312053310A4732380A4D313137204C6551
:103E200076656C696E6720646F6E652E0A004D6F53
:103E300076652061786973004D61696E003F0053BB
:103E400074617274207072696E74200043616E63D5
:103E5000656C005072696E740043616E6E6F742001
:103E6000656E746572207375626469723A2000022F
:103E70002E2E004D61696E00436F6F6C646F776E1C
:103E80000046616E2073706565640046616E207344
:103E9000706565640042656400426564004E6F7A37
:103EA0007A6C65004E6F7A7A6C65004D61696E00C0
:103EB000486F74656E6400486F74656E64005A00E4
:103EC0005A005900590058005800544D432064725C
:103ED0006976657273001000C90210012C0140015F
:103EE000220170011801B0010E01F001040150021D
:103EF000FA00B002F0003003E600D003DC009004CA
:103F0000D2007005C800A006BE000008B400B009C9
:103F1000AA00D00BA000600E960060118C00001566
:103F2000820020197800C01D6E00A0226400B02716
:103F30005A00902C500000314600E0343C0010380C
:103F40003200903A2800603C1E00A03D1400803EE4
:103F50000A00203F00000000200023002600290066
:103F60002C002F00320000010000030106010901AE
:103F700000002200250028002B002E003100340014
:103F800002010000050108010B0100000A0B0209F3
:103F90000C0D0E08070304010000000000000000E3
:103FA0000000000000000000000000000000000011
:103FB00000000000000012111000000000000000CE
:103FC00000000000000000000000000000000000F1
:103FD00000000000000000000000000000000000E1
:103FE00000002100240027002A002D0030003300AB
:103FF00001010000040107010A010102102020084C
:104000000810204010204080020102010804020133
:1040100001020408102040808040201008040201A2
:1040200080040201804020100804020108040201FB
:104030000102040810204080010204081020408082
:1040400010080408801020400440801020400480A4
:1040500005050505070508080808020202020A0A04
:104060000808040404040101010101010101030322
:10407000030303030303040707070C0C0C0C0C0CCD
:104080000C0C0202020206060606060606060B0BCA
:104090000B0B0B0B0B0B07070A0A0A0A0A0A05058A
:1040A0000504040408082020506C616E6E6572429D
:1040B000756666657242797465733A2000204672AF
:1040C0006565204D656D6F72793A2000436F6D70A4
:1040D000696C65643A20536570202031203230329B
:1040E000300A00207C20417574686F723A2028469F
:1040F000616D6520334420496E632E2C204C756C15
:104100007A426F7420476974205265706F736974C6
:104110006F7279290A0000204C6173742055706415
:10412000617465643A2000322E302E302E313434E2
:104130000A004D61726C696E0020536F667477617E
:1041400072652052657365740A0020576174636854
:10415000646F672052657365740A002042726F773E
:104160006E206F75742052657365740A002045785F
:104170007465726E616C2052657365740A00506FCD
:1041800077657255700A0073746172740A00617504
:10419000746F25632E67006572726F722077726983
:1041A00074696E6720746F2066696C650A00446FDD
:1041B0006E6520736176696E672066696C652E0A8C
:1041C000004D323900456E6473746F70732025633F
:1041D00020256320256320256300205A3A002059BA
:1041E0003A0020583A00656E6473746F70732068EB
:1041F00069743A2000473238205A0A47302058382C
:104200003020593139302046333030300A4D313189
:1042100037205072696E742061626F727465642E0B
:10422000004D6F766520302E3032356D6D004D6F4C
:10423000766520302E316D6D004D6F766520316DC5
:104240006D004D6F76652031306D6D004D6F766578
:10425000206178697300486F74656E6420746F6FB5
:1042600020636F6C64004578747275646572200019
:104270004D6F7665205A004D6F76652059004D6F61
:1042800076652058000000000000000000000000DB
:10429000000000000000000000000000000000001E
:1042A00000000000000000000C0000000000000002
:1042B0000C000000000000001200000000000000E0
:1042C00023000000000000002100000000000000AA
:1042D0004C800000000000005E8000000000000034
:1042E0009240000000000000A1400000000000011A
:1042F00021200000000000027F900000000000026A
:104300000010000000000007FFF80000000000049B
:104310000008000000000008000400000000000881
:104320000006000000000010000200000000003045
:104330001E010000000000207F81000000000041FD
:10434000FFE0800000000043FCF0800000000087D8
:104350003B7840000000018EDBFC60000000010F94
:10436000EBCC20000000021FEDB610000000021F81
:10437000DEB6100000000439CD7F080000000436CE
:10438000E0FF08000000087EC0BB84000000187F2A
:10439000005D86000000107FC0ED82000000203C20
:1043A000C07301000000203B337F01000000701B40
:1043B000E77E03800000C81DEEDE04C00000880F09
:1043C000DEDC04400001240FDF3C09200001260749
:1043D000DBF8192000027203E7F01390000251018C
:1043E000FFE02290000489007F80244800090480B7
:1043F0001E004824000BFE400000DFF400100040C7
:1044000000008002001FFFFFFFFFFFFE0000000012
:10441000000000000000000000000000000000009C
:1044200000000000001022103C3C0E1F0010221063
:10443000042211040010221008221104001022107E
:10444000083C110400102210102211040010221048
:1044500020221104001E1C1E3C3C0E040000000023
:10446000000000000000000000000000000000004C
:10447000000000000000000000000000000000003C
:10448000000000000000000000000000000000002C
:10449000000000000000000000000000000000001C
:1044A000000000000000000000000000000000000C
:1044B00000000000000000000000000000000000FC
:1044C0000000004175746F6C6576656C20666169EB
:1044D0006C65640A004175746F6C6576656C206666
:1044E00061696C656400220A00556E6B6E6F776EB1
:1044F00020636F6D6D616E643A20220020746F6FCF
:10450000206C6F6E6720657874727573696F6E20AA
:1045100070726576656E7465640A0020636F6C6402
:1045200020657874727573696F6E20707265766538
:104530006E7465640A00204500205A00205900204E
:104540004D39322058002E0A006F70656E2066616A
:10455000696C65642C2046696C653A2000307800EF
:10456000486F74656E6420544845524D414C20524A
:10457000554E415741590042454420544845524DFB
:10458000414C2052554E4157415900546865726D57
:10459000616C2052756E61776179002F2F616374B1
:1045A000696F6E3A0001050800FF060121023520FF
:1045B000FFFF07FF06FF090050221656808080800B
:1045C0000080153353A0A0A00257575050F850F860
:1045D00050500257572070A0702870201335558016
:1045E000A040A02002475740A0A040A0A050251303
:1045F000538080801226564080808080401226564C
:104600008040404040800245559060F060900255E7
:10461000552020F82020113353604080044151F090
:1046200011335340E0400246561010204080801263
:10463000365640A0A0A0A04012365640C040404090
:10464000E00246566090106080F0024656F020600E
:104650001090600246562060A0F02020024656F0DE
:1046600080E01090600246566080E09090600246C4
:1046700056F01020204040024656609060909060B6
:10468000024656609090701060122555C0C000C060
:10469000C01136566060006040801236562040805F
:1046A000804020034353F000F01236568040202013
:1046B000408012365640A0204000400158583048F3
:1046C00098A8A8904030024656609090F0909002D2
:1046D0004656E090E09090E00246566090808090D0
:1046E00060024656E090909090E0024656F080E0DE
:1046F0008080F0024656F080E0808080024656605E
:104700009080B090600246569090F0909090123653
:1047100056E040404040E002465670202020A04035
:1047200002465690A0C0A0A090024656808080808D
:1047300080F002465690F0F090909002465690D04D
:10474000F0B0B0900246566090909090600246564D
:10475000E09090E08080014757609090D0B060106A
:10476000024656E09090E0909002465660904020BD
:104770009060123656E040404040400246569090CD
:1047800090909060024656909090906060024656DD
:10479000909090F0F0900246569090606090900259
:1047A0005656888850202020024656F0102040801F
:1047B000F0123656E080808080E0024656808040CD
:1047C000201010123656E020202020E016325240F1
:1047D000A0014151F0162252804002445470909042
:1047E000700246568080E09090E0123454608080E1
:1047F0006002465610107090907002445460B0C031
:1048000060024656205040E040400145556090709F
:1048100010600246568080E090909012365640001C
:10482000C04040E01137572000202020A040024621
:1048300056808090E09090123656C040404040E054
:10484000025454D0A8A8A8024454E0909090024486
:104850005460909060014555E090E080800145559E
:104860007090701010024454A0D0808012345460B4
:10487000C020C00246564040E040502002445490C0
:10488000909070123454A0A0A04002545488A8A85C
:104890005002445490606090014555909070906033
:1048A000024454F02040F0024757304020C02040DE
:1048B00030221656808080808080024757C020407A
:1048C000304020C006425250A0FFFFFFFFFFFFFF15
:1048D000FFFFFFFFFFFFFFFFFFFFFFFFFFFFFFFFE8
:1048E000FFFFFFFFFFFFFFFFFFFF090050221656EB
:1048F0008000808080800146562070A0A070200239
:1049000046562050E04050A002555588705070889F
:104910000256568850F820F82022175780808000D1
:104920008080800247577080E0907010E01731510E
:10493000A002565670A8C8C8A87014355560A0606B
:1049400000E003435350A050123353E020201431B1
:1049500051E002565670E8D8E8D870173151E0158A
:10496000335340A04012355540E04000E014355527
:1049700040A02040E0143555C020C020C01622526F
:104980004080014555909090E08002565678E8E8C6
:104990006828282411518011225240801435554036
:1049A000C04040E014355540A04000E0034353A010
:1049B00050A0024757808080A060F02002475780B7
:1049C00080A0D010207002475780408060A0F02067
:1049D00012365640004080A0400247574020609069
:1049E000F0909002475720406090F0909002475717
:1049F00060906090F0909002475750A06090F090C7
:104A00009002475790006090F09090024757609056
:104A10006090F0909002465670A0A0F0A0B00147C0
:104A200057609080809060400247574020F080E0BF
:104A300080F00247572040F080E080F00247576046
:104A400090F080E080F00247579000F080E080F026
:104A50001237578040E0404040E01237572040E096
:104A6000404040E012375740A0E0404040E012375D
:104A700057A000E0404040E00256567048E84848E1
:104A80007002475750A090D0B090900247574020F6
:104A90006090909060024757204060909090600234
:104AA00047576090609090906002475750A0609088
:104AB000909060024757900060909090601233533E
:104AC000A040A002465670B0B0D0D0E00247574098
:104AD0002090909090600247572040909090906076
:104AE00002475760909090909060024757900090D6
:104AF0009090906002575710208850202020024646
:104B00005680E09090E0800246566090A0A090A071
:104B10000247574020007090907002475720400095
:104B2000709090700247572050007090907002472C
:104B30005750A000709090700246565000709090B0
:104B40007002475760906070909070025454F06803
:104B5000B078113555608080604002475740200092
:104B600060B0C06002475720400060B0C06002479C
:104B70005760900060B0C060024656500060B0C000
:104B800060123757804000C04040E0123757204045
:104B900000C04040E012375740A000C04040E01243
:104BA0003656A000C04040E0024757A040A0107019
:104BB000906002475750A000E09090900247574005
:104BC0002000609090600247572040006090906005
:104BD0000247576090006090906002475750A000D5
:104BE000609090600246569000609090601235553B
:104BF0004000E0004002445470B0D0E0024757400B
:104C00002000909090700247572040009090907044
:104C10000247576090009090907002465690009026
:104C2000909070014858204000909070906001472B
:104C3000578080E090E0808001475790009090700E
:104C4000906001050700FE0500FB01F220FFFE0554
:104C5000FE05FE020040021525808080008005329E
:104C600042A0A002556550F850F8500146562070F9
:104C7000C030E02002556590102040480255656024
:104C800080689068051222808002253540808080EF
:104C9000400225358040404080043343A040A003BB
:104CA000334340E0400122324080043141E00211B0
:104CB0002180025565081020408002455560909083
:104CC0009060022535C040404040024555E01060EC
:104CD00080F0024555E0106010E00245552060A0CC
:104CE000F020024555F080E010E00245556080E07C
:104CF0009060024555F0102040400245556090609C
:104D0000906002455560907010600313238000800E
:104D1000021424800080800235452040804020031A
:104D20003343E000E0023545804020408002455595
:104D3000E0106000400255657088B8A870024555C3
:104D4000609090F090024555E090E090E00235458B
:104D50006080808060024555E0909090E00235458B
:104D6000E080E080E0023545E080E080800245554B
:104D70007080B090700245559090F090900235454B
:104D8000E0404040E002455530101090600245552B
:104D900090A0C0A09002354580808080E0025565DB
:104DA00088D8A8888802455590D0B0909002455583
:104DB0006090909060024555E09090E080014656EA
:104DC000609090906010024555E09090E090024510
:104DD0005570806010E0023545E04040404002459B
:104DE0005590909090600245559090A0A04002553B
:104DF0006588A8A8A85002455590906090900245FB
:104E0000559090701060023545E0204080E002250A
:104E100035C0808080C00255658040201008022582
:104E200035C0404040C005324240A0024151F0052B
:104E3000223280400244547090907002455580E0C8
:104E40009090E0023444608080600245551070907C
:104E5000907002445460B0C0600235452040E0408C
:104E60004000465670909070106002455580E0906A
:104E700090900215258000808080002737400040F8
:104E8000404040800245558090A0E090021525806A
:104E900080808080025464F0A8A8A8024454E09066
:104EA000909002445460909060004656E09090E0EC
:104EB0008080004656709090701010023444A0C05C
:104EC000808002445470C030E002354540E04040EC
:104ED00020024454909090700244549090A040025C
:104EE0005464A8A85050023444A04040A000465644
:104EF000909090701060024454F02040F0023545CC
:104F000060408040600215258080808080023545A9
:104F1000C0402040C005425250A0FFFFFFFFFFFFEE
:104F2000FFFFFFFFFFFFFFFFFFFFFFFFFFFFFFFF91
:104F3000FFFFFFFFFFFFFFFFFFFFFF020040FFFF3C
:104F4000FFFFFFFFFFFFFFFFFFFFFFFFFFFFFFFF71
:104F5000FFFFFFFFFFFFFFFFFFFFFFFFFFFFFFFF61
:104F6000FFFFFFFFFFFFFFFFFFFFFFFFFFFFFFFF51
:104F7000FFFFFFFFFFFFFFFFFFFFFFFFFFFFFFFF41
:104F8000FFFFFFFFFFFFFFFFFFFFFFFFFFFFFFFF31
:104F9000FFFFFFFFFFFFFFFFFFFFFFFFFF01060D0A
:104FA00000FE09016602D620FFFE0BFE0AFE0D0080
:104FB000602219698080808080808000801833633F
:104FC000A0A0A00357675050F850F85050025969FC
:104FD0002078A0A0702828F02002596948A8501015
:104FE000204050A89002586840A0A040A098906827
:104FF000281363808080113B6B204040808080803C
:1050000080404020113B6B804040202020202040E9
:10501000408006556520A870A8200455652020F81A
:105020002020113363604080065161F811336340E2
:10503000E040025969080810102040408080025961
:10504000692050888888888850200259692060A08B
:105050002020202020F802596970888808102040FC
:1050600080F8025969F80810207008088870025901
:1050700069101030505090F81010025969F8808073
:10508000B0C80808887002596970888080F08888E4
:105090008870025969F808101020204040400259D9
:1050A00069708888887088888870025969708888D3
:1050B00088780808887011386840E040000040E0B7
:1050C0004011386840E040000060408002596908A3
:1050D0001020408040201008045464F80000F802BA
:1050E000596980402010081020408002596970885A
:1050F0008808102020002002596970888898A8A884
:10510000B080780259692050888888F88888880299
:105110005969F048484870484848F0025969708811
:1051200080808080808870025969F04848484848EB
:105130004848F0025969F8808080F0808080F80249
:105140005969F8808080F080808080025969708879
:105150008080809888887002596988888888F88853
:10516000888888123969E040404040404040E00271
:105170005969381010101010109060025969888811
:1051800090A0C0A09088880259698080808080802B
:105190008080F80259698888D8A8A88888888802F9
:1051A000596988C8C8A8A8989888880259697088D9
:1051B00088888888888870025969F0888888F08093
:1051C000808080015A6A70888888888888A87008DA
:1051D000025969F0888888F0A0908888025969701F
:1051E0008880807008088870025969F82020202083
:1051F00020202020025969888888888888888870BB
:10520000025969888888885050502020025969883E
:10521000888888A8A8A8A850025969888850502072
:1052200050508888025969888850502020202020BA
:10523000025969F808101020404080F8113B6BE0DB
:10524000808080808080808080E0025969808040FA
:10525000402010100808113B6BE020202020202067
:10526000202020E0085363205088015161F82A2251
:105270006280400256667008788898680259698092
:105280008080F088888888F00256667088808088E0
:1052900070025969080808788888888878025666F4
:1052A0007088F880887002596930484040F040406A
:1052B000404000586870888888780888700259696A
:1052C000808080B0C8888888881238684000C040D4
:1052D000404040E0004A6A100030101010109090DA
:1052E0006002596980808090A0C0A09088123969BE
:1052F000C040404040404040E0025666D0A8A8A8C8
:10530000A888025666B0C888888888025666708861
:1053100088888870005868F0888888F080808000CD
:1053200058687888888878080808025666B0C88067
:1053300080808002566670886010887002586840CD
:1053400040F0404040483002566688888888986817
:105350000256668888885050200256668888A8A819
:10536000A8500256668850202050880058688888C7
:10537000889868088870025666F810204080F80106
:105380005B6B1820202020C02020202018221969C3
:10539000808080808080808080015B6BC0202020A6
:1053A000201820202020C008536348A890FFFFFF4A
:1053B000FFFFFFFFFFFFFFFFFFFFFFFFFFFFFFFFFD
:1053C000FFFFFFFFFFFFFFFFFFFFFFFFFFFF0D00DE
:1053D0006022196980008080808080808003586806
:1053E0002070A8A0A0A8702002596930484040E071
:1053F000404048B003566688705050708802596922
:1054000088885050F820F8202022196980808080F8
:105410000080808080124A6A609080609090601066
:1054200090601A3262A0A00359697088A8D8C8D8C1
:10543000A88870045767700878887800F803566663
:105440002850A0A05028045363F80808163161E0E2
:105450000359697088E8D8D8E8D888700A5161F88B
:10546000174464609090600357672020F820200064
:10547000F807356540A02040E007356540A0402092
:10548000C02A226240800058688888888898E8800E
:105490008002596978E8E8E8E86828282826216128
:1054A000C0202262408007356540C04040E004577C
:1054B00067708888887000F8035666A050282850C6
:1054C000A0025A6A40C04040E00818283808025A32
:1054D0006A40C04040E01028081038025A6A40A0D4
:1054E0004020A04818283808025969200020204090
:1054F00080888870025A6A40200020508888F88886
:1055000088025A6A10200020508888F88888025A39
:105510006A30480020508888F88888025A6A2850E3
:105520000020508888F88888025A6A50500020501D
:105530008888F88888025A6A20502020508888F885
:10554000888802596958A0A0A0B0E0A0A0B8005B6C
:105550006B7088808080808088702040025A6A400A
:105560002000F88080F08080F8025A6A102000F84D
:105570008080F08080F8025A6A304800F88080F01D
:105580008080F8025A6A505000F88080F08080F8DD
:10559000123A6A804000E04040404040E0123A6ADF
:1055A000204000E04040404040E0124A6A609000E5
:1055B000E04040404040E0123A6AA0A000E0404095
:1055C000404040E0025969F0484848E8484848F0FF
:1055D000025A6A2850008888C8A8988888025A6A9F
:1055E00040200070888888888870025A6A102000DD
:1055F00070888888888870025A6A30480070888865
:1056000088888870025A6A2850007088888888883C
:1056100070025A6A505000708888888888700355D4
:10562000658850205088015B6B08709898A8A8A8DE
:10563000C8C87080025A6A40200088888888888894
:1056400070025A6A10200088888888888870025AF8
:105650006A30480088888888888870025A6A505062
:105660000088888888888870025A6A102000888894
:10567000502020202002596980F0888888F080809E
:1056800080025969609090A0A0908888B002596902
:1056900040200070087888986802596910200070CE
:1056A00008788898680259693048007008788898A6
:1056B000680259692850007008788898680259690A
:1056C000505000700878889868025A6A3048300054
:1056D000700878889868025666702870A0A85000F4
:1056E0005868708880808870204002596940200086
:1056F0007088F88088700259691020007088F880DE
:1057000088700259693048007088F88088700259A2
:10571000695050007088F8808870123969804000A4
:10572000C040404040E0123969204000C040404045
:1057300040E0124969609000C040404040E01239AA
:1057400069A0A000C040404040E0025A6A5020607A
:1057500010708888888870025969285000B0C888FD
:10576000888888025969402000708888888870027B
:1057700059691020007088888888700259693048FB
:10578000007088888888700259692850007088885D
:105790008888700259695050007088888888700322
:1057A0005767202000F8002020015868087098A84A
:1057B000A8C8708002596940200088888888986845
:1057C00002596910200088888888986802596930D1
:1057D00048008888888898680259695050008888ED
:1057E00088889868005B6B10200088888898680813
:1057F0008870005A6A8080B0C88888C8B0808000ED
:105800005B6B505000888888986808887000060C88
:1058100000FE07022603BC017FFE08FE08FE050805
:105820000806000040F0C888889878100508080627
:105830000000C0F88888888888F8050505060001FA
:105840002030F830200508080600002070F82020DD
:105850002020E00509090600FF2070A8A8B8888864
:105860007020050606060001E08CEA8C8A0A05090C
:10587000090600FFF8A88888888888A8F8050A0A19
:105880000600FE205050505088A8A88870030303DB
:1058900006000340A040FFFFFFFFFFFFFFFFFFFFE9
:1058A000FFFFFFFFFFFFFFFFFFFFFFFF00000006FE
:1058B00005FF0107070602008080808080008003CA
:1058C0000303060105A0A0A005060606000050F887
:1058D0005050F8500509090600FF2070A8A0702854
:1058E000A87020050707060000C8C8102040989837
:1058F00005070706000040A0A040A8906801030328
:105900000602058080800309090601FF20404080CF
:1059100080804040200309090601FF80404020208C
:105920002040408005070706000020A8702070A8CE
:10593000200505050600012020F8202002030306AB
:1059400001FFC04080050101060003F802020206C3
:105950000100C0C0050707060000081010204040E5
:1059600080050707060000708898A8C8887003079C
:105970000706010040C040404040E0050707060020
:1059800000708808102040F8050707060000F80896
:10599000103008887005070706000010305090F896
:1059A0001010050707060000F880F0080888700549
:1059B0000707060000304080F0888870050707065A
:1059C0000000F808101020202005070706000070CE
:1059D00088887088887005070706000070888878B6
:1059E000081060020505060100C0C000C0C0020624
:1059F000060601FFC0C000C0408003050506010186
:105A00002040804020050303060002F800F803054B
:105A10000506010180402040800507070600007050
:105A20008810202000200507070600007088B8A80D
:105A3000B88070050707060000708888F888888895
:105A4000050707060000F04848704848F0050707BA
:105A500006000070888080808870050707060000B7
:105A6000F04848484848F0050707060000F88080DD
:105A7000F08080F8050707060000F88080F080803D
:105A800080050707060000708880809888700507E9
:105A900007060000888888F88888880307070601B9
:105AA00000E04040404040E0050707060000381095
:105AB00010101090600507070600008890A0C0A095
:105AC0009088050707060000808080808080F805A8
:105AD000070706000088D8A8888888880507070671
:105AE00000008888C8A89888880507070600007005
:105AF000888888888870050707060000F08888F085
:105B000080808005070706000070888888A8906854
:105B1000050707060000F08888F0A09088050707B1
:105B2000060000708880700888700507070600006E
:105B3000F8202020202020050707060000888888FC
:105B40008888887005070706000088888888505074
:105B50002005070706000088888888A8A850050740
:105B6000070600008888502050888805070706002F
:105B70000088885020202020050707060000F8082C
:105B800010204080F80309090601FFE08080808032
:105B9000808080E00507070600008040402010104C
:105BA000080309090601FFE020202020202020E032
:105BB0000503030600052050880501010600FEF8D4
:105BC000030303060105804020050505060000705B
:105BD000087888780507070600008080F0888888A4
:105BE000F00505050600007080808870050707062F
:105BF0000000080878888888780505050600007088
:105C000088F08070050707060000304840E04040FB
:105C1000400507070600FE70888888780870050729
:105C2000070600008080F08888888803070706013F
:105C3000004000C0404040E00409090601FE100099
:105C40003010101010906005070706000080808853
:105C500090E09088030707060100C04040404040A4
:105C6000E0050505060000D0A8A8A8A805050506BA
:105C70000000B0C88888880505050600007088887F
:105C800088700507070600FEF0888888F080800588
:105C900007070600FE788888887808080505050645
:105CA0000000B0C88080800505050600007880707F
:105CB00008F00507070600002020F820202018051E
:105CC0000505060000888888986805050506000017
:105CD00088888850200505050600008888A8A850F7
:105CE00005050506000088502050880507070600B6
:105CF000FE88888850204080050505060000F810C1
:105D00002040F80309090601FF2040404080404040
:105D100040200109090602FF808080808080808009
:105D2000800309090601FF80404040204040408038
:105D300005030306000248A890FF640248011124ED
:105D40001FBECFEFD1E2DEBFCDBF00E00CBF13E03E
:105D5000A0E0B2E0ECE0FCED02E00BBF02C0079077
:105D60000D92AC3DB107D9F729E1ACEDB3E001C02C
:105D70001D92A832B207E1F71EE2CEE9DEE200E0B2
:105D800006C021970109802FFE010F946A6DCD395D
:105D9000D10780E00807A9F70F943F5A0D94F46DDE
:105DA0000C940000089590E080E0089590913B09E4
:105DB000E92FF0E0E45BF94E80839F5F953040F47B
:105DC00090933B0980911F0B8F5F80931F0B089569
:105DD00010923B09F7CF8F929F92AF92BF92CF92D2
:105DE000DF92EF92FF92CF934B015C0169017A0140
:105DF00022ED30E040EA50ECC701B6010F94846C0C
:105E000087FD48C027E030E044E353E4C701B60112
:105E10000F94CD6518160CF43DC029E630E040E142
:105E200051ECC501B4010F94846C87FD33C027E0A9
:105E300030E04CE253E4C501B4010F94CD6518166F
:105E40004CF123EA31E040E450ECC501B4010F9479
:105E5000846C87FD1FC027E030E043E253E4C501B6
:105E6000B4010F94CD651816ACF022ED30E040E897
:105E700050ECC701B6010F94846C87FD0BC0C1E0E4
:105E800027E030E048E253E4C701B6010F94CD6546
:105E900018160CF4C0E08C2FCF91FF90EF90DF909C
:105EA000CF90BF90AF909F908F9008952FEB280FC9
:105EB0002A3108F042C0E22FF0E080916B0590910A
:105EC0006C05A0916D05B0916E0504C0B695A795BF
:105ED000979587952A95D2F780FD02C08170089525
:105EE000EF5AFA4FE081EE2329F18091B50B9091A2
:105EF000B60BE80FF92FF11D808190ED980F9A30C5
:105F000030F08E3251F4818180538A3098F4F093CE
:105F10004004E0933F0481E008958D3211F08B320C
:105F200049F4818190ED980F9A3088F38E3211F404
:105F30008281EACFF0E0E0E0EACF80E008950E94BD
:105F4000562F882341F081E020913F043091400496
:105F5000232B09F480E00895CF92DF92EF92FF9215
:105F60000F931F93CF93DF9300D000D01F921F9207
:105F7000CDB7DEB7DC01ED91FC910084F185E02D19
:105F80001995AB01BC01072F11272227332749831D
:105F90005A836B837C836801790192E0F694E794DD
:105FA000D794C7949A95D1F78D81C0FA80F968018A
:105FB0007901F694E794D794C794C0FA81F98D8358
:105FC00068017901B8E1CB22DD24EE24FF2481E0D1
:105FD000CD28CE28CF2809F480E09D8180FB92F95E
:105FE00000FB94F956FB882780F980FB95F907FBA5
:105FF00096F907FB97F99058862F8F71FA01F37085
:10600000F887EF8329813A814B815C81692F782F52
:106010008E2F988528960FB6F894DEBF0FBECDBFA1
:10602000DF91CF911F910F91FF90EF90DF90CF9074
:106030000895DF92EF92FF920F931F93CF93DF9318
:10604000EC01D62E1CAD0BAD7C0184E0E80EF11CFA
:10605000E98DFA8DC7011995412F480F2D2D602F1D
:10606000C7010E948A9D9BAD890F8BAF81E090E0B4
:10607000DF91CF911F910F91FF90EF90DF900895E6
:106080008F929F92AF92BF92CF92DF92EF92FF9248
:106090000F931F93CF93DF93EC018B017A018A85D5
:1060A0009B858617970731F0888199810E94429CD1
:1060B0001B870A87888599850196F9F46A818E8104
:1060C000680F97014C81888199810E94F69D2E81ED
:1060D0003F81820F932F911D9F838E8390E080E0FC
:1060E000DF91CF911F910F91FF90EF90DF90CF90B4
:1060F000BF90AF909F908F900895CE80DF80F70182
:10610000008110E0002309F1A880B980602FC5014B
:106110000E949A9CF501118911954701FFEF8F1A92
:106120009F0AF40181914F01F501882341F0908984
:10613000190F082F682FC5010E949A9CF2CF0032D8
:1061400079F083899189890F180FC10ED11C288598
:1061500039852C153D0508F0B1CF81E090E0C0CF26
:106160008089F2CFCF93DF93EC01FE0184912196D9
:10617000882319F00F944023F8CFDF91CF91089531
:106180000F931F93CF93C62F8C01F80181918F013C
:10619000882331F0CC2321F00F944023C150F5CF58
:1061A000CF911F910F910895CF93DF93EC018991C7
:1061B000882319F00F944023FACFDF91CF910895EF
:1061C0002F923F924F925F927F928F929F92AF92C7
:1061D000BF92CF92DF92EF92FF920F931F93CF93D4
:1061E000DF93D62EC72E742EFC0180809180A28072
:1061F000B380C501B40120E13EE040E050E00F94DF
:10620000C069122F032FC22FD32F8CE3282E312CDD
:10621000412C512CC501B401A20191010F94C06918
:10622000CA01B901A20191010F94C069F62EE72EAF
:10623000772051F1C501B40120E831E541E050E09B
:106240000F94C0698901EF92FF92CE0168E170E07E
:106250000F94426D9F938F933F932F938BEB9AE014
:106260009F938F93CF92DF920F946465EDB7FEB743
:106270003A960FB6F894FEBF0FBEEDBF88E00A3025
:106280001105D0F089E018C0C436D10538F57F93E8
:106290006F930F931F9381EB9AE09F938F93CF920D
:1062A000DF920F9464658DB79EB708960FB6F89489
:1062B0009EBF0FBE8DBF85E0DF91CF911F910F91E3
:1062C000FF90EF90DF90CF90BF90AF909F908F9016
:1062D0007F905F904F903F902F9008957F936F93A2
:1062E0000F931F9389EA9AE09F938F93CF92DF9247
:1062F0000F946465EDB7FEB738960FB6F894FEBFFD
:106300000FBEEDBF86E0D8CF0E949ED920915D06DA
:1063100091E0821301C090E0821380935D06892F83
:10632000089580913F0490914004009731F04AE035
:1063300050E070E060E00D94CC6260E070E0CB0172
:106340000895CF93DF93EB010E949F2F882319F0CC
:106350000E949131EB01CE01DF91CF9108950E940F
:106360009131CB010895CF93DF93EB010E949F2FD2
:10637000882321F0DF91CF910C94AF31CE01DF91D2
:10638000CF9108950E94913197FD0CC00E949131E8
:106390006F3F71058105910509F034F40E94913138
:1063A000862F089580E008958FEF0895CF93C62F2C
:1063B0000E949F2F882319F0CF910C94C2318C2F0B
:1063C000CF91089580913F0490914004892B41F032
:1063D0000E94C23191E0811101C090E0892F08959F
:1063E00091E0FCCFCF93DF93C82FD62F0E949F2F31
:1063F000882321F0DF91CF910C94E2318C2F0E9401
:10640000562F811101C08D2FDF91CF910895CF922A
:10641000DF92EF92FF920F931F93CF93DF938B0145
:10642000CAE5D2E020916E0230916F024091700275
:1064300050917102FC0160817181828193810F947E
:106440001E6B2C853D854E855F850F94246A6C8775
:106450007D878E879F87C12CD12C760126E632E07E
:1064600042E652E06EE572E0CE010F94F53EDF9118
:10647000CF911F910F91FF90EF90DF90CF900C94F0
:1064800076BE80E1EAE5F2E0A4E8B6E001900D9284
:106490008A95E1F70895CF92DF92EF92FF920F93E2
:1064A0001F93CF9390913C02913009F461C0662311
:1064B00051F010922E0410922A0410922B04109284
:1064C0002C0410922D04C82F0F94054CC0902A0460
:1064D000D0902B04E0902C04F0902D049B01AC0193
:1064E0002C193D094E095F0969017A01F7FC40C08A
:1064F00020912E04C7FD15C04C2F0C2E000C550BFF
:106500004C5F5F4FE22F022E000CFF0B4E175F0710
:106510007CF144EFC42EDD24D394E12CF12C2C1714
:1065200034F438EEC32E33E0D32EE12CF12CC60E1A
:10653000D71EE81EF91EC0922A04D0922B04E092C6
:106540002C04F0922D04022F017010E084E2809F51
:10655000B001819F700D701B112460597C4F82E344
:1065600090E00E94FFD880912E048F5F80932E04CC
:10657000CF911F910F91FF90EF90DF90CF900895F2
:1065800080913F0490914004009731F04AE050E040
:1065900070E060E00D94FA6360E070E0CB01089574
:1065A0000F931F93CF9380913F04909140040097E5
:1065B000E9F0FC018F01C1912C2F2F7D81F0C534B2
:1065C00011F0C536B9F7F801108270E060E00F9461
:1065D0006E61F801C083CF911F910F91089570E013
:1065E00060E0CF911F910F910D946E6160E070E0BB
:1065F000CB01F1CFCF92DF92EF92FF926A017B0144
:106600000E949F2F882331F0FF90EF90DF90CF9072
:106610000C94D032C701B601FF90EF90DF90CF907D
:106620000895CF92DF92EF92FF920F931F93CF9333
:10663000DF9380E8C82E82E0D82E94E8E92E96E019
:10664000F92E0AE512E0D0E0C0E0F60181916F0179
:106650000E949F2F882309F473C00E94D032FE014C
:10666000E95BFA4F2081211104C020914F052223BC
:1066700039F0F80120813181428153810F94246ADD
:10668000F70160837183828393832196F4E0EF0E98
:10669000F11C0C5F1F4FC430D105B9F640E050E04B
:1066A000BA0186E40E94FA3220E030E0A9010F949A
:1066B000846C181684F40E94D03220E030E040E769
:1066C00052E40F941E6B60935602709357028093AE
:1066D0005802909359028091641183FD28C08091E3
:1066E0002609882321F120916602309167024091AA
:1066F00068025091690260919006709191068091B4
:106700009206909193060F94236A20913309309159
:10671000340940913509509136090F94246A6093E9
:106720003309709334098093350990933609DF91CA
:10673000CF911F910F91FF90EF90DF90CF90089530
:10674000F80180819181A281B381F70180839183D7
:10675000A283B3839ACF9091B70B9817D1F00E9480
:1067600076BE8091B70B882361F042E652E06EE579
:1067700072E08AE592E00E9449CC1092B70B0C942B
:1067800073C581E08093B70B8AE592E00E94B0CC9C
:10679000F6CF08955A9887FD44C05B98000000002A
:1067A000000000005A9A5A9886FD47C05B98000086
:1067B0000000000000005A9A5A9885FD3CC05B9882
:1067C00000000000000000005A9A5A9884FD31C071
:1067D0005B9800000000000000005A9A5A9883FD60
:1067E00026C05B9800000000000000005A9A5A98EA
:1067F00082FD1BC05B9800000000000000005A9A58
:106800005A9881FD10C05B98000000000000000055
:106810005A9A5A985B9800000000000000005A9AAB
:1068200008955B9ABBCF5B9AEFCF5B9AE4CF5B9AFC
:10683000D9CF5B9ACECF5B9AC3CF5B9AB8CF0F9379
:106840004CE0849F402D112421E0240F2093220846
:106850008CE0840F80939E0B90E002963091461658
:106860003817190621F01CF080E00F9108958091EF
:1068700048162817C8F781E080933216662351F036
:106880004D5F0BE020E860E082E196E10F94C65591
:106890001092321680919E0B90914616891720F324
:1068A00020914816909122082917F0F2109249166B
:1068B00080934A1681E0D9CFEF92FF920F9380E048
:1068C000E82E81E2F82E03E127E047E064E282E16E
:1068D00096E10E94219E0F9489272BE433E04BE23E
:1068E00065E282E196E10E94F69D25E533E047E30B
:1068F00067E082E196E10F91FF90EF900C94F69D96
:10690000EF92FF920F931F93CF93DF93CDB7DEB734
:106910002C970FB6F894DEBF0FBECDBF6F3F710549
:106920008105910509F0C0F48EE096E10E941930CE
:10693000E0911616F09117163196849190E02C96FE
:106940000FB6F894DEBF0FBECDBFDF91CF911F9180
:106950000F91FF90EF9008951091491600914A16FB
:1069600020916A0621110FC040EE50E2602F812F66
:106970000F94622720E030E0120F10934916009325
:106980004A16C901DCCFE0901616F090171622E1E6
:1069900036E13A832983212F30E03C832B83202F5B
:1069A00030E03E832D8318861F822FEF3FEF3A871A
:1069B00029871C861B869E012F5F3F4FAB01BC01C0
:1069C000C7010F946726B70182E196E10E94429CBD
:1069D0002F813885D1CFCF93DF93FC0125AD2111D5
:1069E00004C021E025AF0F940654C0911416D09135
:1069F0001516E0914316F091441682E01995E09146
:106A00004316F091441681E0199530E020E044E10E
:106A1000BE0182E196E10F94025425E436E147E19C
:106A2000BE0182E196E10F940254E0914316F09189
:106A3000441680E0DF91CF91199480916B06982FD6
:106A40009370913059F081608D7F80936B068AEF4F
:106A50000E94CA3388E28A950000E9F70895CF932F
:106A6000C82F80916B06982F9370933059F08160F6
:106A7000826080936B0688EF0E94CA3388E28A9511
:106A80000000E9F78C2FCF910D944023CF93DF9333
:106A900090916B0692FB222720F92817C9F0D1E0CC
:106AA000392F387093FFD0E020E2811124E292E088
:106AB000311101C090E0C82F822F892B0E942F3501
:106AC00080916B06C0FB82F9D0FB83F980936B0643
:106AD000DF91CF91089586E20E942F3580916B0659
:106AE0008460886080936B0686E20E942F358091D7
:106AF0006B068460886080936B0681E00E94463557
:106B000082E00E942F3580916B068F7E80936B060A
:106B10000895EF92FF920F931F93CF93DF93C82FA7
:106B20007B0180E00E9446358C2F80640E942F35C7
:106B30000E941D35D0E0C0E0F701EC0FFD1F05916C
:106B40001491812F0F944023802F0F94402322967D
:106B5000C032D10589F7DF91CF911F910F91FF903E
:106B6000EF90089580E00E94463581E00E942F3525
:106B70006FE070E080E090E00D94D24BCF93DF9314
:106B8000C82FD62F81E00E9446358D2F80680E9445
:106B90002F358C2F8F708068DF91CF910C942F351B
:106BA000CF92DF92EF92FF920F931F93CF93DF93D9
:106BB000C42E982F9170D92ED82FD695F62EF294F8
:106BC00080EFF82208EC10E2C1E0F801E4906F2DAC
:106BD0006C0F8D2F0E94BE350E941D35CC20C9F050
:106BE0008E2DD11080E00F944023D11001C0E12CF4
:106BF0008E2D0F944023CF5F0F5F1F4FC53029F7B5
:106C0000DF91CF911F910F91FF90EF90DF90CF9088
:106C1000089580E00F94402380E0EBCF1F93CF9343
:106C2000DF93182FC62FD1E0D627611104C08BED5A
:106C300090E20E94B2304D2F612F85E00E94D03546
:106C40004C2F612F89E0DF91CF911F910C94D035AB
:106C5000DF92EF92FF920F931F93CF93DF93D82E83
:106C6000C62FC295C07F8A01D0E1DC0F6C2F8D2D1D
:106C70000E94BE350E941D35F801E590F4908F2DDD
:106C80000F9440238E2D0F9440230E5F1F4FCF5F34
:106C9000DC13ECCFDF91CF911F910F91FF90EF901C
:106CA000DF900895CF93C82F80E00E9446358C2F47
:106CB0008068CF910C942F351F93CF93DF9388E199
:106CC0000E9452360E941D3587E793E10F941E23E0
:106CD000C82F813158F487E793E10E94D430C03146
:106CE000B1F180E20F944023CF5FF9CFC0917613CA
:106CF000D0E0C958DC4ECE010F941E23182F60E15E
:106D0000CE010E94C030103178F48EE20F944023FF
:106D10001F3051F08EE20F9440236EE0611B21F092
:106D200087E793E10E94C03087E793E10F941E2329
:106D300090917613981778F49F5FE92FF0E0E95867
:106D4000FC4E8081807C8038B9F390937613DF917C
:106D5000CF911F91089510927613F9CF5D9A88E232
:106D60008A950000E9F780916B068E7F80936B0611
:106D70000895EF92FF920F931F93CF93DF93CDB7B8
:106D8000DEB72C970FB6F894DEBF0FBECDBF1091C3
:106D9000491600914A1620916A0621111AC048EA44
:106DA00050E2602F812F0F94622780E090E0180F4F
:106DB0001093491600934A162C960FB6F894DEBF2E
:106DC0000FBECDBFDF91CF911F910F91FF90EF903C
:106DD0000895E0901616F090171622E136E13A83F6
:106DE0002983212F30E03C832B83202F30E03E830A
:106DF0002D8318861F827A8769871C861B869E01D1
:106E00002F5F3F4F4EEF5FEEBC01C7010F94272766
:106E1000B70182E196E10E94429C8F819885C7CF9D
:106E20006FEF7FEF0C94B936EF92FF920F931F93A1
:106E3000CF93DF93CDB7DEB72C970FB6F894DEBFB4
:106E40000FBECDBF1091491600914A1620916A06D7
:106E500021111AC048E850E2602F812F0F94622759
:106E600080E090E0180F1093491600934A162C9674
:106E70000FB6F894DEBF0FBECDBFDF91CF911F914B
:106E80000F91FF90EF900895E0901616F09017166E
:106E900022E136E13A832983212F30E03C832B83A2
:106EA000202F30E03E832D8318861F827A876987E2
:106EB0001C861B869E012F5F3F4F41E050EFBC01B7
:106EC000C7010F942727B70182E196E10E94429CF7
:106ED0008F819885C7CFEF92FF920F931F93CF9327
:106EE000DF937B01C42F622F0E941F348823D1F1CE
:106EF000CC23F9F001151105E1F4C7010F94FC2230
:106F000025E130E0A901481B5109CA0157FD01964E
:106F100095958795C0E8DFE7D80F8D2F8C0F87FDFB
:106F200009C060E270E080E090E00E948034C150CF
:106F3000F4CFC0E86C2F70E0C7010E94B936C81BBF
:106F40000115110531F06C2F70E0C8010E94143753
:106F5000C81BC73038F060E270E080E090E00E942B
:106F60008034F6CFDF91CF911F910F91FF90EF907A
:106F700008956FEF7FEF0C941437AF92BF92CF92CA
:106F8000DF92EF92FF920F931F93CF93DF935C01F9
:106F90006B010F94FC22E82EC6010F941E23F12CE6
:106FA00003E110E0081B1109C5E20E151F050CF4E2
:106FB000CFE18C2F90E09C012E5F3F4F4091461611
:106FC0004217130609F094F50997209148162817DF
:106FD000190664F110924916C0934A16C5010E9421
:106FE0001037D1E0C114D104B1F06AE370E080E061
:106FF00090E00E9480340E151F05D4F4C45F809188
:107000004616C81740F0209148164C2F4950550B92
:10701000241715067CF4DF91CF911F910F91FF90FB
:10702000EF90DF90CF90BF90AF900895D0E0DACF8F
:10703000DD2389F3802F880F080F000F0093491676
:10704000C0934A1660E270E080E090E00E948034D5
:10705000C601DF91CF911F910F91FF90EF90DF90CC
:10706000CF90BF90AF900C94B937CF92DF92EF9250
:10707000FF920F93CF93DF93982F862F6A017901A8
:10708000692F0E941F34882309F448C0C7010023D8
:1070900009F10F94FC22C82F83E190E08C1B910929
:1070A000D82FDD0FD80FDD0F6D2F70E0C6010E94C5
:1070B000B936D81B6AE370E080E090E00E9480342B
:1070C000D73058F060E270E080E090E00E948034B9
:1070D000D81BF6CF0F941E23DECF80919E0B9C2FE2
:1070E000990F990FC91BCC0FC058C09349168093B4
:1070F0004A16C701002349F0DF91CF910F91FF900D
:10710000EF90DF90CF900C941037DF91CF910F91DB
:10711000FF90EF90DF90CF900C94B937DF91CF9133
:107120000F91FF90EF90DF90CF900895CF92DF9274
:10713000EF92FF926C01990FEE08FF084AE0C70139
:10714000B601F7FE0DC06DE28EE096E10E941930A7
:1071500066277727CB016C197D098E099F094AE0C4
:10716000FF90EF90DF90CF900D94EA422F923F92E4
:107170004F925F926F927F928F929F92AF92BF9247
:10718000CF92DF92EF92FF920F931F93CF93DF93F3
:10719000EB01FC0180809180A280B380C501B40125
:1071A00020E831E541E050E00F94C069C9016DE687
:1071B00071E00F94426D6B017C01C501B40120E1C7
:1071C0003EE040E050E00F94C069CA01B90128E1F7
:1071D00030E040E050E00F94C069362E272E062F95
:1071E000172F8CE3482E512C612C712CC501B40152
:1071F000A30192010F94C069B62EA72ECA01B9014E
:10720000A30192010F94C069CB01C114D10469F1AB
:10721000AF92BF927F936F932F923F92FF92EF9224
:10722000DF92CF9285E69EE19F938F93DF93CF937A
:107230000F9464658DB79EB70E960FB6F8949EBFF7
:107240000FBE8DBFDF91CF911F910F91FF90EF90F7
:10725000DF90CF90BF90AF909F908F907F906F9076
:107260005F904F903F902F900895E114F104C9F082
:10727000AF92BF927F936F932F923F92FF92EF92C4
:1072800085E59EE19F938F93DF93CF930F94646581
:10729000EDB7FEB73C960FB6F894FEBF0FBEEDBF3C
:1072A000D1CF012BB9F0AF92BF927F936F932F9202
:1072B0003F9289E49EE19F938F93DF93CF930F9446
:1072C00064658DB79EB70A960FB6F8949EBF0FBE41
:1072D0008DBFB8CF892BA9F0AF92BF927F936F93E8
:1072E00081E49EE19F938F93DF93CF930F94646526
:1072F000EDB7FEB738960FB6F894FEBF0FBEEDBFE0
:10730000A1CFAF92BF928DE39EE19F938F93DF93C6
:10731000CF930F9464650F900F900F900F900F9084
:107320000F9090CF90919B1793FB882780F993FF44
:1073300006C081E090913A14911101C080E0089557
:107340002F923F924F925F926F927F928F929F9275
:10735000AF92BF92CF92DF92EF92FF920F931F9363
:10736000CF93DF93CDB7DEB761970FB6F894DEBF4A
:107370000FBECDBF8C870E94AE362C85211136C042
:107380000E949ED94091031490917402499FA001DC
:107390001124440F452F441F550B51952091120283
:1073A00030911302609128147091291426273727F1
:1073B0006091A9067091AA06262737272427A901DC
:1073C0004827CA0120915E0630915F068217930715
:1073D00049F4E7E7F3E180E09191992309F449C288
:1073E0008927FACF90935F0680935E060E949ED90C
:1073F0008F870E940BCE688779878A879B875091F9
:107400001202588B80911302898B60912414709121
:10741000251480912614909127140F94906B2B01C2
:1074200020902814309029146091A5067091A6062A
:107430008091A7069091A8060F94906B4B017E87D0
:107440006D87E090A906F090AA062114310469F036
:10745000DD24D394C20182199309241435041CF04D
:10746000C1018419950903970CF4D12C8091050270
:107470008170CC24C3948D1101C0CC8481E00E9422
:1074800052360E941D355F924F924CEC642E40E2C2
:10749000742E7F926F928E010F5F1F4F1F930F9379
:1074A0000F946465C8010E94D4300F900F900F9024
:1074B0000F900F900F90DD20A1F08AE10F944023F0
:1074C0003F922F927F926F921F930F930F94646558
:1074D000C8010E94D4300F900F900F900F900F9022
:1074E0000F90CC2021F06D2D80E00E940E3680910F
:1074F0000502D0FA80F980930502E114F10479F0D5
:10750000ED85FE8577247394C4018E199F09EE16CC
:10751000FF061CF0C7018819990903970CF4712C18
:107520008091050282FB882780F966246394871185
:1075300001C06C8481E10E9452360E941D359F92E9
:107540008F923CECC32E30E2D32EDF92CF921F936A
:107550000F930F946465C8010E94D4300F900F9070
:107560000F900F900F900F907720A1F08AE10F9469
:107570004023FF92EF92DF92CF921F930F930F94CD
:107580006465C8010E94D4300F900F900F900F9047
:107590000F900F90662021F0672D81E00E940E363B
:1075A0008091050270FA82F980930502809103149C
:1075B000A82EB12CFF85F1110CC09091740297FD9B
:1075C00008C0899F50011124AA0CAB2CAA1CBB082F
:1075D000B19486E00E9452360E941D3524E62A9D11
:1075E000C0012B9D900D112481589F4F6FEF70E0CB
:1075F0000F94566D7F936F939CECC92E90E2D92E19
:10760000DF92CF921F930F930F946465C8010E947D
:10761000D43085E20F94402388E00E94523640E047
:10762000B801CE0108960E94E030800F912F911D85
:1076300020E2FC0120830E941D3566E0C8010E9403
:10764000C03086E10E9452360E941D35F989FF93B1
:1076500028892F93DF92CF921F930F930F94646525
:10766000C8010E94D43085E20F9440230FB6F894ED
:10767000DEBF0FBECDBFAB2879F085E00E94523649
:107680000E941D355F8516E0511114E080E00F94D3
:107690004023812F0F9440231E141F040CF01F86DB
:1076A00080E10E9452360E941D351E141F040CF00A
:1076B000DBC08F8512E0811110E080E00F94402341
:1076C000812F0F9440239C85992309F482CE109238
:1076D00076130E945C360E94843180919B1782FF52
:1076E0002AC00E949239882309F4CAC08091931756
:1076F00090919417A0919517B09196170097A105B6
:10770000B10509F4BDC0BC01CD016D597F4F8F4F4C
:107710009F4F24E630E040E050E00F94C069609154
:107720009717709198178091991790919A170F94C5
:10773000C06920936106C0906106EC85E11105C027
:10774000809162068C1509F474C0C09262068C2D7B
:1077500069E10F94366DF0E19F9FC001112469E14A
:1077600070E00F94566D80E090E84C0102C0959453
:1077700087946A95E2F7DD24D394EC2CF12C6D2DDF
:107780008CE00E94BE350E941D3589E1A82EB12CE7
:10779000712C0FEF1FEFEA14FB0444F4C501499765
:1077A00010E000E08E159F050CF4840121E0D21654
:1077B00009F46CC04DE0D41609F468C053E07512AA
:1077C00061C00160812F0F944023802F0F944023CC
:1077D000739489E1A80EB11C94E07912DACFD394A6
:1077E000EEE0DE12CCCF8CE00E9452360E941D35B6
:1077F00080E20F9440238E010F5F1F4FF9E0FC15CC
:1078000008F047C0FF92EF9280ED90E29F938F9334
:107810001F930F930F946465C8010E94D43088EDC4
:1078200090E20E94B2300F900F900F900F900F9047
:107830000F900E94AE3661960FB6F894DEBF0FBE71
:10784000CDBFDF91CF911F910F91FF90EF90DF900F
:10785000CF90BF90AF909F908F907F906F905F90F0
:107860004F903F902F90089580E20F94402380E244
:1078700028CF909160068917E1F08093600627CFAA
:1078800020E057CF71109ECF10689CCF0FEF1FEFF5
:1078900099CFFF92EF928CEC90E29F938F931F937E
:1078A0000F930F946465C8010E94D43084ED90E278
:1078B000B8CF0E948431882309F40FCF0E945C3630
:1078C0000CCF4F925F926F927F928F929F92AF9266
:1078D000BF92CF92DF92EF92FF920F931F93CF93BD
:1078E0001092700510926F052FE32093730510928C
:1078F00072051092710510926B0510926C05109232
:107900006D0510926E059C01F90190812F5F3F4F2C
:107910009032D1F39E34C9F4818190ED980F9A3062
:1079200020F08D3211F08B3281F432969F012F5F5F
:107930003F4F808180538A3008F475C09F012F5FCC
:107940003F4F8081803209F470C0F093B60BE09312
:10795000B50B8F010F5F1F4FC0816AE270E0C80155
:107960000F94BA6D009731F0FC013197808180321D
:10797000E1F31182CD3429F0C43519F0C73409F090
:1079800042C0F80180810F5F1F4F8032D1F38053D6
:107990008A30C8F5C093730590E080E0AAE0AF019B
:1079A0004F5F5F4F2081022E000C330B20533109B3
:1079B000A89FB001A99F700D1124C901860F971FC0
:1079C000FA01208120532A3050F39093720580935E
:1079D0007105DF0131962C912032D9F3CD3499F520
:1079E0008737910524F5853791054CF48C31910545
:1079F00031F08E31910519F08731910521F5B09361
:107A00007005A0936F05CF911F910F91FF90EF909C
:107A1000DF90CF90BF90AF909F908F907F906F90AE
:107A20005F904F900895F90181CFF90187CF8A3295
:107A300023E0920744F08433E3E09E0704F3803AA6
:107A4000F3E09F07E1F21091B50BC12CD12C760128
:107A500050E040E0812C912C5401839401C0DF015F
:107A6000FD0131962C91222309F481C02132E1F4E9
:107A7000CD34D1F480329105B9F4C0926B05D09227
:107A80006C05E0926D05F0926E05F0937005E09341
:107A90006F0563E270E0CF010F94BA6D009709F4AF
:107AA000B2CFDC011C92AFCF21542A3108F05AC06A
:107AB000DF013D91303291F060ED630F6A30E8F004
:107AC0003E3271F4318130533A30B8F041155105EE
:107AD00019F4AF014150510930E013C0FD01E8CF66
:107AE0003D3211F03B3291F7318160ED630F6A3026
:107AF00020F03E3259F73281E6CF3E2F311B3097CE
:107B000059F3622F70E02401350104C0440C551C68
:107B1000661C771C2A95D2F7C428D528E628F728B2
:107B20006F5A7A4FDB013C93208121542A3108F4AB
:107B300096CFDF01FD012D91222309F490CF30ED86
:107B4000320F3A30B8F333ED320F323098F32B3234
:107B500089F39F012F5F3F4F6081603209F07FCF33
:107B6000F901F7CF41155105F9F6AD01DDCF50937D
:107B7000700540936F05C0926B05D0926C05E09242
:107B80006D05F0926E053FCF1F93CF93DF93EC010D
:107B9000162F1D8A1E8A8F89807F8F8BE881F9813D
:107BA0000190F081E02D20E030E0A90164E1CE01F8
:107BB0001995612FCE010F9425528B898E7F8B8B67
:107BC0002A89382F8C89482F437050E0E881F98149
:107BD0000190F081E02D60E0CE01DF91CF911F9107
:107BE00019941F93CF93DF93EC010F944952182FF0
:107BF0008FEF8D8B8E8B8F898F608F8BE881F981D2
:107C00000190F081E02D2FEF3FEF4FE050E064E175
:107C1000CE01199560E0CE010F9425528B898160C9
:107C20008B8B2A89382F8C89482F437050E0E8814C
:107C3000F9810190F081E02D60E0CE011995812F4E
:107C4000DF91CF911F91089580E00E94AB33ECEA61
:107C5000F5E180E090E0A0E8BFE380839183A28318
:107C6000B3831482158216821782108611861286BB
:107C700013861486158616861786808B918BA28BA9
:107C8000B38B148A158A168A178A108E118E128E5B
:107C9000138E148E158E168E178E80A391A3A2A319
:107CA000B3A30895282FE82FF0E09091AF0B892F10
:107CB00090E0B0E0A0E004C0B695A79597958795B1
:107CC0002A95D2F780FF14C08091630690916406D4
:107CD000860F971F9093640680936306EE0FFF1F35
:107CE000E556F94F80819181680F791F7183608318
:107CF0000895CF92DF92EF92FF926B017C0183E3B4
:107D0000C816D104E104F10470F082E3C81AD10866
:107D1000E108F10862E370E080E090E00F94D24B5C
:107D20000E947CAFECCFC701B6010F94D24BFF90FD
:107D3000EF90DF90CF900C947CAF80910204811182
:107D400007C00E9469EA882319F081E08093020449
:107D5000089510920314109265060895CF93C82FCA
:107D600080933A090E946CC6CC2369F024982C9A1F
:107D700065E070E080E090E00F94D24B0E9476BE08
:107D8000149ACF910895249A2C981498FACF8F9230
:107D90009F92AF92BF92CF92DF92EF92FF920F939A
:107DA000CF93DF931F92CDB7DEB75C017B01490112
:107DB0006B01C40ED51EF501808191810F949A69E3
:107DC0008983002311F0F7018083BE016F5F7F4F2D
:107DD000C4010F944226F50180819181019691831F
:107DE0008083FFEFEF1AFF0AEC14FD0421F780E017
:107DF0000F90DF91CF910F91FF90EF90DF90CF9098
:107E0000BF90AF909F908F900895CF93DF93CDB7A1
:107E1000DEB760970FB6F894DEBF0FBECDBF9C01F2
:107E2000E62F660FFF0BE657F04CE491E750EC307D
:107E300008F0C4C0F0E08827EF5DF04C8F4F0D9440
:107E40006A6D593F2D3F803F7E3F5B3FB73FB53F57
:107E5000823FDE3FDC3FDA3FB93F81E0FE013596ED
:107E60009AE0DF011D929A95E9F740EB50E05A83C2
:107E7000498341EB50E05C834B8343EB50E05887F0
:107E80004F8344EB50E05A87498792E09F87888B65
:107E900080E13497D90101900D928A95E1F7C901EB
:107EA00060960FB6F894DEBF0FBECDBFDF91CF91C5
:107EB000089580E0D3CF81E08F5F40E950E0F90181
:107EC0005183408341E950E05383428342E950E0CB
:107ED0005583448348E950E0578346834AE950E09C
:107EE000518740874CE950E05387428746E950E08C
:107EF0005587448793E096878787D1CF80E0DCCF92
:107F000080E0DBCF81E08F5F40EA50E0D90111963D
:107F10005C934E9341EA50E013965C934E93129714
:107F200042EA50E015965C934E93149748EA50E06D
:107F300017965C934E9316974AEA50E019965C9315
:107F40004E9318974CEA50E01B965C934E931A9709
:107F500046EA50E01D965C934E931C9794E01E9663
:107F60009C931E971F968C939ACF80E0CCCF80E095
:107F7000CBCF81E08F5F40E251E0F9015183408334
:107F800041E251E05383428342E251E0558344830E
:107F900048E251E0578346834AE251E051874087E7
:107FA0004CE251E05387428746E251E055874487CF
:107FB00095E0A1CF80E0DECF80E0DDCF80E1D90188
:107FC0001D928A95E9F76BCF9091C10095FD0CC089
:107FD0009091C00095FF08C08093C6008091C000BA
:107FE00080648093C00008952091E0032F5F2F717B
:107FF0000FB607FC27C09091E103921328C090911F
:10800000C00095FF1EC09091E1034091E0039413DE
:1080100006C09091C1009F7D9093C10012C0E92FCE
:10802000F0E0E052FC4F32819F5F9F713093C600B9
:108030009093E1033091C00030643093C000491741
:1080400041F3D9CF9091E103921301C0FBCFE091AE
:10805000E003F0E0E052FC4F82832093E003809144
:10806000C10080628093C100089585E40C94E43FD0
:108070008AE50C94E43F89E50C94E43F88E50C9490
:10808000E43FFC01693071F06B3081F06830A1F49D
:10809000858996892789A22FAF70BC018A2F90E02D
:1080A0000D945D28808D918D228DF5CF66A177A1ED
:1080B00091A580A59170F4CF89E00C94E43F0F93D3
:1080C0001F93CF93DF93C82F142FD22F662319F15C
:1080D0008F3008F087C0E82F880FFF0B8827EC58F7
:1080E000FF4B8F4F0D946A6D8340AA40B140BD4055
:1080F000C340C840CE40D340F240F240DA40F240A4
:10810000DF40E840ED4089E00E94E43F0E943E40AD
:1081100089E00E94E43F112309F472C0CF3008F0D7
:10812000D6C0EC2F0C2E000CFF0B8827E556FF4B1A
:108130008F4F0D946A6DF8401F41264132413841FE
:108140003D4143414841674167414F416741544187
:108150005D41624188E695E10F9441520F945D289C
:10816000D7CF80916A1590916B1520916C15A22F35
:10817000AF70BC018A2F90E0F1CF88E695E10F94B3
:10818000274E682F07C088E695E10F940052E6CF8E
:1081900060916D1570E090E080E0E0CF88E695E1B9
:1081A0000F941F4EDBCF80916E1590916F1520912B
:1081B0007015DDCF88E695E10F948D53CFCF809178
:1081C00095159091961520919715A22FAF73D1CF49
:1081D00088E695E10F94F651D4CF88E695E10F94A7
:1081E0004024BCCF6C2F88E695E10E94414090CF9F
:1081F00089E00E94E43F0E943B4089E00E94E43F06
:10820000DD2309F472C0CF3008F0D6C0EC2F0C2E5D
:10821000000CFF0B8827E05FFE4B8F4F0D946A6DBB
:108220006D4194419B41A741AD41B241B841BD412F
:10823000DC41DC41C441DC41C941D241D74189E242
:1082400095E10F9441520F945D28D7CF80912B1563
:1082500090912C1520912D15A22FAF70BC018A2F63
:1082600090E0F1CF89E295E10F94274E682F07C087
:1082700089E295E10F940052E6CF60912E1570E0EF
:1082800090E080E0E0CF89E295E10F941F4EDBCFD4
:1082900080912F159091301520913115DDCF89E215
:1082A00095E10F948D53CFCF80915615909157152E
:1082B00020915815A22FAF73D1CF89E295E10F9489
:1082C000F651D4CF89E295E10F944024BCCF6C2FB6
:1082D00089E295E10E94414090CF89E00E94E43F0D
:1082E0000E94384089E00E94E43F002309F472C0F4
:1082F000CF3008F0BEC0EC2F0C2E000CFF0B8827EF
:10830000EB57FE4B8F4F0D946A6DE241F141F841FE
:1083100004420A420F4215421A423942394221426E
:10832000394226422F4234428AEE94E10F94415260
:108330000F945D28D7CF8091EC149091ED1420918B
:10834000EE14A22FAF70BC018A2F90E0F1CF8AEE1D
:1083500094E10F94274E682F07C08AEE94E10F94A2
:108360000052E6CF6091EF1470E090E080E0E0CF43
:108370008AEE94E10F941F4EDBCF8091F014909120
:10838000F1142091F214DDCF8AEE94E10F948D5315
:10839000CFCF809117159091181520911915A22F04
:1083A000AF73D1CF8AEE94E10F94F651D4CF8AEE19
:1083B00094E10F944024BCCF6C2F8AEE94E10E948C
:1083C000414090CF89E00E94E43F0E94354089E01F
:1083D0000E94E43F8AE0DF91CF911F910F910C94AE
:1083E000E43F8BEA94E10F9441520F945D28EFCF64
:1083F0008091AD149091AE142091AF14A22FAF7064
:10840000BC018A2F90E0F1CF8BEA94E10F94274EC4
:10841000682F07C08BEA94E10F940052E6CF609179
:10842000B01470E090E080E0E0CF8BEA94E10F942C
:108430001F4EDBCF8091B1149091B2142091B314F0
:10844000DDCF8BEA94E10F948D53CFCF8091D81478
:108450009091D9142091DA14A22FAF73D1CF8BEA67
:1084600094E10F94F651D4CF8BEA94E10F94402419
:10847000BCCF6C2F8BEA94E10E944140A8CF6930B9
:1084800051F11CF4683031F008956A30D1F06B304E
:1084900069F00895DC01ED91FC910084F185E02DF7
:1084A000199590FF17C08AE20C94E43FDC01ED912E
:1084B000FC910084F185E02D1995CB0193700D940A
:1084C0005728DC01ED91FC910084F185E02D199590
:1084D00077FDE9CF08950F949C520D945028CF93C7
:1084E000DF93EC01FE0184912196882319F00E940C
:1084F000E43FF8CFDF91CF910895FF920F931F9340
:10850000CF93DF93F62E042F122F882339F184E5C1
:108510009DE00E946F420E943E4084E49DE00E94E4
:108520006F4288E695E10F94E550D82F882361F0DB
:1085300088E39DE00E946F4280E39DE0D13031F0FE
:108540008CE29DE0D23011F085E39DE00E946F4205
:108550008AE00E94E43FC1E0D11101C0C0E0FF20E9
:1085600049F185E89DE00E946F420E943B4085E70B
:108570009DE00E946F4289E295E10F94E550D82F6B
:10858000882361F089E69DE00E946F4281E69DE0CC
:10859000D13031F08DE59DE0D23011F086E69DE0DE
:1085A0000E946F428AE00E94E43F81E0D11101C045
:1085B00080E0C80F002349F186EB9DE00E946F42E6
:1085C0000E94384086EA9DE00E946F428AEE94E164
:1085D0000F94E550D82F882361F08AE99DE00E942E
:1085E0006F4282E99DE0D13031F08EE89DE0D230DB
:1085F00011F087E99DE00E946F428AE00E94E43F0B
:1086000081E0D11101C080E0C80F112349F187EE4C
:108610009DE00E946F420E94354087ED9DE00E94E0
:108620006F428BEA94E10F94E550D82F882361F0D4
:108630008BEC9DE00E946F4283EC9DE0D13031F0E5
:108640008FEB9DE0D23011F088EC9DE00E946F42EC
:108650008AE00E94E43F81E0D11101C080E0C80FB0
:10866000CC2351F060E080EF9DE0DF91CF911F912E
:108670000F91FF900C942CD9DF91CF911F910F9106
:10868000FF900895CF92DF92EF92FF920F931F9386
:10869000CF93DF93C82F142FD22F662309F44DC236
:1086A00089E00E94E43FCD3008F042C2EC2F0C2E4E
:1086B000000CFF0B8827E05AFC4B8F4F0D946A6D1E
:1086C0006D439143C743F9432B445D448F44C144F8
:1086D0009845984598459845F3440E943E4011239B
:1086E00009F44EC289E00E94E43F0E943B40DD2332
:1086F00009F469C289E00E94E43F0E9438400023E7
:1087000029F089E00E94E43F0E9435408AE0DF9131
:10871000CF911F910F91FF90EF90DF90CF900C942D
:10872000E43F88E695E10F944F52882319F08AE2DE
:108730000E94E43F112309F423C289E00E94E43F30
:1087400089E295E10F944F52882319F08AE20E9442
:10875000E43FDD2309F437C289E00E94E43F8AEE5A
:1087600094E10F944F52882319F08AE20E94E43F6B
:10877000002361F289E00E94E43F8BEA94E10F94C8
:108780004F52882319F28AE20E94E43FBFCF88E665
:1087900095E10F945A52882319F08AE20E94E43F2F
:1087A000112309F4EDC189E00E94E43F89E295E1DB
:1087B0000F945A52882319F08AE20E94E43FDD2385
:1087C00009F401C289E00E94E43F8AEE94E10F942B
:1087D0005A52882319F08AE20E94E43F002309F4E8
:1087E00095CF89E00E94E43F8BEA94E10F945A52BE
:1087F000C8CF88E695E10F946552882319F08AE284
:108800000E94E43F112309F4BBC189E00E94E43FC8
:1088100089E295E10F946552882319F08AE20E945B
:10882000E43FDD2309F4CFC189E00E94E43F8AEEF2
:1088300094E10F946552882319F08AE20E94E43F84
:10884000002309F463CF89E00E94E43F8BEA94E1BE
:108850000F94655296CF88E695E10F947052882365
:1088600019F08AE20E94E43F112309F489C189E0EA
:108870000E94E43F89E295E10F947052882319F039
:108880008AE20E94E43FDD2309F49DC189E00E9451
:10889000E43F8AEE94E10F947052882319F08AE243
:1088A0000E94E43F002309F431CF89E00E94E43FB5
:1088B0008BEA94E10F94705264CF88E695E10F94AF
:1088C0007B52882319F08AE20E94E43F112309F4C5
:1088D00057C189E00E94E43F89E295E10F947B5201
:1088E000882319F08AE20E94E43FDD2309F46BC17A
:1088F00089E00E94E43F8AEE94E10F947B52882342
:1089000019F08AE20E94E43F002309F4FFCE89E0D7
:108910000E94E43F8BEA94E10F947B5232CF88E6C9
:1089200095E10F948652882319F08AE20E94E43F71
:10893000112309F425C189E00E94E43F89E295E111
:108940000F948652882319F08AE20E94E43FDD23C7
:1089500009F439C189E00E94E43F8AEE94E10F9462
:108960008652882319F08AE20E94E43F002309F42A
:10897000CDCE89E00E94E43F8BEA94E10F948652C9
:1089800000CF88E695E10F949152882319F08AE28E
:108990000E94E43F112309F4F3C089E00E94E43F00
:1089A00089E295E10F949152882319F08AE20E949E
:1089B000E43FDD2309F407C189E00E94E43F8AEE29
:1089C00094E10F949152882319F08AE20E94E43FC7
:1089D000002309F49BCE89E00E94E43F8BEA94E1F6
:1089E0000F949152CECE88E695E10F9440246B010E
:1089F0007C0189E00E94E43F0E943E4089E00E94A1
:108A0000E43FC701B6010F945D2881E0C81AD10880
:108A1000E108F1088EEFC8168FEFD806E806F806D1
:108A200020F08AE89BE00E946F428AE00E94E43FC7
:108A3000112309F4A5C089E00E94E43F89E295E191
:108A40000F9440246B017C0189E00E94E43F0E9466
:108A50003B4089E00E94E43FC701B6010F945D28C6
:108A600081E0C81AD108E108F1088EEFC8168FEF2F
:108A7000D806E806F80620F08AE99BE00E946F42DB
:108A80008AE00E94E43FDD2309F49DC089E00E9452
:108A9000E43F8AEE94E10F9440246B017C0189E06D
:108AA0000E94E43F0E94384089E00E94E43FC701F1
:108AB000B6010F945D2881E0C81AD108E108F108D9
:108AC0008EEFC8168FEFD806E806F80620F08AEA7F
:108AD0009BE00E946F428AE00E94E43F002309F479
:108AE00015CE89E00E94E43F8BEA94E10F94402484
:108AF0006B017C0189E00E94E43F0E94354089E0DF
:108B00000E94E43FC701B6010F945D2881E0C81AB6
:108B1000D108E108F1088EEFC8168FEFD806E806F5
:108B2000F80620F08AEB9BE00E946F428AE02CCE90
:108B30006C2F88E695E10E943F42112309F189E0FC
:108B40000E94E43FCD30B8F4EC2F0C2E000CFF0B4C
:108B50008827E255FA4B8F4F0D946A6D7543A043F9
:108B6000D64308443A446C449E44D044BB45BB457C
:108B7000BB45BB451E456C2F89E295E10E943F42F3
:108B8000DD2309F189E00E94E43FCD30B8F4EC2FF9
:108B90000C2E000CFF0B8827EF52FA4B8F4F0D94D1
:108BA0006A6D7D43AF43E543174449447B44AD447C
:108BB000DF44DE45DE45DE45DE4549456C2F8AEE65
:108BC00094E10E943F42002309F4A0CD89E00E9475
:108BD000E43FCD30B8F4EC2F0C2E000CFF0B8827AF
:108BE000EB50FA4B8F4F0D946A6D8443BD43F443B1
:108BF000264458448A44BC44EE4402460246024697
:108C0000024674456C2F8BEA94E10E943F427ECD70
:108C1000811104C08DEB99E00C946F4283EC99E0D4
:108C2000FBCFCF93DF93EB010E946F42CE01DF9128
:108C3000CF910D9457280F931F93CF93DF938B0100
:108C40000E946F42E8018991882319F00E94E43F55
:108C5000FACFDF91CF911F910F91089586EB99E0A4
:108C60000C946F424F925F926F927F928F929F927D
:108C7000AF92BF92CF92DF92EF92FF920F931F932A
:108C8000CF93DF931F92CDB7DEB780919B1782FF02
:108C90001FC180911F0B811102C010925C06EE244F
:108CA000E39440919717509198176091991770919C
:108CB0009A178091931790919417A0919517B0915E
:108CC0009617481759076A077B0708F4E12C10E04C
:108CD00000E0AA24A39480E6982E96E1C92E9EE196
:108CE000D92E29E6822E80911F0B853008F0F0C026
:108CF000E110EEC0E0905C06E110EAC080913F1404
:108D000090914014A0914114B09142148093971710
:108D100090939817A0939917B0939A1741E050E059
:108D2000BE016F5F7F4F87E394E10E9458A30197D4
:108D3000D9F5898190E0F82E4090971750909817B8
:108D40006090991770909A174091931750919417CB
:108D50006091951770919617BB24B39444165506ED
:108D60006606770608F4B12C4416550666067706A3
:108D7000F0F4019609F468C08AE0F81609F46AC0B4
:108D80002DE0F21609F466C083E2F81619F02AE322
:108D9000F21279C080915B06811175C023E2F21254
:108DA00059C0A0925C0656C08FEF9FEFC4CF0E94BF
:108DB00076BE87E394E10E9427A5809192178823CD
:108DC00079F1815080939217889DC001112441E070
:108DD00061E08D53994F0E9406ABE091921784E0B9
:108DE000E89FF0011124E154F94F408151816281E3
:108DF00073814093971750939817609399177093C6
:108E00009A1787E394E10E94C4A10E94719E809109
:108E10009B1782FD57C089E29EE10E946F42BECF40
:108E20000E9430A50E943DCE0E940BCE6D3371058D
:108E30008105910520F0D0923D09C0923C09109225
:108E400061060E947ED9E3CF0E942E468AE19EE110
:108E50000E946F4210925B060115110531F40E94C9
:108E60007CAFEB2C10E000E03ECF80913B09989E58
:108E7000000D111D1124F801E25CF64F108280E014
:108E80000E94D62EEECF0F35110508F02CCF8BE3C4
:108E9000F81203C0A0925B0626CF80915B06811179
:108EA00022CF80913B09F801989EE00DF11D11241D
:108EB000E25CF64FF082E12C0F5F1F4F14CF10924F
:108EC0005B06CDCF23E2F212FACF10E000E069CFCB
:108ED0000F90DF91CF911F910F91FF90EF90DF9056
:108EE000CF90BF90AF909F908F907F906F905F904A
:108EF0004F90089580EB99E00C946F42CF93C82F68
:108F000082E0C11184E040E060E00F941C120E94F6
:108F10007A4789ED99E0CC2311F08BEF99E0CF915E
:108F20000C946F429091641193FD0FC09091FD0BD2
:108F300091110BC040912814509129142091720274
:108F400030917302421753074CF040E0682F8BE0DA
:108F50000F941C1261E080E00C9485DB0E947A473C
:108F600088EC99E00E946F4280E008958F929F9272
:108F7000AF92BF92CF92DF92EF92FF920F931F9327
:108F8000CF93DF9300D000D01F921F92CDB7DEB7F2
:108F90006C015B017A01022F8EE49AE00F9458264F
:108FA0008091641183FD1CC020E030E0A901F7012D
:108FB00060817181828193810F94CD65882381F0D6
:108FC0001091FD0B11110CC020912814309129141F
:108FD0008091720290917302281739070CF45FC0D8
:108FE0009091BE0681E0890F8093BE0680919B1709
:108FF00082FD7AC00E94FECE80E1EAE5F2E0AFE2B7
:10900000B4E001900D928A95E1F70E9476BE20E0CF
:1090100030E0A901F60160817181828193810F9412
:10902000CD65882319F18091FD0B811111C06091EC
:1090300024147091251480912614909127140F9474
:10904000906B20917202309173026217730774F073
:1090500080E090E0A0E2B1E489839A83AB83BC8393
:10906000BE016F5F7F4FC6010E94073241E061E0A1
:1090700081E00E94CFC3811104C0B50182E00E944B
:1090800074DF20E030E0A901F70160817181828105
:1090900093810F94CD6581112EC011E011C00E9403
:1090A0007A4784E69AE00E946F42002349F01092CA
:1090B00024080E947EF860E085E59AE00E942CD9A1
:1090C000812F28960FB6F894DEBF0FBECDBFDF917B
:1090D000CF911F910F91FF90EF90DF90CF90BF90B5
:1090E000AF909F908F9008958B7F80939B179E5F8A
:1090F0009093BE067FCF81E00E949247182F811186
:1091000007C0002351F2109224080E947EF8C5CFB8
:10911000002329F040E061E083E00F941C1280E01E
:1091200090E0A0E0B0E489839A83AB83BC8380E0C5
:1091300090E0A0ECB0E48D839E83AF83B887BE013E
:109140006F5F7F4FCE0105960E9407328090F31328
:109150009090F413A090F513B090F61380E090E097
:10916000A8ECB1E48093F3139093F413A093F51358
:10917000B093F61380E090E0A0E0B1E489839A8395
:10918000AB83BC83F70180819181A281B3818D8300
:109190009E83AF83B887BE016F5F7F4FCE01059678
:1091A0000E9407328092F3139092F413A092F51369
:1091B000B092F613149A64E670E080E090E00E94AA
:1091C000793E7ECF1F93CF93DF93EC010E9490AC4A
:1091D0000E942E4680E999E00E946F42209711F488
:1091E000C7E8D9E00E94D6D961E0CE010E942CD90F
:1091F0000E947EF80E94AE360E946B350E94B23506
:1092000086E20E942F3580916B068460886080938F
:109210006B060E94AE36C0911316C695C6958EE0B9
:1092200096E10E94EB34DC2FDD0F1D2F1C0F0F94F5
:10923000892710924916C0934A1687E793E10E9446
:10924000B93710924916D0934A168FE699E00E94DA
:1092500010371092491610934A1682E699E00E9440
:10926000103782E196E10F94CF568111E0CF8EE75F
:1092700099E00F94582689EE93E030E6019729F0A3
:10928000232F2A950000E9F7F9CFF89489EE93E0AF
:1092900038EE019729F0232F2A950000E9F7F9CF3E
:1092A0000E9490AC359902C0A895FCCF359B02C0B6
:1092B000A895FCCFF0E0E0E0DF91CF911F911994E9
:1092C0007F928F929F92AF92BF92CF92DF92EF9256
:1092D000FF920F931F93CF93DF931F92CDB7DEB70B
:1092E0007C0159018B016B01C40ED51E0C151D05A7
:1092F000C9F1F70180809180F80171908F01798226
:10930000C4010F949A69781601F1672DC4010F9476
:10931000A269C4010F949A6999818917B1F00E94DA
:109320007A4785EA97E00E946F4281E00F90DF91D3
:10933000CF911F910F91FF90EF90DF90CF90BF9052
:10934000AF909F908F907F900895BE016F5F7F4F89
:10935000C5010F944226F701808191810196918386
:109360008083C4CF80E0E2CFCF92DF92EF92FF9272
:109370000F931F93CF93DF93CDB7DEB7A0970FB6B0
:10938000F894DEBF0FBECDBF611571058105910553
:1093900079F100E0C42ED12CF12CE12CA70196012B
:1093A0000F94C06911E0100FE1E0F0E0EC0FFD1F39
:1093B000E00FF11D07FDFA956083B901CA01012F85
:1093C000611571058105910549F7115010F1E1E032
:1093D000F0E0EC0FFD1FE10FF11D17FDFA959081F4
:1093E00087E39A3008F480E3890F0E94E43FEDCFD1
:1093F00080E3A0960FB6F894DEBF0FBECDBFDF911D
:10940000CF911F910F91FF90EF90DF90CF900C9430
:10941000E43FA0960FB6F894DEBF0FBECDBFDF913C
:10942000CF911F910F91FF90EF90DF90CF90089513
:10943000CF92DF92EF92FF926A017B010E946F420E
:109440004AE0C701B601FF90EF90DF90CF900C94F7
:10945000B449CF92DF92EF92FF926B017C01F7FE4D
:109460000BC08DE20E94E43FF094E094D094C0944D
:10947000C11CD11CE11CF11C4AE0C701B601FF90E0
:10948000EF90DF90CF900C94B4496C3089F0673145
:1094900031F06A3089F40F94F6510D9450280F94EE
:1094A000A552682F880F770B880B990B0C94294ACB
:1094B0000F9449520C9408460895CF93DF93E0919E
:1094C0001E0BF0E0E45BF94E8081882309F447C06D
:1094D0008EED9CE10E946F42C0911E0B80E6C89FFA
:1094E000E0011124C25CD64F88818E3479F480E289
:1094F0000E94E43F89910E94E43F899190ED980F8A
:109500009A30C8F38D32B9F38B32A9F38BED9CE11D
:109510000E946F428091AA159091AB15891B8F70A4
:109520006FE070E0681B7109072E000C880B990B27
:109530000E94294A88ED9CE10E946F4280911F0B96
:1095400065E070E0681B7109072E000C880B990B11
:109550000E94294A8AE0DF91CF910C94E43FDF9189
:10956000CF910895CF93DF93EB010E946F42BE012C
:10957000DD0F880B990BDF91CF910C94294ACF9383
:1095800084E50E949F2FC0E08823F9F00E94C23139
:10959000C82F1816D4F40E947A478DE40E94E43F45
:1095A0006091710570917205072E000C880B990B64
:1095B0000E94294A6C2FCC0F770B85EA92E10E941A
:1095C000B24A8AE00E94E43FCFEF8C2FCF910895FA
:1095D000AF92BF92CF92DF92EF92FF921F93CF9301
:1095E000DF9360E089E40E94D631182F80E8A82E2E
:1095F00082E0B82ED0E0C1E0F50181915F010E94C8
:109600009F2F8823B9F00E9491316B017C01C11416
:10961000D104E104F10471F0D23009F454C0D33024
:1096200009F457C0D13009F448C0123010F40F9437
:109630008350C0E0DF5FD430F9F6CC2309F454C086
:109640000E943E400F94444FAB01BC0181E492E183
:109650000E94184A8AE00E94E43F0E943B400F9417
:10966000F54EAB01BC018AE592E10E94184A8AE0FE
:109670000E94E43F0E9438400F94A64EAB01BC010B
:1096800083E792E10E94184A8AE00E94E43F0E9428
:1096900035400F94574EAB01BC018CE892E10E941B
:1096A000184A8AE0DF91CF911F91FF90EF90DF90F1
:1096B000CF90BF90AF900C94E43F123008F0B9CF38
:1096C0000F943350B6CF123008F0B3CF0F94E34F5E
:1096D000B0CF0E94BF4A87FD07C08111AACFC70142
:1096E000B6010F94934FA5CFDF91CF911F91FF90BB
:1096F000EF90DF90CF90BF90AF900895EF92FF92E0
:109700000F931F93CF93DF9383E50E94562F8823F7
:1097100009F44AC00E94BF4A082F0E94E231C82FB4
:1097200060E089E40E94D631182F80E8E82E82E0BC
:10973000F82ED0E0F70181917F010E94562F8823F7
:1097400079F0D230F9F0D33029F1D13099F01111FC
:1097500007C0C093A3156C2F88E695E10F9425529E
:10976000DF5FD43039F7DF91CF911F910F91FF90D8
:10977000EF9008951111F4CFC09364156C2F89E216
:1097800095E1ECCF1111ECCFC09325156C2F8AEE2B
:1097900094E1E4CF07FDE7CF0111E2CFC093E614D7
:1097A0006C2F8BEA94E1DACF0E943E408DEB91E181
:1097B0000E946F4288E695E10F944952811146C09C
:1097C00085EA91E10E946F428AE00E94E43F0E9494
:1097D0003B4084EE91E10E946F4289E295E10F9453
:1097E0004952811136C08CEC91E10E946F428AE0AF
:1097F0000E94E43F0E9438408BE092E10E946F4259
:109800008AEE94E10F944952811126C083EF91E1D1
:109810000E946F428AE00E94E43F0E94354082E34A
:1098200092E10E946F428BEA94E10F9449528111B8
:1098300016C08AE192E10E946F428AE0DF91CF91E7
:109840001F910F91FF90EF900C94E43F81EB91E119
:10985000B9CF88ED91E1C9CF8FEF91E1D9CF86E201
:1098600092E1E9CF8F929F92AF92BF92CF92DF9217
:10987000EF92FF92CF936B017C01B42E20E030E099
:10988000A9010F94CD6587FF07C08DE20E94E43FD8
:10989000F7FAF094F7F8F094C0E060E070E080E050
:1098A0009FE3CB1541F02DEC3CEC4CEC5DE30F94C9
:1098B0003366CF5FF6CF9B01AC01C701B6010F94B1
:1098C000246A6B017C010F94976B4B015C014AE0A9
:1098D0000E94B449CC2391F1C501B4010F94D26523
:1098E0009B01AC01C701B6010F94236A6B017C0197
:1098F0008EE20E94E43FC15008F120E030E040E2F7
:1099000051E4C701B6010F9433664B015C010F941B
:10991000906B6B01770FEE08FF08C701B6010E943C
:10992000294AC701B6010F94D4659B01AC01C5015A
:10993000B4010F94236A6B017C01DDCFCF91FF90BE
:10994000EF90DF90CF90BF90AF909F908F90089551
:109950000F931F93CF93DF93182FD42FC22F66231B
:1099600009F413C489E00E94E43F173108F008C4E9
:10997000E12F012E000CFF0B8827EE53F34B8F4F86
:109980000D946A6DD94CC050F94C234D4E4D774D16
:10999000D24D094EC0503E4EC050774EC050B34ECF
:1099A000DC4E304F784FBA4FE34F04502F50585091
:1099B00097500E943E40DD2309F422C489E00E94B2
:1099C000E43F0E943B40CC2309F455C489E00E9447
:1099D000E43F0E943840002329F089E00E94E43FE0
:1099E0000E9435408AE0DF91CF911F910F910C9436
:1099F000E43F88E695E10F94BD530E940846DD23BD
:109A000009F4FEC389E00E94E43F89E295E10F94E6
:109A1000BD530E940846CC2309F42DC489E00E945E
:109A2000E43F8AEE94E10F94BD530E940846002360
:109A3000C9F289E00E94E43F8BEA94E10F94BD53A0
:109A40000E940846CFCF80919E1590919F150F944C
:109A50005728DD2309F4D4C389E00E94E43F8091B4
:109A60005F15909160150F945728CC2309F403C417
:109A700089E00E94E43F80912015909121150F9478
:109A80005728002309F4AECF89E00E94E43F80917B
:109A9000E1149091E2140F945728A4CF88E695E141
:109AA0000F94FC500F945728DD2309F4A9C389E0D3
:109AB0000E94E43F89E295E10F94FC500F945728EF
:109AC000CC2309F4D8C389E00E94E43F8AEE94E1F4
:109AD0000F94FC500F945728002309F483CF89E09A
:109AE0000E94E43F8BEA94E10F94FC50D4CF88E6C7
:109AF00095E10F94FC50BC0190E080E00F94D2659A
:109B000021EE3AE744EB5FE30F94336640E00E94B6
:109B1000324CDD2309F474C389E00E94E43F89E2FA
:109B200095E10F94FC50BC0190E080E00F94D26569
:109B300021EE3AE744EB5FE30F94336640E00E9486
:109B4000324CCC2309F497C389E00E94E43F8AEEAB
:109B500094E10F94FC50BC0190E080E00F94D2653A
:109B600021EE3AE744EB5FE30F94336640E00E9456
:109B7000324C002309F436CF89E00E94E43F8BEA9F
:109B800094E10F94FC50BC0190E080E00F94D2650A
:109B900021EE3AE744EB5FE30F94336640E00E9426
:109BA000324C20CF80916B158F710F9450288FE22B
:109BB0009BE00E946F42DD2309F422C389E00E94EA
:109BC000E43F80912C158F710F9450288CE49BE01A
:109BD0000E946F42CC2309F44EC389E00E94E43F07
:109BE0008091ED148F710F94502889E69BE00E94BC
:109BF0006F42002309F4F6CE89E00E94E43F809191
:109C0000AE148F710F94502886E89BE00E946F423B
:109C1000E9CE80916A158F710F9450288BE29BE0FA
:109C20000E946F42DD2309F4EBC289E00E94E43F09
:109C300080912B158F710F94502888E49BE00E942F
:109C40006F42CC2309F417C389E00E94E43F80915E
:109C5000EC148F710F94502885E69BE00E946F42B0
:109C6000002309F4BFCE89E00E94E43F8091AD1447
:109C70008F710F94502882E89BE0C8CF88E695E169
:109C80000F949C520F94502887E29BE00E946F42F1
:109C9000DD2309F4B5C289E00E94E43F89E295E141
:109CA0000F949C520F94502884E49BE00E946F42D2
:109CB000CC2309F4E0C289E00E94E43F8AEE94E1FB
:109CC0000F949C520F94502881E69BE00E946F42B3
:109CD000002309F487CE89E00E94E43F8BEA94E1F7
:109CE0000F949C520F9450288EE79BE08FCF88E60C
:109CF00095E10F949A53811133C086E19BE00E9455
:109D00006F42DD2309F47CC289E00E94E43F89E2CE
:109D100095E10F949A53811162C283E39BE00E9404
:109D20006F42CC2309F4A7C289E00E94E43F8AEE87
:109D300094E10F949A5381118DC280E59BE00E94BB
:109D40006F42002309F44ECE89E00E94E43F8BEA83
:109D500094E10F949A538111B7C28DE69BE056CFE0
:109D60008DE19BE0CCCF88E695E10F94424E0F94B5
:109D70005728DD2309F444C289E00E94E43F89E2C8
:109D800095E10F94424E0F945728CC2309F473C2E7
:109D900089E00E94E43F8AEE94E10F94424E0F94D2
:109DA0005728002309F41ECE89E00E94E43F8BEA85
:109DB00094E10F94424E6FCE88E695E10F941F4ECA
:109DC0006F3F2FEF72072FE08207910509F443C020
:109DD0004AE00E94B449DD2309F412C289E00E94DE
:109DE000E43F89E295E10F941F4E6F3F2FEF72071A
:109DF0002FE08207910509F4F5C14AE00E94B449B9
:109E0000CC2309F438C289E00E94E43F8AEE94E151
:109E10000F941F4E6F3F2FEF72072FE082079105BF
:109E200009F41BC24AE00E94B449002309F4DACDC8
:109E300089E00E94E43F8BEA94E10F941F4E6F3F4C
:109E40002FEF72072FE08207910509F440C24AE024
:109E50000E94B449C7CD83E29BE00E946F42BBCF12
:109E600080916E1590916F1520917015A22FAF7093
:109E7000BC018A2F90E04AE00E94B449DD2309F436
:109E8000BFC189E00E94E43F80912F159091301569
:109E900020913115A22FAF70BC018A2F90E04AE0CB
:109EA0000E94B449CC2309F4E6C189E00E94E43F52
:109EB0008091F0149091F1142091F214A22FAF70C0
:109EC000BC018A2F90E04AE00E94B449002309F4C3
:109ED00089CD89E00E94E43F8091B1149091B21441
:109EE0002091B314A22FAF70BC018A2F90E0AFCFA6
:109EF0000F94444F6115710581059105B9F14AE050
:109F00000E94B449DD2309F47BC189E00E94E43F4B
:109F10000F94F54E611571058105910509F467C12E
:109F20004AE00E94B449CC2309F4A5C189E00E940B
:109F3000E43F0F94A64E611571058105910509F462
:109F400091C14AE00E94B449002309F44BCD89E055
:109F50000E94E43F0F94574E6115710581059105EC
:109F600009F075CF8DE20E94E43F3CCD8DE20E9466
:109F7000E43FC8CF88E695E10F9486520E940846D8
:109F8000DD2309F43DC189E00E94E43F89E295E1C7
:109F90000F9486520E940846CC2309F46CC189E0D4
:109FA0000E94E43F8AEE94E10F9486520E94084694
:109FB000002309F417CD89E00E94E43F8BEA94E185
:109FC0000F9486523DCD8091A2150E940846DD2354
:109FD00009F416C189E00E94E43F809163150E9454
:109FE0000846CC2309F447C189E00E94E43F8091F0
:109FF00024150E940846002309F4F4CC89E00E944D
:10A00000E43F8091E5141CCD88E695E10F94B853A8
:10A010000F945028DD2309F4F3C089E00E94E43F47
:10A0200089E295E10F94B8530F945028CC2309F49A
:10A0300022C189E00E94E43F8AEE94E10F94B85374
:10A040000F945028002309F4CDCC89E00E94E43F0E
:10A050008BEA94E10F94B8530F945028C3CC88E650
:10A0600095E10F94314E0F945028DD2309F4C8C0B8
:10A0700089E00E94E43F89E295E10F94314E0F940C
:10A080005028CC2309F4F7C089E00E94E43F8AEE0F
:10A0900094E10F94314E0F945028002309F4A2CC80
:10A0A00089E00E94E43F8BEA94E10F94314ED4CFD3
:10A0B00088E695E10F94DC50682F880F770B880BAA
:10A0C000990B0E94294ADD2309F49AC089E00E9475
:10A0D000E43F89E295E10F94DC50682F880F770BFD
:10A0E000880B990B0E94294ACC2309F4C4C089E04B
:10A0F0000E94E43F8AEE94E10F94DC50682F880FB1
:10A10000770B880B990B0E94294A002309F46ACC2B
:10A1100089E00E94E43F8BEA94E10F94DC50682FC1
:10A12000880F770B880B990B0E94294A5BCC88E635
:10A1300095E10F94D3500F945028DD2309F460C0AB
:10A1400089E00E94E43F89E295E10F94D3500F9497
:10A150005028CC2309F48FC089E00E94E43F8AEEA6
:10A1600094E10F94D3500F945028002309F43ACC73
:10A1700089E00E94E43F8BEA94E10F94D3506CCFC6
:10A18000612F88E695E10E94454ADD2309F438C035
:10A1900089E00E94E43F173108F02DC0E12F012E25
:10A1A000000CFF0B8827E852FF4A8F4F0D946A6D11
:10A1B000E14CFB50054D2F4D5A4D8F4DE14D184E42
:10A1C000FB504E4EFB50874EFB50BF4EF14E444F5E
:10A1D000884FC64FED4F10503B506950A3508AE353
:10A1E0009BE09DCD80E49BE00E946F4209CE8DE212
:10A1F0000E94E43F98CE612F89E295E10E94454A92
:10A20000CC2309F438C089E00E94E43F173108F0FC
:10A210002DC0E12F012E000CFF0B8827ED5EFE4ABA
:10A220008F4F0D946A6DE94C3651114D3B4D664D83
:10A23000A74DF04D274E36515E4E3651974E365152
:10A24000CB4E064F584F994FD24FF74F1C504750A7
:10A250007A50AF5087E59BE072CD8DE59BE00E9480
:10A260006F42E3CD8DE20E94E43F6ECE612F8AEE15
:10A2700094E10E94454A002309F4B4CB89E00E948E
:10A28000E43F173138F5E12F012E000CFF0B882732
:10A29000E35BFE4A8F4F0D946A6DF04C6A511C4D82
:10A2A000474D724DBF4DFF4D364E6A516E4E6A514D
:10A2B000A74E6A51D74E1B4F6C4FAA4FDE4F01502D
:10A2C000285053508B50BB5084E79BE09FCC8AE7CB
:10A2D0009BE09CCC612F8BEA94E10E94454A82CBA3
:10A2E000FF920F931F93CF93DF93C82FD62F142F76
:10A2F000F22E8AE29DE00E946F420F2D212F4D2FFA
:10A300006C2F80E00E94A84C81E29DE00E946F4289
:10A31000212F4D2F6C2F82E00E94A84C85E19DE0FB
:10A320000E946F42212F4D2F6C2F83E00E94A84C7A
:10A3300089E09DE00E946F42212F4D2F6C2F84E019
:10A340000E94A84C8DEF9CE00E946F42212F4D2F60
:10A350006C2F85E00E94A84C81EF9CE00E946F4228
:10A36000212F4D2F6C2F86E00E94A84C84EE9CE09C
:10A370000E946F42212F4D2F6C2F87E00E94A84C26
:10A3800089ED9CE00E946F42212F4D2F6C2F89E0B8
:10A390000E94A84C8FEC9CE00E946F42212F4D2F11
:10A3A0006C2F8AE00E94A84C87EC9CE00E946F42D0
:10A3B000212F4D2F6C2F8BE00E94A84C8BEB9CE043
:10A3C0000E946F42212F4D2F6C2F8CE00E94A84CD1
:10A3D00083EB9CE00E946F42212F4D2F6C2F8DE06C
:10A3E0000E94A84C8CEA9CE00E946F42212F4D2FC6
:10A3F0006C2F8EE00E94A84C8DE99CE00E946F4279
:10A40000212F4D2F6C2F8FE00E94A84C85E99CE0F6
:10A410000E946F42212F4D2F6C2F80E10E94A84C8B
:10A420008AE89CE00E946F42212F4D2F6C2F81E122
:10A430000E94A84C8CE69CE00E946F42212F4D2F79
:10A440006C2F82E10E94A84C82E69CE00E946F4241
:10A45000212F4D2F6C2F83E10E94A84C87E59CE0B3
:10A460000E946F42212F4D2F6C2F84E10E94A84C37
:10A4700086E49CE00E946F42212F4D2F6C2F85E1D6
:10A480000E94A84C8EE39CE00E946F42212F4D2F2A
:10A490006C2F86E10E94A84C8EE29CE00E946F42E5
:10A4A000212F4D2F6C2F87E10E94A84C84E29CE065
:10A4B0000E946F42212F4D2F6C2F80E00E9442435B
:10A4C00088E19CE00E946F42212F4D2F6C2F88E085
:10A4D0000E9442438DE09CE00E946F42212F4D2F4D
:10A4E0006C2F8BE00E94424383E09CE00E946F420D
:10A4F000212F4D2F6C2F8AE00E9442438DEF9BE06D
:10A500000E946F42212F4D2F6C2F81E00E94424309
:10A5100088EF9BE00E946F42212F4D2F6C2F82E02D
:10A520000E94424383EF9BE00E946F42212F4D2FF8
:10A530006C2F83E00E9442438DEE9BE00E946F42AD
:10A54000212F4D2F6C2F84E00E94424387EE9BE029
:10A550000E946F42212F4D2F6C2F85E00E944243B5
:10A5600081EE9BE00E946F42212F4D2F6C2F86E0E1
:10A570000E9442438DED9BE00E946F42212F4D2FA0
:10A580006C2F87E00E9442438AEC9BE00E946F425E
:10A59000212F4D2F6C2F8CE00E9442438AE0DF91E7
:10A5A000CF911F910F91FF900C94E43FAF92BF9217
:10A5B000CF92DF92EF92FF920F931F93CF93DF938F
:10A5C00000D01F92CDB7DEB719821A821B821C827F
:10A5D00000E812E0CE0101967C0184E8A82E82E01A
:10A5E000B82EDD24D394CC24C394F80181918F013B
:10A5F0000E94562F882319F0F701C082D12CFFEF5B
:10A60000EF1AFF0AA016B10681F7DD2029F081E0DC
:10A6100089838A838B838C8383E50E94562F8823CA
:10A6200009F4D6C00E94E2318111C8C010924105E0
:10A630001092400507C07093410560934005672B59
:10A6400009F0D9C086E50E94562FDC80EB80FA80A5
:10A650001981882309F4ABC083EA91E10E946F421B
:10A660000D2D2E2D4F2D612F80E00E945F408BE934
:10A6700091E10E946F422E2D4F2D612F81E00E94AB
:10A680005F408FE891E10E946F422E2D4F2D612F88
:10A6900082E00E945F4087E891E10E946F422E2D88
:10A6A0004F2D612F83E00E945F4080E891E10E947E
:10A6B0006F422E2D4F2D612F84E00E945F4084E772
:10A6C00091E10E946F422E2D4F2D612F85E00E9457
:10A6D0005F408CE691E10E946F422E2D4F2D612F3D
:10A6E00086E00E945F4082E691E10E946F422E2D3B
:10A6F0004F2D612F87E00E945F4087E591E10E9426
:10A700006F422E2D4F2D612F88E00E945F408FE415
:10A7100091E10E946F422E2D4F2D612F89E00E9402
:10A720005F4085E491E10E946F422E2D4F2D612FF5
:10A730008AE00E945F408BE391E10E946F422E2DE0
:10A740004F2D612F8BE00E945F4082E391E10E94D8
:10A750006F422E2D4F2D612F8CE00E945F4087E2CB
:10A7600091E10E946F422E2D4F2D612F8DE00E94AE
:10A770005F408BE191E10E946F422E2D4F2D612FA2
:10A780008EE00E945F402D2D4E2D6F2D812F0F905A
:10A790000F900F900F90DF91CF911F910F91FF902D
:10A7A000EF90DF90CF90BF90AF900C947D422D2D15
:10A7B0004E2D6F2D812F0E947051E5CF84EF91E0D7
:10A7C000909341058093400586EE90E10E946F4290
:10A7D00080E50E949F2F882309F434CF0E94913195
:10A7E000643F41E0740708F426CF84EF91E0909332
:10A7F00041058093400586EE90E10E946F4222CF92
:10A80000CF92DF92EF92FF926A017B010E946F422A
:10A8100042E0C701B601FF90EF90DF90CF900C941B
:10A82000324C2F923F924F925F926F927F928F9213
:10A830009F92AF92BF92CF92DF92EF92FF920F93CF
:10A840001F93CF93DF93CDB7DEB7CB55D1090FB6AA
:10A85000F894DEBF0FBECDBF70E060E085E40E94DB
:10A86000B331182F81E0810F8230E8F08EE590E25D
:10A87000C55ADF4F0FB6F894DEBF0FBECDBFDF91D4
:10A88000CF911F910F91FF90EF90DF90CF90BF90ED
:10A89000AF909F908F907F906F905F904F903F9080
:10A8A0002F900C946F4265E070E083E40E94B33116
:10A8B000B82E60E085E50E94F23168968FAF689708
:10A8C00040E050E06CE872E417FD04C040E050E066
:10A8D00066E173E483E50E94FA320F94906B072ED1
:10A8E000000C880B990B0F94D46569837A838B8352
:10A8F0006C969FAF6C970F94054C6A8B7B8B8C8BFF
:10A900009D8B1F3F09F0AEC420E030E047E053E4E8
:10A9100069817A818B816C969FAD6C970F94846C62
:10A9200018160CF0D1C183E390E2A2CF20E030E012
:10A9300040E05EE32C962CAF3DAF4EAF5FAF2C975F
:10A940008AE999E9A9E1BFE360968CAF9DAFAEAF0C
:10A95000BFAF609761961FAF6197A8E3BFE16396B1
:10A96000BFAFAEAF6397E3E7FFE16596FFAFEEAF32
:10A970006597FCC1A8A5B9A52C9011963C9011979C
:10A9800012960C9112971396BC916B96BFAF6B9772
:10A9900069C26796EEADFFAD67978083C1C25BEE7B
:10A9A000C52ED12CE12CF12C64C324E130E040E031
:10A9B00050E02C873D874E875F8744E1C42ED12C21
:10A9C000E12CF12C64C3CC86DD86EE86FF865FC366
:10A9D0006796EEADFFAD679780832DC4D501C401A6
:10A9E0002BAD3CAD4DAD5EAD821B930BA40BB50BF7
:10A9F000B7FD5BC061968FAD61970E9416DB8AE060
:10AA00000E94E43FD501C4018053984FAF4FBF4F20
:10AA10008BAF9CAFADAFBEAF9FAD91117CC0249604
:10AA20002CAD3DAD4EAD5FAD2497B101802F6B963F
:10AA30009FAD6B970F94846C18160CF054C020E0F7
:10AA400030E040E050E4B101802F6B969FAD6B97F2
:10AA50000F94246A24966CAF7DAF8EAF9FAF24977E
:10AA60002AA93BA94CA95DA9280D391D4A1D5B1DCA
:10AA700028962CAF3DAF4EAF5FAF28972FA938ADCA
:10AA800049AD5AAD69817A818B816C969FAD6C9787
:10AA90000F94236A9101402F6B965FAD6B970F94D3
:10AAA000CD65881F8827881F8FAFD501C401880F07
:10AAB000991FAA1FBB1F4A895B896C897D898AA45B
:10AAC0009BA4ACA4BDA4480D591D6A1D7B1D841B0D
:10AAD000950BA60BB70B81389F44A241B105C8F175
:10AAE0008AE19FE147C2D501C40128962CAD3DAD56
:10AAF0004EAD5FAD2897821B930BA40BB50B6596EB
:10AB00004EAD5FAD65976CE97FE1B7FDCECF812F8C
:10AB10000E9471ADCACF20E030E040EA51E4698183
:10AB20007A818B816C969FAD6C970F94236A9B0101
:10AB3000AC01B101802F6B969FAD6B970F94CD65E3
:10AB400087FFB3CF63964EAD5FAD639763E67FE15A
:10AB5000DECF6A968EAC9FAC6A97A888B9888A14B3
:10AB60009B040CF0AEC09501233031050CF4A9C054
:10AB70008DEB9EE10E946F421F3F09F08AC04DEAB3
:10AB80005EE15D834C838BE99EE10E946F428C8184
:10AB90009D810E946F42B301A20189EB9EE10E9458
:10ABA00000548AE00E94E43F8BE99EE10E946F42DC
:10ABB0008C819D810E946F4248A159A16AA17BA10D
:10ABC00085EB9EE10E9400548AE00E94E43F8BE9FD
:10ABD0009EE10E946F428C819D810E946F424CA138
:10ABE0005DA16EA17FA181EB9EE10E9400548AE0ED
:10ABF0000E94E43F68968FAC6897882081F12CEA28
:10AC000035EC47E25EE368A179A18AA19BA10F948C
:10AC100033666B017C012CEA35EC47E25EE36CA104
:10AC20007DA18EA19FA10F941E6B1F3FB9F540928D
:10AC3000AC065092AD066092AE067092AF06C0921E
:10AC4000B006D092B106E092B206F092B3066093DD
:10AC5000B4067093B5068093B6069093B706C55AAE
:10AC6000DF4F0FB6F894DEBF0FBECDBFDF91CF919F
:10AC70001F910F91FF90EF90DF90CF90BF90AF901A
:10AC80009F908F907F906F905F904F903F902F900C
:10AC900008958CEA9EE19D838C8375CF27E1120293
:10ACA000F0011124E05EFB4E43865486658676866D
:10ACB000C786D08AE18AF28A638B748B858B968BE8
:10ACC000CECF0E947FEAAFC08FE190E20E946F4238
:10ACD0000E9490AC8FE78093AB062CE330E080E0DD
:10ACE00090E0A0E0B1E48FAB98AFA9AFBAAFA8EE07
:10ACF000B3E00F94146A6AAB7BAB8CAB9DAB2A8933
:10AD00003B894C895D89260F371F481F591F28969C
:10AD10002CAF3DAF4EAF5FAF289781E080935002DC
:10AD20001F3F09F003CE8BEA9AEAAAEABEE32C960B
:10AD30008CAF9DAFAEAFBFAF2C972DEC3CEC4CE48D
:10AD40005EE360962CAF3DAF4EAF5FAF609761960C
:10AD50001FAE61974FE45FE163965FAF4EAF6397BD
:10AD600089E89FE165969FAF8EAF65972A893B89F9
:10AD70004C895D892AA73BA74CA75DA72BAF3CAFA9
:10AD80004DAF5EAF8FE790E0A0E0B0E08C879D878D
:10AD9000AE87BF871CA21DA21EA21FA218A219A2C5
:10ADA0001AA21BA2412C512C32011C8290E49887DC
:10ADB000ACE1AA8FB6E4BB8F1C8E1D8E1E8E1F8E3B
:10ADC0001FAE24964CAE5DAE6EAE7FAE2497FFE70D
:10ADD000CF2ED12CE12CF12C1EA61FA618AA19AA41
:10ADE000E1E0EE8B198A188A212C312C00E06B9659
:10ADF0001FAE6B97F7E11F02C0011124805E9B4ECE
:10AE00009C01265F3F4F67963FAF2EAF6797AC011F
:10AE10004C5F5F4F59A748A78B2CBB0C99086A96CB
:10AE20009FAE8EAE6A9780915002882309F4A4C029
:10AE30000F94054C4B015C0120919A062EAB222306
:10AE400009F481C00E9455AD1F3F09F093CD2090B9
:10AE5000A5063090A6060091A7063091A8066B962D
:10AE60003FAF6B972C8D3D8D4E8D5F8DB101802F47
:10AE70006B969FAD6B970F94846C18163CF42C8ED8
:10AE80003D8E0E8F6B96EFAD6B97EF8F2C813885D3
:10AE90004A8D5B8DB101802F6B969FAD6B970F94A0
:10AEA000CD6587FF07C02C8238860A8F6B96FFAD71
:10AEB0006B97FB8F2E89222309F479C09101402FD3
:10AEC0006B965FAD6B9769817A818B816C969FAD34
:10AED0006C970F94CD6587FF36C0B501A4018AA594
:10AEE0009BA5ACA5BDA5481B590B6A0B7B0BDB01D1
:10AEF000CA0188589341A109B109B7FD24C08C85C6
:10AF00009D85AE85BF858C199D09AE09BF09B59594
:10AF1000A795979587951F3F09F03BCD8093AB068A
:10AF20004EA75FA768AB79ABF981FC8F2A812D8F83
:10AF30003B813E8F6C964FAD6C974F8F8A8A9B8A70
:10AF4000AC8ABD8A1E8A20E030E040EA51E4698183
:10AF50007A818B816C969FAD6C970F94246A9101D6
:10AF6000402F6B965FAD6B970F94CD6587FF36CD05
:10AF70008BEA9FE10E946F42C55ADF4F0FB6F894EB
:10AF8000DEBF0FBECDBFDF91CF911F910F91FF901C
:10AF9000EF90DF90CF90BF90AF909F908F907F9079
:10AFA0006F905F904F903F902F900C9490AC9101D8
:10AFB000402F6B965FAD6B9769817A818B816C9620
:10AFC0009FAD6C970F94846C18160CF0BCCFD50114
:10AFD000C4012A893B894C895D89821B930BA40B90
:10AFE000B50BAC01BD01485853416109710977FDAA
:10AFF000AACF48895989452B09F40CC12EA53FA534
:10B0000048A959A9280F391F4A1F5B1F2E8B3F8B58
:10B01000488F598F2EA53FA548A959A9281B390B40
:10B020004A0B5B0BC701B6010F94B0692E893F89AB
:10B03000488D598D0F94E269CC84DD84EE84FF84C1
:10B04000C20ED31EE41EF51E34E1C316D104E10482
:10B05000F1040CF4AACC4CEEC416D104E104F104C2
:10B060000CF09DCC50E8C516D104E104F1040CF4B9
:10B07000AACCCC86DD86EE86FF868EEF90E0A0E03F
:10B08000B0E08C199D09AE09BF096C017D0187E113
:10B0900090E20E946F426C857D858E859F850E941F
:10B0A000294A82E190E20E946F42C701B6010E94E4
:10B0B000294A4C8158856A8D7B8D8BE090E20E94F5
:10B0C00000544C8D5D8D6E8D7F8D84E090E20E94EA
:10B0D000005448895989433051050CF49BC0C7017D
:10B0E000B6010F94D46520E030E040E850E40F94BE
:10B0F00033662B013C012C8138854A8D5B8D6C8D2C
:10B100007D8D8E8D9F8D0F94236A2BED3FE049E45A
:10B1100050E40F94336620E030E040E05FE30F94AA
:10B1200033669B01AC01C301B2010F941E6B6887AB
:10B1300079878A879B876E897F89888D998D0F94FF
:10B14000D4652FE632E143E85AE30F9433666C830B
:10B150007D838E839F8360962CAD3DAD4EAD5FADFC
:10B160006097688579858A859B850F9433662B0166
:10B170003C01AC019B016C817D818E819F810F948C
:10B1800033662C962CAD3DAD4EAD5FAD2C970F9434
:10B1900033666CA37DA38EA39FA3A3019201C30179
:10B1A000B2010F94246A2C813D814E815F810F94FE
:10B1B0001E6B68A379A38AA39BA3488559856A85DA
:10B1C0007B858EEF9FE10E9400544C815D816E81F2
:10B1D0007F8188EF9FE10E94005488EE9FE10E94EA
:10B1E0006F42B301A20182EE9FE10E94005448A188
:10B1F00059A16AA17BA18CED9FE10E9400544CA152
:10B200005DA16EA17FA186ED9FE10E9400548AE0BE
:10B210000E94E43F8C859D85AE85BF858C0D9D1D6C
:10B22000AE1DBF1DB595A795979587951F3F09F052
:10B23000CFCB8093AB06288939892F5F3F4F398B5D
:10B24000288B39813C834A8148875B815A8F6C9671
:10B250008FAD6C978B8F8AA69BA6ACA6BDA69EA928
:10B260009E8B71CEE12E012E000CFF08F70183E0CA
:10B27000EE0FFF1F8A95E1F7E85BFD4F668177814E
:10B280006F507109072E000C880B990B0F94D46531
:10B290009B01AC0169817A818B816C969FAD6C9723
:10B2A0000F94846C18160CF43ECB8FE190E20E9450
:10B2B0006F420E9490AC87E18E9DF0018F9DF00D52
:10B2C0001124E05EFB4E8FE7828724E130E080E0CE
:10B2D00090E0A0E5B1E407CDCF92DF92EF92FF922C
:10B2E0000F931F93CF93DF93C0E8D2E06E0101E08C
:10B2F00010E0FF24F394F60181916F010E94562F14
:10B300008823C1F00E9476BE80913F049091400452
:10B310007801EE0CFF1CEE0CFF1C892B09F453C0C6
:10B320000E94D032F701EC54F44F60837183828322
:10B330009383F12C0F5F1F4F04301105E1F686E473
:10B340000E94562F882329F10E9476BE0E94D03297
:10B350006B017C0120E030E040E85FE30F94846CF7
:10B3600018160CF44BC020E030E0A901C701B6016B
:10B370000F94CD6587FD49C020E030E04FE753E4EE
:10B38000C701B6010F9433660F94976B6093C40B9B
:10B39000F12C83E50E94562F8823D9F10E9476BEB6
:10B3A0000E94D03260936A0270936B0280936C02A9
:10B3B00090936D02DF91CF911F910F91FF90EF90CD
:10B3C000DF90CF900895F801E555F44F6081662332
:10B3D00089F070E090E080E00F94D4659B01AC01AF
:10B3E000F701E456F44F60817181828193810F945B
:10B3F0001E6B98CF60E070E0CB0194CFC12CD12CB4
:10B4000030E8E32E3FE3F32EB7CFC12CD12C7601E9
:10B41000B3CFFF2079F28CEB90E10E946F428091D4
:10B42000C40B811104C089EB90E10E946F4280EB54
:10B4300090E10E946F428091C40BF4E68F9FC0019F
:10B44000112481589F4F6FEF70E00F94566D70E09C
:10B4500090E080E00F94D26520E030E048EC52E4C8
:10B460000F941E6BAB01BC018CE890E10E9400546C
:10B470008FE690E10E946F428DE490E10E946F425E
:10B4800008EB1BE080E20E94E43F89910E94E43FC8
:10B49000F80161917191819191918F0142E00E9437
:10B4A000324C8AE00E94E43FF2E0C338DF0751F7F4
:10B4B00040916A0250916B0260916C0270916D0232
:10B4C00089E290E10E9400548AE00E94E43F87E014
:10B4D00090E10E946F428091AC0B811117C0809166
:10B4E000AD0B811113C08091AE0B81110FC083EFA2
:10B4F0009FE00E946F428AE0DF91CF911F910F91F0
:10B50000FF90EF90DF90CF900C94E43F0CEA1BE0AB
:10B51000C1E0D0E0F80181918F01882341F180E200
:10B520000E94E43FFE01E158FD4F80810E94E43F0C
:10B53000F801319760816623F9F0CE01880F991FD9
:10B54000880F991F9C012456344F790170E090E0D8
:10B5500080E00F94D4659B01AC01F701608171819B
:10B56000828193810F941E6B42E00E94324C21969F
:10B57000C430D10579F6BFCF60E070E0CB01F4CFE5
:10B580008DE00E94E43F8AE00C94E43FE4E7F5E0BC
:10B590008081818381EE9CE10E946F4260917213F1
:10B5A0007091731380917413909175136F5F7F4F37
:10B5B0008F4F9F4F0E94294A0E94C05A0C945D4AA7
:10B5C0000F931F93CF938C01C62F8DEA9CE10E94AD
:10B5D0006F42C8010E946F428AE30E94E43F6C2FD1
:10B5E00070E090E080E00E94294ACF911F910F9176
:10B5F0000C94C05ACF93DF93EC018BEF9AE00E943A
:10B600006F42688179818A819B8140E10E94B449BF
:10B610000E94C05A8C8181FF04C08AEE9AE00E9489
:10B620006F428C8182FF04C086ED9AE00E946F42D7
:10B6300021E041E061E081E00E94705189EC9AE0F4
:10B64000DF91CF910C94E248CF93DF93EC01899185
:10B65000882319F00E94E43FFACFDF91CF910C9438
:10B66000C05A80917405909175052FEF3FEF9817A0
:10B6700051F0E92FF0E0EC58FA4F228130E09F5F63
:10B680009F7790937505C9010895CF92DF92EF924D
:10B69000FF920F931F93CF93DF9300E680911F0BD0
:10B6A000853008F02DC18091740590917505891B36
:10B6B0008F7709F425C10E94315BAC0197FDEECF75
:10B6C00020917013309171138A3019F08D3009F088
:10B6D000E4C010925A062115310519F40E947CAF7E
:10B6E000DDCF26503A4FF90110821092711310925B
:10B6F0007013CAEFD5E0FE018191803209F443C096
:10B700008E3409F0B6C061E17EE1CE010F944A6546
:10B710007C01892B41F06EE470E0CE0104960F9419
:10B72000BA6D009709F4CE014AE050E070E060E0A5
:10B7300001960F94CC62AB01BC014093F605509387
:10B74000F7056093F8057093F90580917213909155
:10B750007313A0917413B09175130196A11DB11DBF
:10B76000481759076A077B0781F0EF2871F48EEDBF
:10B770009DE1DF91CF911F910F91FF90EF90DF90AE
:10B78000CF900D94252AEF01B6CF6AE270E0CE018A
:10B790000F94E96D9C01009701F1982F9C1B10E01C
:10B7A000992339F09150FE01E90FF11D808118278E
:10B7B000F7CF4AE050E070E060E0C90101960F94D5
:10B7C000CC62C12ED12CF12CE12C6C157D058E059F
:10B7D0009F0531F08FEB9DE1CCCF85E99DE1C9CF8D
:10B7E0008091F6059091F705A091F805B091F905C3
:10B7F0008093721390937313A0937413B093751383
:10B800008091380281111CC067E470E0CE010F9472
:10B81000BA6D0097A9F04AE050E070E060E0019650
:10B820000F94CC62643071058105910548F484EF72
:10B830009CE10E946F4260E08AEE9CE10E942CD95C
:10B840008091FA058B3309F429CF80911F0B853045
:10B8500008F024CF80913B09809FC00111246AEF3A
:10B8600075E0825C964F0F94C56D81E00E94D62EE4
:10B8700015CF80919B1780FFC3CF61EC71E4CE019F
:10B880000F944A65009731F0FC01838180538A3020
:10B8900008F0B6CF8BE69DE16CCF2F3531050CF06B
:10B8A000FDCE8C35C1F40E94315B97FDF7CE20911F
:10B8B0005A062111F3CE2091701330917113A90112
:10B8C0004F5F5F4F509371134093701326503A4F60
:10B8D000F9018083E3CE8B3321F481E080935A0613
:10B8E000DDCE80915A068111D9CEC901019690937F
:10B8F00071138093701326503A4FF9014083CECED6
:10B90000DF91CF911F910F91FF90EF90DF90CF903B
:10B9100008954F925F926F927F928F929F92AF9213
:10B92000BF92CF92DF92EF92FF920F931F93CF932C
:10B93000DF93CDB7DEB7A0970FB6F894DEBF0FBE8A
:10B94000CDBF182F0E947FEA0F94054C6B017C013C
:10B95000009100020023F1F0809150058823D1F07E
:10B960004091030450910404609105047091060411
:10B9700026013701441A550A660A770AB301A20163
:10B9800077FD1AC0833009F4E6C00CF0D5C08130D1
:10B990000CF0DAC0202F30E0A8EEB3E00F94146A68
:10B9A000C60ED71EE81EF91EC0920304D0920404EE
:10B9B000E0920504F092060480911F0B853020F47C
:10B9C0000E94455B0E9432460F94054C6B017C013E
:10B9D00080914B0590914C05A0914D05B0914E057D
:10B9E0000097A105B10539F14091B8065091B9060B
:10B9F0006091BA067091BB06840F951FA61FB71FF2
:10BA000036014701681A790A8A0A9B0AD401C301E0
:10BA1000B7FD11C00E942E466091B50B7091B60B18
:10BA200088E299E00E941B468AE00E94E43F90E091
:10BA300080E00E94E2488091010290910202A09170
:10BA40000302B09104020097A105B10589F030917D
:10BA5000AA152091AB15321709F482C00F94054C3A
:10BA60006093B8067093B9068093BA069093BB06AC
:10BA700080911F04909120043599A6C0019690935F
:10BA8000200480931F0480911F04909120048E3E17
:10BA9000924054F00E942E4688E099E00E946F4246
:10BAA00090E080E00E94E2480F94054C00910B0466
:10BAB00010910C0420910D0430910E042B013C01D7
:10BAC000401A510A620A730A9301820137FD9BC032
:10BAD0008B019C010C53164F2F4F3F4F00930B04CB
:10BAE00010930C0420930D0430930E04079B0AC09E
:10BAF000069B08C0059B06C02091AB06211102C021
:10BB0000049908C0609307047093080480930904A3
:10BB100090930A04009107041091080420910904ED
:10BB200030910A04011511052105310509F052C0B3
:10BB30008091020160E05CC0843009F02BCF0E944C
:10BB40007A478FEB97E004C00E947A478EEE97E029
:10BB50000E946F421FCF0E947A4787ED97E0F8CF8F
:10BB60002091BE0621112DC011112BC04091B806A5
:10BB70005091B9066091BA067091BB06840F951F6B
:10BB8000A61FB71F46015701881A990AAA0ABB0ABD
:10BB9000D501C401B7FD15C080912104811168CF82
:10BBA00081E080932104179A8091AF0B8E7F809360
:10BBB000AF0B169A8091AF0B8D7F8093AF0B149AC9
:10BBC00057CF1092210454CF181619060CF05BCFF2
:10BBD000019755CF601B710B820B930B60567A4E09
:10BBE0008109910997FFA4CF8091020180956FEFA1
:10BBF000887080930001079B02C00699A1C070E085
:10BC000086E00F94FB4A0F94054C009113041091A9
:10BC1000140420911504309116044B015C01801A24
:10BC2000910AA20AB30AB7FC0EC08B019C010C500A
:10BC30001E4F2F4F3F4F0093130410931404209373
:10BC4000150430931604E0914005F09141053097BA
:10BC500009F41BC620910F04309110044091110487
:10BC6000509112042B013C01421A530A640A750ACE
:10BC700077FC0BC66E0F7F1F811D911D60930F0413
:10BC8000709310048093110490931204772473949A
:10BC900088E695E10E94AC2F298B3A8B4B8B5C8B0D
:10BCA0006D8B7E8B8F8B988F89899A89AB89BC89A4
:10BCB0000197A109B1098E3F9F4FAF4FBF4F08F0C9
:10BCC000F3C0B7FC93C08091A11561FF41C08F5FA5
:10BCD0008093A1158091A1158A3048F08AE00E94D6
:10BCE000E43F0E943E40CE0141960E94FA5A8D895F
:10BCF00080FF45C08091A015811141C00E940BCEEC
:10BD0000698F7A8F8B8F9C8F41E0613871458140BC
:10BD1000910508F440E0BE016F5F7F4FCE01499668
:10BD20000E94E0308AE00E94E43F8E010F5F1F4FC7
:10BD3000F80181918F01882381F00E94E43FF8CFC0
:10BD4000662319F068E770E05BCF70E060E058CFE1
:10BD5000882309F4BFCF8150BBCF88E298E00E94CE
:10BD60006F420E943E4060919E1570919F1585E044
:10BD700098E00E94114680E098E00E946F429D8901
:10BD80008091A01590FFE8C0853050F100919E157C
:10BD900010919F1588E695E10F94BD538823D9F043
:10BDA00005361105C0F0B8016253710970939F15F3
:10BDB00060939E1588E695E10F9453510E943E4092
:10BDC00060919E1570919F158BE298E00E9411463C
:10BDD0008AE00E94E43F8091A0159D8990FFBCC03D
:10BDE0008F5F8093A01581E08093A215772009F4DE
:10BDF0005BC088E695E10F94F651182F0E943E40F3
:10BE00008AE30E94E43F612F70E090E080E04AE026
:10BE10000E94B4498FE20E94E43F8E890F9450281B
:10BE20008FE20E94E43F8D8987FF9CC08F89988DA7
:10BE30000F9457288CE70E94E43F8091A115882336
:10BE400019F085E40E94E43F8D8981FF03C08FE4EF
:10BE50000E94E43F8D8980FF03C087E50E94E43F94
:10BE60008D8984FF03C087E40E94E43F8D8985FFAC
:10BE700003C084E50E94E43F8D8986FF03C089E406
:10BE80000E94E43F8091A215882319F086E40E9465
:10BE9000E43F8CE70E94E43F8091A01581110F944C
:10BEA000502889E00E94E43F89E295E10E94AC2F8E
:10BEB000298B3A8B4B8B5C8B6D8B7E8B8F8B988F0A
:10BEC00089899A89AB89BC890197A109B1098E3FFB
:10BED0009F4FAF4FBF4F08F0F5C0B7FC95C08091A2
:10BEE000621561FF43C08F5F809362158091621578
:10BEF0008A3048F08AE00E94E43F0E943B40CE0135
:10BF000041960E94FA5A8D8980FF47C08091611541
:10BF1000811143C00E940BCE698F7A8F8B8F9C8FCB
:10BF200041E0613871458140910508F440E0BE016F
:10BF30006F5F7F4FCE0149960E94E0308AE00E94F9
:10BF4000E43F8E010F5F1F4FF80181918F0188231D
:10BF500091F00E94E43FF8CF882309F447CF109274
:10BF6000A01544CF8DE20E94E43F64CF882309F4FA
:10BF7000BDCF8150B9CF8AE698E00E946F420E94FF
:10BF80003B4060915F157091601587E498E00E94D6
:10BF9000114682E498E00E946F429D89809161156C
:10BFA00090FFE8C0853050F100915F151091601549
:10BFB00089E295E10F94BD538823D9F00536110528
:10BFC000C0F0B801625371097093601560935F15FA
:10BFD00089E295E10F9453510E943B4060915F15B7
:10BFE000709160158DE698E00E9411468AE00E94EB
:10BFF000E43F809161159D8990FFBCC08F5F809365
:10C00000611581E080936315772009F45BC089E2B4
:10C0100095E10F94F651182F0E943B408AE30E944D
:10C02000E43F612F70E090E080E04AE00E94B44974
:10C030008FE20E94E43F8E890F9450288FE20E9485
:10C04000E43F8D8987FF9CC08F89988D0F94572876
:10C050008CE70E94E43F80916215882319F085E403
:10C060000E94E43F8D8981FF03C08FE40E94E43F7A
:10C070008D8980FF03C087E50E94E43F8D8984FF9E
:10C0800003C087E40E94E43F8D8985FF03C084E5F7
:10C090000E94E43F8D8986FF03C089E40E94E43F4B
:10C0A00080916315882319F086E40E94E43F8CE7B1
:10C0B0000E94E43F8091611581110F94502889E01E
:10C0C0000E94E43F8AEE94E10E94AC2F298B3A8BC8
:10C0D0004B8B5C8B6D8B7E8B8F8B988F89899A892C
:10C0E000AB89BC890197A109B1098E3F9F4FAF4F22
:10C0F000BF4F08F0F5C0B7FC95C08091231561FFD4
:10C1000043C08F5F80932315809123158A3048F0B8
:10C110008AE00E94E43F0E943840CE0141960E948E
:10C12000FA5A8D8980FF47C080912215811143C042
:10C130000E940BCE698F7A8F8B8F9C8F41E0613884
:10C1400071458140910508F440E0BE016F5F7F4F6B
:10C15000CE0149960E94E0308AE00E94E43F8E01C1
:10C160000F5F1F4FF80181918F01882391F00E948A
:10C17000E43FF8CF882309F447CF1092611544CFEC
:10C180008DE20E94E43F64CF882309F4BDCF815043
:10C19000B9CF8CEA98E00E946F420E9438406091CB
:10C1A00020157091211589E898E00E94114684E8D5
:10C1B00098E00E946F429D898091221590FFE8C00F
:10C1C000853050F100912015109121158AEE94E1EF
:10C1D0000F94BD538823D9F005361105C0F0B8017E
:10C1E0006253710970932115609320158AEE94E1D2
:10C1F0000F9453510E943840609120157091211581
:10C200008FEA98E00E9411468AE00E94E43F809104
:10C2100022159D8990FFBCC08F5F8093221581E01D
:10C2200080932415772009F45BC08AEE94E10F9483
:10C23000F651182F0E9438408AE30E94E43F612F94
:10C2400070E090E080E04AE00E94B4498FE20E94F2
:10C25000E43F8E890F9450288FE20E94E43F8D893D
:10C2600087FF9CC08F89988D0F9457288CE70E9478
:10C27000E43F80912315882319F085E40E94E43F70
:10C280008D8981FF03C08FE40E94E43F8D8980FF88
:10C2900003C087E50E94E43F8D8984FF03C087E4E3
:10C2A0000E94E43F8D8985FF03C084E50E94E43F3E
:10C2B0008D8986FF03C089E40E94E43F80912415A4
:10C2C000882319F086E40E94E43F8CE70E94E43F53
:10C2D0008091221581110F94502889E00E94E43F3B
:10C2E0008BEA94E10E94AC2F298B3A8B4B8B5C8BB1
:10C2F0006D8B7E8B8F8B988F89899A89AB89BC894E
:10C300000197A109B1098E3F9F4FAF4FBF4F08F072
:10C3100003C1B7FC95C08091E41461FF43C08F5FF7
:10C320008093E4148091E4148A3048F08AE00E94FB
:10C33000E43F0E943540CE0141960E94FA5A8D8911
:10C3400080FF47C08091E314811143C00E940BCE4F
:10C35000698F7A8F8B8F9C8F41E061387145814066
:10C36000910508F440E0BE016F5F7F4FCE01499612
:10C370000E94E0308AE00E94E43F8E010F5F1F4F71
:10C38000F80181918F01882391F00E94E43FF8CF5A
:10C39000882309F447CF1092221544CF8DE20E94E2
:10C3A000E43F64CF882309F4BDCF8150B9CF8EEE2E
:10C3B00098E00E946F420E9435406091E1147091B4
:10C3C000E2148BEC98E00E94114686EC98E00E9403
:10C3D0006F429D898091E31490FF94C0853050F1A5
:10C3E0000091E1141091E2148BEA94E10F94BD5393
:10C3F0008823D9F005361105C0F0B80162537109E0
:10C400007093E2146093E1148BEA94E10F9453511A
:10C410000E9435406091E1147091E21481EF98E040
:10C420000E9411468AE00E94E43F8091E3149D89B6
:10C4300090FF68C08F5F8093E31481E08093E514E0
:10C44000772009F46BC08BEA94E10F94F651182F12
:10C450000E9435408AE30E94E43F612F70E090E043
:10C4600080E04AE00E94B4498FE20E94E43F8E8956
:10C470000F9450288FE20E94E43F8D8987FF48C0C7
:10C480008F89988D0F9457288CE70E94E43F809104
:10C49000E414882319F085E40E94E43F8D8981FF2C
:10C4A00003C08FE40E94E43F8D8980FF03C087E5CD
:10C4B0000E94E43F8D8984FF03C087E40E94E43F2B
:10C4C0008D8985FF03C084E50E94E43F8D8986FF46
:10C4D00003C089E40E94E43F8091E514882319F0A9
:10C4E00086E40E94E43F8CE70E94E43F8091E314DD
:10C4F00081110F94502889E00E94E43F8AE00E9455
:10C50000E43F0CC0882309F49BCF1092E31498CF2A
:10C510008DE20E94E43FB8CF7110F0CF80911B04F0
:10C5200090911C04A0911D04B0911E0426013701B6
:10C53000481A590A6A0A7B0AD301C201B7FD8DC0A5
:10C540009091AA158091AB15209174029817D9F09B
:10C55000E091AB1536E5E39FF0011124ED5AF34F5E
:10C560008081289F90011124220F232F221F330B3B
:10C570003195122F8091AB159091AA15981771F0F3
:10C580008F5F8F70F9CF80910314289F9001112441
:10C59000220F232F221F330B3195122F112309F461
:10C5A00043C00F94054C8090170490901804A090FD
:10C5B0001904B0901A0481149104A104B10471F417
:10C5C0006C597F4F8F4F9F4F6093170470931804DF
:10C5D0008093190490931A041FEF06C06819790913
:10C5E0008A099B0997FDF8CF212F30E050E040E009
:10C5F0002150310941095109A9EBB0E00F94016ABA
:10C600002EEF30E040E050E00F94E26949015A011A
:10C6100086E4880E911CA11CB11CEFEF8E169104CC
:10C6200009F0DEC061E009C01092170410921804EE
:10C630001092190410921A0460E088E00F94964951
:10C64000F4E6CF0ED11CE11CF11CC0921B04D09269
:10C650001C04E0921D04F0921E040E947CAF8091A5
:10C660009406813009F072C00F94054C6B017C0177
:10C670008091260490912704A0912804B091290468
:10C6800026013701481A590A6A0A7B0AD301C201F6
:10C69000B7FD3AC08090950690909606A0909706B8
:10C6A000B09098060E940BCEAB01BC01409395065A
:10C6B00050939606609397067093980680912B0985
:10C6C00090912C09A0912D09B0912E0988199909F2
:10C6D000AA09BB09840F951FA61FB71F80932B09BA
:10C6E00090932C09A0932D09B0932E09D701C60170
:10C6F000805F984DAF4FBF4F8093260490932704DF
:10C70000A0932804B09329048091220490912304DB
:10C71000A0912404B091250436014701681A790AD2
:10C720008A0A9B0AD401C301B7FD10C020E8C20EDB
:10C730002EEED21EE11CF11CC0922204D0922304E2
:10C74000E0922404F09225040E94B3BD0E9499D87F
:10C7500080914605882369F10F94054C00914205AC
:10C76000109143052091440530914505601B710BE4
:10C77000820B930B97FD1DC00F94054C6B017C0140
:10C780002091460530E0A8EEB3E00F94146AC60E7F
:10C79000D71EE81EF91EC0924205D0924305E092D2
:10C7A0004405F092450580E00E9416DB8AE00E9475
:10C7B000E43FA0960FB6F894DEBF0FBECDBFDF9169
:10C7C000CF911F910F91FF90EF90DF90CF90BF908E
:10C7D000AF909F908F907F906F905F904F90089553
:10C7E00068E0CE0101960E94053FAF85AA2309F4B7
:10C7F00027CFE981FA816081288930E083E090E0E9
:10C80000AC01421B530B440F551F042E01C0880F6F
:10C810000A94EAF78095862362E070E001C0660F13
:10C820004A95EAF7862B80838FEF90E0A23021F0C3
:10C83000ED85FE85808191812D5F3F4F220F331F53
:10C8400044244394512C4C0E5D1E240D351DF901DA
:10C85000008111816FEF70E00F94426D90E080E0F5
:10C860000F94D2652B013C01B40190E080E00F945D
:10C87000D2659B01AC01C301B2010F9433660F94E2
:10C88000906BF80171836083DBCE712CB7FE00CA18
:10C8900045CE2F923F924F925F926F927F928F92EE
:10C8A0009F92AF92BF92CF92DF92EF92FF920F933F
:10C8B0001F93CF93DF93CDB7DEB763970FB6F8948E
:10C8C000DEBF0FBECDBF8091641183FD54C183E5EF
:10C8D0000E949F2F8887882309F448C10E94D03284
:10C8E0000F94906B6C3871050CF05EC17093AA06C2
:10C8F0006093A9060E9487966091A9067091AA0686
:10C90000072E000C880B990B0F94D4652091A50677
:10C910003091A6064091A7065091A8060F94846C0A
:10C9200018160CF444C18DE79EE160E00E942CD9FA
:10C9300081E0809350021A821B821C821D8219861C
:10C940001A861B861C8619821E862CE32F873CE1E3
:10C95000388B46E4498B312C212C50E85A8B8FEBD5
:10C960008B8B91E09D87812C912C54016091A906BD
:10C970007091AA06072E000C880B990B0F94D465B2
:10C980007B018C01232D322D4A895B890F94CD6563
:10C990008823B9F02091A5063091A6064091A706FC
:10C9A0005091A806A885B701C801A11103C10F9431
:10C9B000CD65881F8827881F89833E2C2F2C0A8BE2
:10C9C0001B8B0F94054C6B017C01DC01CB0129858D
:10C9D0003A854B855C85821B930BA40BB50BB7FD89
:10C9E0002EC0D701C60188519C4FAF4FBF4F8987DA
:10C9F0009A87AB87BC8780E00E9416DB89E79EE1BF
:10CA00000E946F4281149104A104B10409F4FAC098
:10CA1000C501B40168517C4F8F4F9F4F6C197D0940
:10CA20008E099F0928EE33E040E050E00F94C06982
:10CA3000CA01B9010E94294A8AE00E94E43F80E0CD
:10CA40000E94895C0F94054C6093B8067093B906F8
:10CA50008093BA069093BB069091A5069E83A09101
:10CA6000A606AF830091A7061091A806292F3A2F9A
:10CA7000A801632D722D8A899B890F94236A2B014B
:10CA80003C0120E030E0A9010F94846C87FF04C0D2
:10CA900077FA709477F8709420E030E040EA50E440
:10CAA000C301B20181149104A104B10409F0AEC024
:10CAB0000F94CD6587FF0BC0BD8546015701BB2391
:10CAC00031F028EE820E23E0921EA11CB11C3981A8
:10CAD0003323A9F18A819B81AC81BD81892B8A2B6B
:10CAE0008B2B61F0D701C6012A813B814C815D818E
:10CAF000821B930BA40BB50BB7FD21C02E813F8188
:10CB0000A8016E857F85888999890F94236A20E022
:10CB100030E040EC5FE30F94CD6587FD4FC0D70157
:10CB2000C601805A9541AF4FBF4F8A839B83AC8328
:10CB3000BD839E819E87AF81AF87088B198B8091C3
:10CB400050028823D9F181149104A104B10461F049
:10CB5000B8EECB1AB3E0DB0AE108F108C818D9082F
:10CB6000EA08FB08F7FE2AC01D8600CF82E50E9476
:10CB70009F2F8111B3CE63960FB6F894DEBF0FBE20
:10CB8000CDBFDF91CF911F910F91FF90EF90DF907C
:10CB9000CF90BF90AF909F908F907F906F905F905D
:10CBA0004F903F902F9008956CE870E09FCE8CE8F6
:10CBB0009EE1BBCE0F94CD6587FF1EC080915002D1
:10CBC0008823C9F263960FB6F894DEBF0FBECDBFBF
:10CBD000DF91CF911F910F91FF90EF90DF90CF9059
:10CBE000BF90AF909F908F907F906F905F904F908D
:10CBF0003F902F900C947ED93E2C2F2C0A8B1B8BB0
:10CC00001982DFCE8FE30E94E43F16CF0F94846C2D
:10CC100018160CF05CCF4601570159CFCF93DF9324
:10CC2000EC018881882349F18A3039F18D3029F16E
:10CC30008B33F9F080911F0B8530D8F480913B093C
:10CC400020E6829FC0011124BE01825C964F0F94A2
:10CC5000C56D80E00E94D62E0E947A47BE018BEC03
:10CC60009CE10E941B4688EC9CE1DF91CF910C94E3
:10CC70006F4280E00E94895CD4CFDF91CF9108950C
:10CC80002F923F924F925F926F927F928F929F92DC
:10CC9000AF92BF92CF92DF92EF92FF920F931F93CA
:10CCA000CF93DF93CDB7DEB7C854D1090FB6F89450
:10CCB000DEBF0FBECDBF382E0E94113382E50E9429
:10CCC0009F2F882309F44AC10E94D0326B017C0156
:10CCD00020E030E0A9010F94CD65882309F42EC12E
:10CCE00040905A0250905B0260905C0270905D022E
:10CCF00020915E0230915F0240916002509161028A
:10CD00002D8B3E8B4F8B588F80918406909185069A
:10CD1000A0918606B09187068D8F9E8FAF8FB8A3A6
:10CD2000209188063091890640918A0650918B06A1
:10CD30002DA33EA34FA358A79C01AD01C301B2018F
:10CD40000F94CD6581110DC02DA13EA14FA158A515
:10CD50006D897E898F89988D0F94CD65882309F41C
:10CD6000EDC020E030E0A901C701B6010F94CD6508
:10CD7000881F8827881F8311E8C080E090E0A0E822
:10CD8000BFE389A79AA7ABA7BCA7A30192016D8DAA
:10CD90007E8D8F8D98A10F94236A69A37AA38BA3AC
:10CDA0009CA32D893E894F89588D6DA17EA18FA1AD
:10CDB00098A50F94236A698F7A8F8B8F9C8F29A1F6
:10CDC0003AA14BA15CA1CA01B9010F9433664B0192
:10CDD0005C01298D3A8D4B8D5C8DCA01B9010F9490
:10CDE00033669B01AC01C501B4010F94246A0F9412
:10CDF000D26C4B015C01AC019B0160E070E080E80B
:10CE00009FE30F941E6B6DA77EA78FA798AB20E0C2
:10CE100030E040E05FE3C501B4010F9433664B019D
:10CE20005C01A7019601C701B6010F9433666B013F
:10CE30007C01A5019401C501B4010F9433669B01E7
:10CE4000AC01C701B6010F94236A0F94D26C29A5D7
:10CE50003AA54BA55CA50F9433664B015C01698D27
:10CE60007A8D8B8D9C8D90582DA53EA54FA558A9E8
:10CE70000F943366A50194010F9433666B017C0116
:10CE80002D8D3E8D4F8D58A1C301B2010F94246AA0
:10CE900020E030E040E05FE30F9433669B01AC019B
:10CEA000C701B6010F94246AA30192010F94236A6B
:10CEB0006B017C012DA13EA14FA158A56D897E89F2
:10CEC0008F89988D0F94246A20E030E040E05FE382
:10CED0000F9433662B013C012DA53EA54FA558A903
:10CEE00069A17AA18BA19CA10F943366A50194013D
:10CEF0000F9433669B01AC01C301B2010F94246A05
:10CF00002D893E894F89588D0F94236A6D8B7E8BB6
:10CF10008F8B988F20E030E0A901C701B6010F94F4
:10CF2000CD658111E8C020E030E0A9016D897E89DE
:10CF30008F89988D0F94CD658111DDC00E942E469A
:10CF400082EB9CE10E946F42AEC020E030E040E8FE
:10CF50005FEB29A73AA74BA75CA717CF89E40E94EC
:10CF60009F2FC12CD12C7601882321F00E94D03232
:10CF70006B017C018AE40E949F2F882309F4ADC0D5
:10CF80000E94D032C3CF20E030E0A901C501B40136
:10CF90000F94846C87FF22C2B7FAB094B7F8B094AC
:10CFA0001DC2498D5A8DBA0190E080E00F94D26580
:10CFB00029A13AA14BA15CA10F9433664B015C01FE
:10CFC0000F94196B6B017C01C501B4010F94C46C03
:10CFD0004B015C01A70196016D8D7E8D8F8D98A10F
:10CFE0000F9433662B013C012D893E894F89588D62
:10CFF000C501B4010F943366A30192010F94246A12
:10D000002B013C01A50194016D8D7E8D8F8D98A122
:10D010000F9433664B015C012D893E894F89588DF1
:10D02000C701B6010F9433669B01AC01C501B40181
:10D030000F94236A6DA37EA38FA398A759E159A7E4
:10D04000E0C280E1E4E8F6E0DE01119601900D9285
:10D050008A95E1F7C12CD12C80E8E82E8FE3F82ED9
:10D060008E010F5E1F4F9E01235F3F4FAE01475F52
:10D070005F4FBE016B5F7F4FCE0101960F94F53E6F
:10D0800080E1FE013196AAE5B2E001900D928A9509
:10D09000E1F70F94054C6093B8067093B90680933E
:10D0A000BA069093BB06C85BDF4F0FB6F894DEBF9D
:10D0B0000FBECDBFDF91CF911F910F91FF90EF90E9
:10D0C000DF90CF90BF90AF909F908F907F906F90A8
:10D0D0005F904F903F902F90089520E030E0A9019D
:10D0E000C701B6010F94CD65882309F427CF1D8AA7
:10D0F0001E8A1F8A188ED701C601B0588D8F9E8F49
:10D10000AF8FB8A32D893E894F89588D50582DA3D4
:10D110003EA34FA358A7A7019601C701B6010F94DC
:10D1200033664B015C012D893E894F89588DCA01B8
:10D13000B9010F9433669B01AC01C501B4010F9492
:10D14000246A0F94D26C69AF7AAF8BAF9CAF809199
:10D150005A0290915B02A0915C02B0915D0289A39A
:10D160009AA3ABA3BCA39C01AD01C701B6010F9468
:10D17000246A6DA77EA78FA798AB20915E0230919D
:10D180005F02409160025091610229A73AA74BA724
:10D190005CA72D893E894F89588D69A57AA58BA5F5
:10D1A0009CA50F94246A21966CAF7DAF8EAF9FAF84
:10D1B00021978091840690918506A0918606B09172
:10D1C000870689AB9AABABABBCAB2DA53EA54FA5F3
:10D1D00058A9BC01CD010F94236A6B017C012091F9
:10D1E00088063091890640918A0650918B062DABB6
:10D1F0003EAB4FAB58AF21962CAD3DAD4EAD5FADC4
:10D2000021976DA97EA98FA998AD0F94236A4B0130
:10D210005C018091620290916302A0916402B091DE
:10D22000650225968CAF9DAFAEAFBFAF25979C0131
:10D23000AD0160918C0670918D0680918E06909163
:10D240008F060F94236A698F7A8F8B8F9C8FA7012B
:10D2500096016D8D7E8D8F8D98A10F9433662B0175
:10D260003C01A50194016DA17EA18FA198A50F9409
:10D2700033669B01AC01C301B2010F94246A2B01F8
:10D280003C01A50194016D8D7E8D8F8D98A10F9429
:10D2900033664B015C01A70196016DA17EA18FA1B0
:10D2A00098A50F9433669B01AC01C501B4010F949E
:10D2B000236AA30192010F94A36A6B017C0120E011
:10D2C00030E0A9010F94CD6587FF0AC02BED3FE048
:10D2D00049EC50E4C701B6010F94246A6B017C014C
:10D2E0002BED3FE049EC50E4C701B6010F941E6BF3
:10D2F00020E030E040EC51E40F9433660F94026B71
:10D300000F94976B8B01672B11F401E010E0332031
:10D3100051F02BED3FE049EC50E4C701B6010F940A
:10D32000236A6B017C0120E030E0A901C701B6014E
:10D330000F94CD65811122C029A93AA94BA95CA9F6
:10D3400069A17AA18BA19CA10F94CD65811116C012
:10D350002DA93EA94FA958AD69A57AA58BA59CA575
:10D360000F94CD6581110AC008E110E02BEDC22EAB
:10D370002FE0D22E29ECE22E20E4F22EA701960116
:10D3800069AD7AAD8BAD9CAD0F9433664B015C01FA
:10D3900020E030E0A901698D7A8D8B8D9C8D0F94F2
:10D3A000CD65882309F4EFCDA5019401C501B40131
:10D3B0000F9433664B015C01298D3A8D4B8D5C8D4A
:10D3C000CA01B9010F9433669B01AC01C501B401D8
:10D3D0000F94246A0F94D26C4B015C012FE632E16A
:10D3E00043E85AE3C501B4010F94CD6587FD51CEE2
:10D3F00040906602509067026090680270906902E7
:10D40000C501B4010F94C66B0F94976B1B01601795
:10D41000710708F41801B10190E080E00F94D26523
:10D420004B015C01AC019B01C701B6010F941E6B5F
:10D4300069A37AA38BA39CA3A5019401698D7A8D1E
:10D440008B8D9C8D0F941E6B69AF7AAF8BAF9CAFA9
:10D45000A3019201609190067091910680919206CD
:10D46000909193060F94236AA50194010F941E6B6B
:10D4700029966CAF7DAF8EAF9FAF299729A13AA1B6
:10D480004BA15CA1CA01B9010F94336620E030E0E2
:10D4900040E05FE30F9433669B01AC0160E070E015
:10D4A00080E89FE30F94236A69AB7AAB8BAB9CABAC
:10D4B00025962CAD3DAD4EAD5FAD259729873A87BA
:10D4C0004B875C874D865E866F86788A60911202F4
:10D4D00070911302072E000C880B990B0F94D465E2
:10D4E00020915602309157024091580250915902B2
:10D4F0000F9433662AE037ED43E25CE30F94336622
:10D50000698B7A8B8B8B9C8B0F94054C9B01AC01A8
:10D5100028533F4F4F4F5F4F2DAB3EAB4FAB58AFF4
:10D520004D8C5E8C6F8C78A041E050E05A8F498F13
:10D5300059E159A7898D9A8D8215930508F081CDFF
:10D540000E947CAF0F94054C2DA93EA94FA958AD60
:10D55000621B730B840B950B97FD0FC00F94054C4A
:10D560009B01AC0128533F4F4F4F5F4F2DAB3EAB5C
:10D570004FAB58AF80E00E94895C39A5315039A784
:10D58000332309F40ECD9201A30169A17AA18BA1E5
:10D590009CA10F9433666B017C012DA13EA14FA18C
:10D5A00058A569A97AA98BA99CA90F9433669B01F8
:10D5B000AC01C701B6010F94246A6B017C01920192
:10D5C000A30169A97AA98BA99CA90F9433664B0181
:10D5D0005C012DA13EA14FA158A569A17AA18BA103
:10D5E0009CA10F9433669B01AC01C501B4010F945B
:10D5F000236A2B013C01C601D7018DA39EA3AFA3D3
:10D60000B8A79201A3016DA57EA58FA598A90F9437
:10D61000246A69837A838B839C832DA13EA14FA1C9
:10D6200058A521966CAD7DAD8EAD9FAD21970F9421
:10D63000246A6D837E838F83988729AD3AAD4BAD85
:10D640005CAD69857A858B859C850F94246A698792
:10D650007A878B879C8729962CAD3DAD4EAD5FAD0B
:10D6600029976D857E858F8598890F94246A6D87AB
:10D670007E878F87988B80913D02882321F0CE0191
:10D6800001960E943DC3C12CD12C90E8E92E9FE366
:10D69000F92E8E010F5E1F4F9E01235F3F4FAE019B
:10D6A000475F5F4FBE016B5F7F4FCE0101960F94C6
:10D6B000F53E882309F4C5CC898D9A8D01969A8F01
:10D6C000898F38CF2F923F924F925F926F927F92C5
:10D6D0008F929F92AF92BF92CF92DF92EF92FF9282
:10D6E0000F931F93CF93DF93CDB7DEB7CB5FD109F5
:10D6F0000FB6F894DEBF0FBECDBF81E00E94AE3EF4
:10D7000041E061E081E00E94CFC3882311F0912CB9
:10D710002EC08091B70B811112C08CE3FE013196AF
:10D72000DF011D928A95E9F73090B70B8AE40E94D9
:10D73000562F982E882351F00E94243EE8CF60E0B7
:10D740008FE40E94F231882341F3E1CF70E060E082
:10D7500086E50E94B331CF52DF4F99838883C15D44
:10D76000D040059710F18BEC9FE00E946F4280E063
:10D770000E94AE3E892DC550DF4F0FB6F894DEBF34
:10D780000FBECDBFDF91CF911F910F91FF90EF9012
:10D79000DF90CF90BF90AF909F908F907F906F90D1
:10D7A0005F904F903F902F90089560E084E40E9436
:10D7B000F231C551DF4F8883CB5ED040CF52DF4F6F
:10D7C00008811981C15DD0400330110504F560E086
:10D7D00084E50E94F231C351DF4F8883CD5ED04093
:10D7E00062E070E088E50E94B331182F62E070E0DB
:10D7F00089E50E94B331082F80E50E949F2F811197
:10D800000DC0812F823071F082EA9FE0AECF11E02F
:10D81000C351DF4F1883CD5ED040E2CF0E94AF31BD
:10D82000082FF0CF89E79FE0023009F09ECF40E05B
:10D8300050E86BEB75E483E50E94FA3220E030E0BB
:10D8400040E752E40F941E6B6093520270935302B0
:10D85000809354029093550288E40E94562F8823A7
:10D8600009F4A0C00E94D0320F94906B8B0177FF17
:10D8700002C00F5F1F4F159507951195019511096E
:10D88000025B1F4F58010D3F2FEF120724F45DEF8D
:10D89000A52EBB24BA946501C60ED71E33EAC31663
:10D8A000D1041CF043EAC42ED12C0C3F4FEF1407D7
:10D8B00014F40CEF1FEF7801E60EF71E58EAE51698
:10D8C000F1040CF0A1C0B801012E000C880B990BDB
:10D8D0000F94D465C552DF4F688379838A839B8315
:10D8E000CB5DD040B5010B2C000C880B990B0F942D
:10D8F000D465C152DF4F688379838A839B83CF5D70
:10D90000D040C552DF4F288139814A815B81CB5D90
:10D91000D0400E94EB2E882309F47AC0B7010F2C67
:10D92000000C880B990B0F94D4652B013C01B601B8
:10D930000D2C000C880B990B0F94D465A301920158
:10D940000E94EB2EC451DF4F8883CC5ED0408823E9
:10D9500009F45EC0CF52DF4F88819981C15DD0400C
:10D96000892B91F087E49FE00E946F42C551DF4F01
:10D970009881CB5ED040992321F08DE39FE00E94F7
:10D980006F428AE00E94E43F0E9476BE80E00E94DF
:10D99000AB3381E00E947BC68823E9F1832D0E948E
:10D9A000AB33E5CE8CE40E949F2F3DEFA32EBB242A
:10D9B000BA94882329F00E94D0320F94906B5B01B7
:10D9C00082E50E949F2F23EAC22ED12C882329F0C2
:10D9D0000E94D0320F94906B6B0186E40E949F2FBF
:10D9E0000CEF1FEF882329F00E94D0320F94906B28
:10D9F0008B0182E40E949F2F882331F00E94D03255
:10DA00000F94906B7B015FCF98EAE92EF12C5BCFEE
:10DA10008DE59FE0AACE0E9452C460E085E40E949A
:10DA2000F231882309F421C3A1E0CD51DF4FA8834F
:10DA3000C35ED040C952DF4F1882C75DD040CB5380
:10DA4000DF4F19821882C55CD040EFEFFFEFCB5457
:10DA5000DF4FF983E883C55BD040CD52DF4F18829A
:10DA600019821A821B82C35DD040C354DF4F1882D3
:10DA700019821A821B82CD5BD040FFEFC353DF4F68
:10DA8000F883CD5CD0402FEFC753DF4F2883C95CAC
:10DA9000D04031E0CF54DF4F3883C15BD040CA184B
:10DAA000DB08C601DD0CAA0BBB0BC251DF4F88831C
:10DAB0009983AA83BB83CE5ED040E01AF10A870126
:10DAC000FF0C220B330BCA50DF4F088319832A83C4
:10DAD0003B83C65FD0402CE0CB54DF4F08811981D7
:10DAE000C55BD040209FC001219F900D11248C0167
:10DAF0000F5A194EC754DF4F19830883C95BD040B2
:10DB0000CB54DF4F88819981C55BD0400196880F47
:10DB1000991F880F991F0DE610E00C0F1D1F080FAD
:10DB2000191FC951DF4F19830883C75ED0400DE329
:10DB300010E00C0F1D1F080F191FCF53DF4F198363
:10DB40000883C15CD040CB53DF4F28813981C55C4D
:10DB5000D040032E000C440B550BCE50DF4F2883D2
:10DB600039834A835B83C25FD040CB53DF4F088148
:10DB70001981C55CD040000F111FC650DF4F1983BB
:10DB80000883CA5FD040C753DF4F1881C95CD040BB
:10DB9000CF54DF4F0881C15BD040101709F4C2C2D7
:10DBA000C251DF4F688179818A819B81CE5ED040EE
:10DBB0000F94D4656B017C01CE50DF4F6881798171
:10DBC0008A819B81C25FD0400F94D4659B01AC01D8
:10DBD000C701B6010F943366C152DF4F28813981E6
:10DBE0004A815B81CF5DD0400F94246A4B015C0178
:10DBF000CA50DF4F688179818A819B81C65FD0409E
:10DC00000F94D4656B017C01602F000F770B880B9C
:10DC1000990B0F94D4659B01AC01C701B6010F9419
:10DC20003366C552DF4F288139814A815B81CB5DE4
:10DC3000D0400F94246A6B017C0120E030E0A90100
:10DC4000C501B4010F94CD6587FF5FC260E070E04D
:10DC5000CB01A50194010F94246A0F94C66BC7559C
:10DC6000DF4F688379838A839B83C95AD04020E041
:10DC700030E0A901C701B6010F94CD6587FF4AC204
:10DC800060E070E0CB01A70196010F94246A0F9425
:10DC9000C66BC355DF4F688379838A839B83CD5AD4
:10DCA000D040CB54DF4F08811981C55BD0400F5F56
:10DCB0001F4FCB54DF4F19830883C55BD040C6503C
:10DCC000DF4FE881F981CA5FD040CF54DF4F188120
:10DCD000C15BD040E10FF11D17FDFA95EE0FFF1F5C
:10DCE00021EA30E02C0F3D1FE20FF31FCB54DF4F32
:10DCF00008811981C55BD04011830083CF52DF4F6B
:10DD00002881C15DD040CD51DF4F4881C35ED040F6
:10DD1000BE0163557F4FCE0187559F4F0F94024040
:10DD2000C354DF4F688379838A839B83CD5BD04064
:10DD30009B01AC010F94166D8111F1C1C354DF4FEB
:10DD4000288139814A815B81CD5BD040CD52DF4F44
:10DD5000688179818A819B81C35DD0400F94246A58
:10DD6000CD52DF4F688379838A839B83C35DD04024
:10DD7000C951DF4FA881B981C75ED040C354DF4F7E
:10DD8000288139814A815B81CD5BD0402D933D93C1
:10DD90004D935D93C951DF4FB983A883C75ED040CF
:10DDA000C755DF4FC880D980EA80FB80C95AD04070
:10DDB000CF53DF4FE881F981C15CD040C192D1924D
:10DDC000E192F192CF53DF4FF983E883C15CD040F9
:10DDD000C355DF4F288039804A805B80CD5AD040C0
:10DDE000248635864686578600E010E020E83FE32B
:10DDF000048F158F268F378FA701960169817A814D
:10DE00008B819C810F94246A69837A838B839C83A2
:10DE1000A20191016D817E818F8198850F94246A82
:10DE20006D837E838F839887C354DF4F2881398128
:10DE30004A815B81CD5BD04069857A858B859C85E5
:10DE40000F94246A69877A878B879C87A70196013C
:10DE5000C701B6010F9433669B01AC016D857E85C9
:10DE60008F8598890F94246A6D877E878F87988B1A
:10DE7000A2019101C201B1010F9433669B01AC0173
:10DE800069897A898B899C890F94246A698B7A8B3A
:10DE90008B8B9C8BC354DF4F288139814A815B81F6
:10DEA000CD5BD040CA01B9010F9433669B01AC0130
:10DEB0006D897E898F89988D0F94246A6D8B7E8BF6
:10DEC0008F8B988FA2019101C701B6010F94336621
:10DED0009B01AC01698D7A8D8B8D9C8D0F94246A8A
:10DEE000698F7A8F8B8F9C8FA7019601C354DF4F68
:10DEF000688179818A819B81CD5BD0400F943366A4
:10DF00009B01AC016D8D7E8D8F8D98A10F94246A3D
:10DF10006D8F7E8F8F8F98A3A2019101C354DF4F25
:10DF2000688179818A819B81CD5BD0400F94336673
:10DF30009B01AC0169A17AA18BA19CA10F94246AD9
:10DF400069A37AA38BA39CA36DA07EA00FA118A5A3
:10DF500020E030E0A901C701B6010F94846C4601AE
:10DF6000570187FF04C0B7FAB094B7F8B094A50181
:10DF70009401B301C8010F94CD6587FF02C034013D
:10DF80008501C301D8018DA39EA3AFA3B8A769A43F
:10DF90007AA40BA51CA520E030E0A901C201B101C3
:10DFA0000F94846C5201410187FF04C0B7FAB0940A
:10DFB000B7F8B094A5019401B301C8010F94CD65E1
:10DFC00087FF02C034018501C301D80189A79AA740
:10DFD000ABA7BCA720E030E040E85FE369AD7AADD5
:10DFE0008BAD9CAD0F94246A69AF7AAF8BAF9CAFB9
:10DFF000C754DF4FE881F981C95BD040C486D5861C
:10E00000E686F786208A318A428A538AC354DF4FD4
:10E01000088119812A813B81CD5BD040048B158B0F
:10E02000268B378B80E00E94895CCF54DF4F0881BC
:10E03000C15BD040C353DF4F1881CD5CD040010F8E
:10E04000CF54DF4F0883C15BD040C754DF4F0881F6
:10E050001981C95BD040045F1F4FC754DF4F19833C
:10E060000883C95BD040312C8ECDB2E0CD51DF4F5B
:10E07000B883C35ED040DECCC354DF4F28813981E2
:10E080004A815B81CD5BD040CA01B9010F94166D06
:10E09000811152C081E0C952DF4F1881C75DD04065
:10E0A0001827C952DF4F1883C75DD0401123D1F024
:10E0B00001E0C353DF4F0883CD5CD04012E0C7536B
:10E0C000DF4F1883C95CD040CF54DF4F1882C15B4B
:10E0D000D04001E010E0CB53DF4F19830883C55CCB
:10E0E000D040F9CC0FEFC353DF4F0883CD5CD04055
:10E0F0001FEFC753DF4F1883C95CD04001E0CF54F6
:10E10000DF4F0883C15BD040E4CF60E070E080E087
:10E110009FE39FCD60E070E080E09FE3B4CD832D6E
:10E120000E94AB33CB53DF4F08811981C55CD040CF
:10E130000130110509F0A0CF80E00E947BC6882342
:10E1400049F1832D0E94AB3320E030E040EC5FE7E3
:10E15000C354DF4F288339834A835B83CD5BD04030
:10E160000E9439C48091B70B81110E9473C50E942F
:10E17000F5DC99249394C354DF4F288139814A8177
:10E180005B81CD5BD040CA01B9010F94166D81113E
:10E19000EECABDCAC354DF4F288139814A815B81F1
:10E1A000CD5BD040CA01B9010F94166D8111D8CF53
:10E1B000C9ACDAACEBACFCAC20E030E0A901C701A3
:10E1C000B6010F94CD65882309F404C2A701960116
:10E1D00069817A818B819C810F941E6BCF54DF4FB4
:10E1E000688379838A839B83C15BD04069837A8308
:10E1F0008B839C83A70196016D817E818F81988599
:10E200000F941E6BCB54DF4F688379838A839B8383
:10E21000C55BD0406D837E838F839887A70196016D
:10E2200069857A858B859C850F941E6BC754DF4F5B
:10E23000688379838A839B83C95BD04069877A87A7
:10E240008B879C87A70196016D857E858F85988930
:10E250000F941E6B4B015C01CF54DF4F2881398135
:10E260004A815B81C15BD040CA01B9010F9433661A
:10E270009B01AC01C501B4010F94236ACF53DF4F5A
:10E28000688379838A839B83C15CD0406D877E8756
:10E290008F87988BA701960169897A898B899C89D8
:10E2A0000F941E6B4B015C01CB54DF4F28813981E9
:10E2B0004A815B81C55BD040CA01B9010F943366C6
:10E2C0009B01AC01C501B4010F94236ACB53DF4F0E
:10E2D000688379838A839B83C55CD040698B7A8B02
:10E2E0008B8B9C8BA70196016D897E898F89988D78
:10E2F0000F941E6B4B015C01C754DF4F288139819D
:10E300004A815B81C95BD040CA01B9010F94336671
:10E310009B01AC01C501B4010F94236A6D8B7E8B08
:10E320008F8B988FA7019601698D7A8D8B8D9C8D2F
:10E330000F941E6B4B015C01CB54DF4F2881398158
:10E340004A815B81C55BD040CF54DF4F68817981C2
:10E350008A819B81C15BD0400F9433669B01AC01E5
:10E36000C501B4010F94236A4B015C01898E9A8E1A
:10E37000AB8EBC8EA701960169A17AA18BA19CA14D
:10E380000F941E6B2B013C01C754DF4F288139814C
:10E390004A815B81C95BD040CB54DF4F6881798172
:10E3A0008A819B81C55BD0400F9433669B01AC0191
:10E3B000C301B2010F94236AC753DF4F6883798387
:10E3C0008A839B83C95CD04069A37AA38BA39CA357
:10E3D000A70196016D8D7E8D8F8D98A10F941E6B78
:10E3E0006B017C01C754DF4F288139814A815B81F1
:10E3F000C95BD040CF54DF4F688179818A819B818E
:10E40000C15BD0400F9433669B01AC01C701B601DC
:10E410000F94236AC353DF4F688379838A839B8376
:10E42000CD5CD0406D8F7E8F8F8F98A3CB53DF4F05
:10E43000288139814A815B81C55CD040CF53DF4F51
:10E44000688179818A819B81C15CD0400F94336659
:10E450006B017C01A5019401C501B4010F943366E1
:10E460009B01AC01C701B6010F94236A6B017C01CB
:10E4700020E030E0A9010F94846C2601370187FF6A
:10E4800004C077FA709477F8709429A53AA54BA543
:10E490005CA56DA17EA18FA198A50F94246A2FEF92
:10E4A00036EE4BED5EE20F943366A30192010F94BA
:10E4B000846C87FF8FC0C753DF4F288139814A8121
:10E4C0005B81C95CD040C501B4010F9433662B0158
:10E4D0003C01C353DF4F288139814A815B81CD5C88
:10E4E000D040CB53DF4F688179818A819B81C55CA5
:10E4F000D0400F9433669B01AC01C301B2010F946D
:10E50000236AA70196010F941E6B2B013C014DA6B7
:10E510005EA66FA678AAC353DF4F288139814A814E
:10E520005B81CD5CD040C501B4010F9433664B01D3
:10E530005C01C753DF4F288139814A815B81C95C07
:10E54000D040CF53DF4F688179818A819B81C15C44
:10E55000D0400F9433669B01AC01C501B4010F9408
:10E56000236AA70196010F941E6B6B017C01C9AA57
:10E57000DAAAEBAAFCAAA3019201CF54DF4F68816B
:10E5800079818A819B81C15BD0400F943366C754E7
:10E59000DF4F288139814A815B81C95BD0400F946C
:10E5A000246A4B015C01A7019601CB54DF4F6881BF
:10E5B00079818A819B81C55BD0400F9433669B0132
:10E5C000AC01C501B4010F94246A90586DAB7EABC9
:10E5D0008FAB98AF8DA59EA5AFA5B8A9CB54DF4F43
:10E5E00088839983AA83BB83C55BD040B058C75446
:10E5F000DF4F88839983AA83BB83C95BD04009A975
:10E600001AA92BA93CA9CF53DF4F088319832A836A
:10E610003B83C15CD04020E030E040E85EE3CD5277
:10E62000DF4F688179818A819B81C35DD0400F94DF
:10E630003366CD52DF4F688379838A839B83C35DC2
:10E64000D040CF52DF4F08811981C15DD040012BEE
:10E6500009F46BC22DA93EA94FA958ADC951DF4F8E
:10E66000288339834A835B83C75ED0404090651618
:10E67000509066166090671670906816209171161B
:10E68000309172164091731650917416C301B20105
:10E690000F94236AC952DF4F688379838A839B83EF
:10E6A000C75DD040C0906116D0906216E0906316AE
:10E6B000F090641620916D1630916E1640916F1691
:10E6C00050917016C701B6010F94236AC552DF4FEF
:10E6D000688379838A839B83CB5DD04080905D166D
:10E6E00090905E16A0905F16B0906016209169160B
:10E6F00030916A1640916B1650916C16C501B401A9
:10E700000F94236AC152DF4F688379838A839B8386
:10E71000CF5DD0408091591690915A16A0915B160A
:10E72000B0915C16CB53DF4F88839983AA83BB8358
:10E73000C55CD040A3019201BC01CD010F94236AB6
:10E74000CD51DF4F688379838A839B83C35ED0403A
:10E750000091551610915616209157163091581663
:10E76000C753DF4F088319832A833B83C95CD0409A
:10E77000A7019601C753DF4F688179818A819B8108
:10E78000C95CD0400F94236A6B017C012091511623
:10E79000309152164091531650915416C353DF4F87
:10E7A000288339834A835B83CD5CD040A5019401E3
:10E7B000C353DF4F688179818A819B81CD5CD040D2
:10E7C0000F94236A4B015C01C552DF4F28813981C8
:10E7D0004A815B81CB5DD0400F9433662B013C01B5
:10E7E000C152DF4F288139814A815B81CF5DD040A2
:10E7F000C701B6010F9433669B01AC01C301B2019E
:10E800000F94236ACF54DF4F688379838A839B8375
:10E81000C15BD040C152DF4F288139814A815B8181
:10E82000CF5DD040CD51DF4F688179818A819B8156
:10E83000C35ED0400F9433662B013C01C952DF4FB9
:10E84000288139814A815B81C75DD040C501B4010F
:10E850000F9433669B01AC01C301B2010F94236A8C
:10E860002B013C01C952DF4F288139814A815B81EC
:10E87000C75DD040C701B6010F9433666B017C01C0
:10E88000C552DF4F288139814A815B81CB5DD04001
:10E89000CD51DF4F688179818A819B81C35ED040F1
:10E8A0000F9433669B01AC01C701B6010F94236A34
:10E8B0006B017C0120917516309176164091771688
:10E8C000509178160F9433664B015C0120917916B4
:10E8D00030917A1640917B1650917C16C301B2019B
:10E8E0000F9433669B01AC01C501B4010F94246AF7
:10E8F0004B015C0120917D1630917E1640917F1670
:10E9000050918016CF54DF4F688179818A819B8135
:10E91000C15BD0400F9433669B01AC01C501B401CB
:10E920000F94246A4B015C01C353DF4F68817981E6
:10E930008A819B81CD5CD0409058A70196010F94AD
:10E940003366C353DF4F688379838A839B83CD5CAF
:10E95000D040C753DF4F288139814A815B81C95C30
:10E96000D040C301B2010F9433669B01AC01C35385
:10E97000DF4F688179818A819B81CD5CD0400F9483
:10E98000236AC753DF4F688379838A839B83C95C7B
:10E99000D040CB53DF4F288139814A815B81C55CF0
:10E9A000D040CF54DF4F688179818A819B81C15BE0
:10E9B000D0400F9433669B01AC01C753DF4F688191
:10E9C00079818A819B81C95CD0400F94236A9B0125
:10E9D000AC01C501B4010F94246A4B015C0120E035
:10E9E00030E0A9010F94846C181624F0B7FAB094A3
:10E9F000B7F8B094A7019601C701B6010F9433662A
:10EA00006B017C01A3019201C301B2010F94336633
:10EA10009B01AC01C701B6010F94246A6B017C0114
:10EA2000CF54DF4F288139814A815B81C15BD0405F
:10EA3000CA01B9010F9433669B01AC01C701B6014D
:10EA40000F94246A0F94D26C9B01AC01C501B401F0
:10EA50000F941E6BAB01BC0186E19FE00E94005445
:10EA60008AE00E94E43F09E613E0D8018D918D0110
:10EA7000882319F00E94E43FF8CF48E0C754DF4FE5
:10EA8000688179818A819B81C95BD0400E94324C28
:10EA90000FE713E0F80181918F01882319F00E949C
:10EAA000E43FF8CF48E0CF53DF4F688179818A8116
:10EAB0009B81C15CD04090580E94324C04E813E026
:10EAC000D8018D918D01882319F00E94E43FF8CF81
:10EAD000C951DF4F688179818A819B81C75ED040AF
:10EAE000905848E00E94324CCF52DF4F0881198184
:10EAF000C15DD04003301105ACF009E813E0D80146
:10EB00008D918D01882319F00E94E43FF8CF48E0F1
:10EB1000CD52DF4F688179818A819B81C35DD0406E
:10EB20000E94324C8AE00E94E43FC551DF4F0881C9
:10EB3000CB5ED0400111E9C1CB54DF4F2881398130
:10EB40004A815B81C55BD040CB56DF4F2883398338
:10EB50004A835B83C559D040CF53DF4F8881998169
:10EB6000AA81BB81C15CD040C756DF4F888399839F
:10EB7000AA83BB83C959D040C12CD12C70E8E72EA1
:10EB80007FE3F72EC356DF4FC882D982EA82FB8229
:10EB9000CD59D040CE018B569F4F0F947557C75714
:10EBA000DF4FC882D982EA82FB82C958D040C3575E
:10EBB000DF4F188219821A821B82CD58D040C75469
:10EBC000DF4F088119812A813B81C95BD040CF5634
:10EBD000DF4F088319832A833B83C159D040CE017C
:10EBE00087579F4F0F947557CB56DF4F2881398138
:10EBF0004A815B81C559D040CF54DF4F2883398388
:10EC00004A835B83C15BD040C357DF4F88819981C2
:10EC1000AA81BB81CD58D040CB54DF4F88839983E4
:10EC2000AA83BB83C55BD040C756DF4F488059805D
:10EC30006A807B80C959D040C757DF4F088119814E
:10EC40002A813B81C958D040C754DF4F08831983BC
:10EC50002A833B83C95BD040C356DF4F88809980AD
:10EC6000AA80BB80CD59D040CF56DF4FC880D98015
:10EC7000EA80FB80C159D040A7019601C301B201CF
:10EC80000F943366CF53DF4F688379838A839B83E6
:10EC9000C15CD040A5019401CB54DF4F68817981DC
:10ECA0008A819B81C55BD0400F9433669B01AC0188
:10ECB000CF53DF4F688179818A819B81C15CD040CD
:10ECC0000F94236AC358DF4F688379838A839B83B9
:10ECD000CD57D040A5019401C754DF4F6881798199
:10ECE0008A819B81C95BD0400F9433664B015C01E4
:10ECF000A7019601CF54DF4F688179818A819B817A
:10ED0000C15BD0400F9433669B01AC01C501B401D7
:10ED10000F94236ACF57DF4F688379838A839B835D
:10ED2000C158D040CB54DF4F288139814A815B8163
:10ED3000C55BD040CF54DF4F688179818A819B8148
:10ED4000C15BD0400F9433666B017C01C754DF4F29
:10ED5000288139814A815B81C95BD040C301B201FE
:10ED60000F9433669B01AC01C701B6010F94236A6F
:10ED7000CB57DF4F688379838A839B83C558D04004
:10ED8000CE0183589F4F0F947557C757DF4F0881A7
:10ED900019812A813B81C958D040C357DF4F488031
:10EDA00059806A807B80CD58D040CF56DF4F888015
:10EDB0009980AA80BB80C159D040C358DF4F888159
:10EDC0009981AA81BB81CD57D040CF54DF4F888332
:10EDD0009983AA83BB83C15BD040CF57DF4F888123
:10EDE0009981AA81BB81C158D040CB54DF4F888321
:10EDF0009983AA83BB83C55BD040CB57DF4F888103
:10EE00009981AA81BB81C558D040C754DF4F888300
:10EE10009983AA83BB83C95BD040CB56DF4FC880A0
:10EE2000D980EA80FB80C559D040C756DF4F488162
:10EE300059816A817B81C959D040C356DF4F88818F
:10EE40009981AA81BB81CD59D0400093AC15109314
:10EE5000AD152093AE153093AF154092B01550927A
:10EE6000B1156092B2157092B3158092B41590925C
:10EE7000B515A092B615B092B715CF54DF4F0881E3
:10EE800019812A813B81C15BD0400093B815109352
:10EE9000B9152093BA153093BB15CB54DF4F0881B9
:10EEA00019812A813B81C55BD0400093BC1510932A
:10EEB000BD152093BE153093BF15C754DF4F088191
:10EEC00019812A813B81C95BD0400093C015109302
:10EED000C1152093C2153093C315C092C415D092AA
:10EEE000C515E092C615F092C7154093C81550930A
:10EEF000C9156093CA157093CB158093CC15909368
:10EF0000CD15A093CE15B093CF15C351DF4F188107
:10EF1000CD5ED040112309F4D6C183E59EE00E9466
:10EF20006F426E0123EAC20ED11CCF54DF4FD9824B
:10EF3000C882C15BD04002E0C353DF4F0883CD5C81
:10EF4000D040212C10ECC754DF4F1883C95BD04050
:10EF500009E7CF53DF4F0883C15CD04014E4CB53A3
:10EF6000DF4F1883C55CD040CF54DF4F0881198133
:10EF7000C15BD040CB54DF4F19830883C55BD040C1
:10EF8000C753DF4F1882C95CD040CB54DF4FA881F4
:10EF9000B981C55BD0400D911C917801EE0CFF1C2E
:10EFA000EE0CFF1CEDE6F0E0EC0FFD1FEE0DFF1D7B
:10EFB0004080518062807380CD52DF4F288139813B
:10EFC0004A815B81C35DD040C301B2010F94236AC3
:10EFD0004B015C01E1E0F0E0EC0FFD1FEE0DFF1DC9
:10EFE00084AD95ADA6ADB7ADC358DF4F8883998387
:10EFF000AA83BB83CD57D040F8013496EE0FFF1F94
:10F00000EE0FFF1F01E010E00C0F1D1FE00FF11FBE
:10F0100084AD95ADA6ADB7ADC757DF4F8883998353
:10F02000AA83BB83C958D040CB56DF4F18821982C0
:10F030001A821B82C559D0409E012B563F4FAE010C
:10F0400047575F4FBE0163587F4F8CEA95E10E949E
:10F0500048CBCB56DF4F288139814A815B81C55926
:10F06000D040C301B2010F94236A7B018C01222D91
:10F07000C754DF4F3881C95BD040CF53DF4F488141
:10F08000C15CD040CB53DF4F5881C55CD0400F945A
:10F09000CD6587FF10C02E2CC754DF4FF882C95BA7
:10F0A000D040CF53DF4F0883C15CD040CB53DF4FFC
:10F0B0001883C55CD04020E030E0A901C501B4014F
:10F0C0000F94846C87FDF1C080E59EE00E946F4242
:10F0D00045E0C501B4010E94324CCB54DF4F08819A
:10F0E0001981C55BD0400C5F1F4FCB54DF4F198394
:10F0F0000883C55BD040C753DF4F1881C95CD0403F
:10F10000113009F0CBC08AE00E94E43FCF54DF4FBA
:10F1100008811981C15BD04002501109CF54DF4FE3
:10F1200019830883C15BD040C353DF4F1881CD5C86
:10F13000D040113009F0ABC08AE00E94E43FCF52CA
:10F14000DF4F08811981C15DD0400430110509F0FD
:10F15000BAC087E29EE00E946F4242E0B42E760180
:10F16000A12CD7018D919C918C01000F111F000FD4
:10F17000111FE1E0F0E0EC0FFD1FE00FF11F44ADC7
:10F1800055AD66AD77ADC358DF4F488359836A8369
:10F190007B83CD57D040FC013496EE0FFF1FEE0F5E
:10F1A000FF1F21E030E02C0F3D1FE20FF31F84AD65
:10F1B00095ADA6ADB7ADC757DF4F88839983AA83B6
:10F1C000BB83C958D040CB56DF4F188219821A82B0
:10F1D0001B82C559D0409E012B563F4FAE01475769
:10F1E0005F4FBE0163587F4F8CEA95E10E9448CB88
:10F1F000EDE6F0E0EC0FFD1FE00FF11FCB56DF4F07
:10F20000288139814A815B81C559D04060817181F3
:10F21000828193810F94236A222DC754DF4F388156
:10F22000C95BD040CF53DF4F4881C15CD040CB5346
:10F23000DF4F5881C55CD0400F94236A2B013C01FD
:10F2400020E030E0A9010F94846C87FD38C084E28F
:10F250009EE00E946F4245E0C301B2010E94324C21
:10F2600034E0E30EF11C41E0A41226C08AE00E94C3
:10F27000E43F52E0C51AD10881E0B8121AC08AE012
:10F280000E94E43F85E09EE00F948F6024C001E07F
:10F29000C353DF4F0883CD5CD04066CE11E0C75327
:10F2A000DF4F1883C95CD04070CE80E20E94E43FFB
:10F2B0000FCFBB24B39453CFAA24A39452CF80E2A0
:10F2C0000E94E43FC8CFCF52DF4F08811981C15D52
:10F2D000D040012BB9F6C551DF4F1881CB5ED0402D
:10F2E000111188C08CE0EAE5F2E0DE01A358BF4FBF
:10F2F00001900D928A95E1F781E08093B70BCE01E2
:10F3000083589F4F0E94B0CCC755DF4F2881398169
:10F310004A815B81C95AD04060915A0270915B0268
:10F3200080915C0290915D020F94236A6B017C01D5
:10F330002DEB37E346E855EB0F94846C87FD4BC00B
:10F340002DEB37E346E855E3C701B6010F94CD65D1
:10F3500018160CF440C0C355DF4F288139814A810B
:10F360005B81CD5AD04060915E0270915F028091C6
:10F370006002909161020F94236A6B017C012DEB76
:10F3800037E346E855EB0F94846C87FD24C02DEBE2
:10F3900037E346E855E3C701B6010F94CD6518166B
:10F3A000D4F0C354DF4F288139814A815B81CD5B22
:10F3B000D0406091620270916302809164029091EA
:10F3C00065020F94236ACB57DF4F688379838A8362
:10F3D0009B83C558D0408CE0FE01E358FF4FAAE55F
:10F3E000B2E001900D928A95E1F7C451DF4F388069
:10F3F000CC5ED0403092B70B0C94B0708F929F923D
:10F40000AF92BF92CF92DF92EF92FF920F931F9332
:10F41000CF93DF9300D01F92CDB7DEB76C017B0195
:10F420008A01B22EA0900D141092091410920A14A1
:10F4300010920B1410920C1410920D140F94114C86
:10F4400020E030E0A901F80160817181828193811F
:10F450000F94CD65882319F1A11015C08091FD0B83
:10F46000811111C06091241470912514809126148B
:10F47000909127140F94906B209172023091730237
:10F480006217730764F081E00E949247811197C070
:10F4900081E080933C02109224080E947EF840E0B4
:10F4A00060E088E00F941C1220E030E0A901609138
:10F4B0003B0470913C0480913D0490913E040F9474
:10F4C000CD6587FF0FC080E090E0A0E2B1E48983C2
:10F4D0009A83AB83BC83BE016F5F7F4F8BE394E065
:10F4E0000E94073280E090E0A8ECB2E489839A831E
:10F4F000AB83BC83AE014F5F5F4F63E374E08FE289
:10F5000094E00E9432C580E090E0A0EAB0E48983F4
:10F510009A83AB83BC83BE016F5F7F4F87E394E028
:10F520000E9454C580913B0490913C04A0913D04FD
:10F53000B0913E048093660290936702A0936802A4
:10F54000B09369028093900690939106A0939206DF
:10F55000B093930680E996E00E9487BE109224083B
:10F560000E947EF885E79AE00F9458268091BE06A7
:10F5700081508093BE06882339F00E94719E80914D
:10F58000BE0681508093BE0680919406823011F4AD
:10F590000E94C6CE0E947ED90E947EF80F900F90E6
:10F5A0000F900F90DF91CF911F910F91FF90EF90EF
:10F5B000DF90CF90BF90AF909F908F900895AA203A
:10F5C00029F140E061E084E00F941C120E947A4728
:10F5D0008DE79AE00E946F4261E08B2D0E944B32D2
:10F5E000A090500583E08093500581E080936F06E2
:10F5F00080916F06882341F060E08B2D0E944B3292
:10F6000081E00E94895CF4CFA092500540E061E067
:10F6100085E00F941C1220E030E0A901F601608122
:10F620007181828193810F94CD65882371F080E090
:10F6300090E0A0ECB0E489839A83AB83BC83BE01E5
:10F640006F5F7F4FC6010E94073220E030E0A901C2
:10F65000F70160817181828193810F94CD65882348
:10F6600051F18090F3139090F413A090F513B090A3
:10F67000F61380E090E0A8ECB1E48093F31390934C
:10F68000F413A093F513B093F61380E090E0A0E09C
:10F69000B0E489839A83AB83BC83BE016F5F7F4FE5
:10F6A000C7010E9407328092F3139092F413A09244
:10F6B000F513B092F613812C912CA12C80E4B82E76
:10F6C00093E0E92E20E030E0A901F801608171812A
:10F6D000828193810F94846C18167CF440E060E082
:10F6E00086E00F941C1289829A82AB82BC82BE0192
:10F6F0006F5F7F4FC8010E940732F0905005E09283
:10F70000500510926F0640E060E087E00F941C12F5
:10F7100080912308811104C081E00E94895CF8CFA8
:10F72000F0925005813071F2BACE0F931F93CF93B0
:10F73000DF93D82FC62F0E947E4761E08C2F0E9456
:10F740004B320F94054C60527C468B4F9F4F609319
:10F75000091470930A1480930B1490930C14109254
:10F760000D141091500583E08093500581E0809343
:10F770006F0601E080916F06882309F447C060E0BE
:10F780008C2F0E944B3280910D148823D9F140E0D8
:10F7900060E08AE00F941C120E947A4787E29AE0A8
:10F7A0000E946F4280916F06882321F081E00E94C1
:10F7B000895CF8CF1092091410920A1410920B145D
:10F7C00010920C1410920D140F94114C80E00E94B2
:10F7D00092478D2F0E947E470F94054C60527C46C5
:10F7E0008B4F9F4F6093091470930A1480930B14EE
:10F7F00090930C1410920D1400936F0661E08C2FFF
:10F800000E944B3281E00E94895CB4CF1093500576
:10F81000DF91CF911F910F910895CF92DF92EF92D8
:10F82000FF92CF93DF93CDB7DEB76C970FB6F89406
:10F83000DEBF0FBECDBF8CE40E94562F882309F493
:10F84000B3C00E94D0326B017C0120E030E0A901FE
:10F850000F94846C87FF04C0F7FAF094F7F8F094E3
:10F86000F7FAF094F7F8F094C98EDA8EEB8EFC8EEE
:10F8700080E090E0A0E2B1E489839A83AB83BC830B
:10F8800080E090E0AAE2B3E48D839E83AF83B887E3
:10F8900080E090E0A0EAB1E489879A87AB87BC87D3
:10F8A00088E50E949F2F882351F040E050E0BA0184
:10F8B00088E50E94FA3269837A838B839C8389E589
:10F8C0000E949F2F882351F040E050E0BA0189E563
:10F8D0000E94FA326D837E838F8398878AE50E9427
:10F8E0009F2F882351F040E050E0BA018AE50E9442
:10F8F000FA3269877A878B879C87F0909B17F2FA98
:10F90000FF24F0F840E061E080E00F941C1280E5F5
:10F910000E949F2FE82E1D861E861F86188A8091C2
:10F92000BE06811134C02E2DAE01435F5F4FBE0174
:10F930006F5F7F4FCE0149960E94B647882339F109
:10F94000FF2011F0EE2019F160E080E00E94957B2D
:10F9500080E090E0A0E0B0E48D8B9E8BAF8BB88F01
:10F96000198A1A8A1B8A1C8A1D861E861F86188A77
:10F970008091BE06882359F020E0AE014B5E5F4FB8
:10F98000BE016F5E7F4FCE010D960E94FE796C9690
:10F990000FB6F894DEBF0FBECDBFDF91CF91FF90C1
:10F9A000EF90DF90CF900895C12CD12CE12C80E412
:10F9B000F82E56CF1F920F920FB60F9211240BB64E
:10F9C0000F922F938F939F93EF93FF938091E10377
:10F9D0002091E003821306C08091C1008F7D809347
:10F9E000C10012C0E82FF0E0E052FC4F92818F5F1F
:10F9F0008F719093C6008093E1039091C000906452
:10FA00009093C000281741F3FF91EF919F918F9140
:10FA10002F910F900BBE0F900FBE0F901F90189557
:10FA20001F920F920FB60F9211240BB60F920F93E5
:10FA30001F932F933F934F935F936F937F938F9376
:10FA40009F93AF93BF93CF93DF93EF93FF93009177
:10FA50007505D091740511E01D0F1F77C091C60088
:10FA60009091DF039C3008F074C0E92F092E000C40
:10FA7000FF0B8827E15CF2488F4F0D946A6D4B7D38
:10FA8000767D847D8C7D937DA97D977DA97D9B7DF1
:10FA90009F7DA97DA37DCD34A9F1CE3419F0C0326C
:10FAA00069F503C081E08093DF03011731F0ED2F8A
:10FAB000F0E0EC58FA4FC283D12FD0937405FF9138
:10FAC000EF91DF91CF91BF91AF919F918F917F91F6
:10FAD0006F915F914F913F912F911F910F910F90D7
:10FAE0000BBE0F900FBE0F901F901895CA3340F4B5
:10FAF000C033D8F6C032C9F2CD32B9F28BE0D3CFE1
:10FB0000CD34E1F782E0CFCFC13321F0C43339F6F1
:10FB100088E0C9CF83E0C7CF84E0C03321F286E01C
:10FB2000C13309F2EBCF85E0C83341F7BCCF87E0A2
:10FB3000C23321F7B8CF89E0C13301F7B4CF8AE0EF
:10FB4000C033E1F6B0CFCA3009F0AFCF1092DF0377
:10FB5000ACCFCA3009F0A9CF809181168823B1F3C8
:10FB6000973049F09A3059F0953081F71092500251
:10FB700010926F06EBCF81E080939906E7CF0E9449
:10FB80003CC10E9476BE8EEF0E9482CD0E9473C55A
:10FB9000DDCF8EBD0DB407FEFDCF08958FEF8EBD76
:10FBA0000DB407FEFDCF8EB50895909164009B7F44
:10FBB00090936400982F906A96959CBD80FD03C039
:10FBC00091E0863009F490E09DBD08952F923F9218
:10FBD0004F925F926F927F928F929F92AF92BF925D
:10FBE000CF92DF92EF92FF920F931F93CF93DF9309
:10FBF000CDB7DEB7A5970FB6F894DEBF0FBECDBF69
:10FC00008DA33090500591E090935005809173053D
:10FC10008D3409F4BFC3843511F40C9432928734C7
:10FC200091F400917105109172050531110509F4E7
:10FC300038C1C4F4043011054CF4023011050CF045
:10FC400038C117FF56C00F94BF3F2BC104301105B8
:10FC500009F442C10C301105B1F78BEF92E10E941B
:10FC60008F921FC10E31110509F48EC29CF50C3123
:10FC7000110509F46BC10CF061C20B31110519F7C4
:10FC800041E061E081E00E94CFC381110AC180E0C0
:10FC900090E0A0E2B1E489839A83AB83BC8380E0E7
:10FCA00090E0AAE2B3E48D839E83AF83B88780E0BF
:10FCB00090E0A0EAB1E489879A87AB87BC8770E0BF
:10FCC00060E080E50E94A131BE016F5F7F4F0E941E
:10FCD00074DFE7C00B35110509F408C30C351105B5
:10FCE00009F407C30A35110509F0ADCF10924F058D
:10FCF000D8C080913802882309F4D3C08AE50E94D5
:10FD0000562F082F89E50E94562F182F88E50E944C
:10FD1000562F402F612F0E94CFC38111C2C00E9475
:10FD2000113380913D02882321F084E896E00E94FF
:10FD30003DC38091641183FD7DC0C0909006D0903A
:10FD40009106E0909206F090930620916602309121
:10FD500067024091680250916902C701B6010F9491
:10FD6000CD65882309F466C08091FD0B81111FC009
:10FD70006091241470912514809126149091271479
:10FD80000F94906B20917202309173026217730787
:10FD900074F4C0926602D0926702E0926802F09218
:10FDA00069020E947A4787ED92E10E946F4240907B
:10FDB0009006509091066090920670909306209164
:10FDC0006602309167024091680250916902C30156
:10FDD000B2010F94236A6B017C0120E030E0A9019D
:10FDE0000F94846C87FF04C0F7FAF094F7F8F0944E
:10FDF00020916E0230916F02409170025091710219
:10FE0000C701B6010F94336620E030E048E453E4C4
:10FE10000F94846C181674F4409266025092670234
:10FE200060926802709269020E947A4788EB92E1C0
:10FE30000E946F426091120270911302072E000C13
:10FE4000880B990B0F94D46520915602309157027C
:10FE500040915802509159020F9433662AE037EDD1
:10FE600043E25CE30F94336669837A838B839C83DC
:10FE7000C12CD12C76018E010F5F1F4F20E936E097
:10FE80004CE856E068E876E084E896E00F94F53EAA
:10FE900080E1E4E8F6E0AAE5B2E001900D928A95EF
:10FEA000E1F78DA181110C943A8A0E945D4A0C946D
:10FEB0003A8A809138028823A1F341E061E081E031
:10FEC0000E94CFC38111EDCF81E00230110509F00E
:10FED00080E00E944066E5CF80E50E949F2FC12C04
:10FEE000D12C7601882321F00E94C0326B017C0165
:10FEF00083E50E949F2F882361F00E94D03220E08A
:10FF000030E04AE754E40F9433660F94976B6B012B
:10FF10007C010E9476BE80917713811105C060E05C
:10FF200082EF92E10E942CD90F94054CC60ED71E89
:10FF3000E81EF91E0F94054C6C197D098E099F0966
:10FF400097FFAFCF80E00E94895CF4CF81E00E94F0
:10FF5000AE3E8091AF0B8770873051F460E08FE444
:10FF60000E94F231882321F080E00E94AE3E99CFBA
:10FF70000E9476BE9090B70B80E00E94AB330E9447
:10FF800052C481E0809338090E946CC688E50E94C3
:10FF9000562F182F89E50E94562F082F8AE50E94B8
:10FFA000562F101304C0181711F40C94509281119D
:10FFB000B6C00E944132A12C82E50E949F2F882367
:10FFC00009F4B5C00E94D0326B017C0120E030E022
:10FFD000A9010F94CD65882339F1111104C00023C4
:10FFE00011F40C948292C0928C06D0928D06E0920D
:10FFF0008E06F0928F06A7019601609162027091C1
:020000021000EC
:10000000630280916402909165020F94CD6587FF31
:100010000BC019821A821B821C82BE016F5F7F4F48
:100020008CE896E00E9454C5112319F080E00E94EC
:1000300075C5002319F081E00E9475C50E9473C543
:10004000109238090E946CC6412C512C32011123A8
:1000500031F0412C512C10EA612E10EC712EC12C84
:10006000D12CB0EAEB2EB0E4FB2E011103C0C12C61
:10007000D12C7601A1100C94569220E030E0A90119
:10008000C301B2010F94CD65811109C020E030E0B9
:10009000A901C701B6010F94CD65882371F118A29B
:1000A00019A21AA21BA2A701960160915E0270918B
:1000B0005F0280916002909161020F94236A6C8FBD
:1000C0007D8F8E8F9F8FA301920160915A02709154
:1000D0005B0280915C0290915D020F94236A6983B8
:1000E0007A838B839C83AE01405E5F4FBE01645E6A
:1000F0007F4FCE0101960E9432C5809137098093CF
:100100003809892D0E94AB330E9439C483E0809363
:1001100075020E94F5DC80E00E94AE3EC2CE0E94D5
:10012000413282E00E9475C5AA24A39445CFC12C18
:10013000D12C80E8E82E80E4F82E4FCF13E00E9407
:10014000626B8823E1F0115049F087E495E10F9448
:10015000582682E894E10E948F92F1CF84ED95E1D8
:100160000F94582685E695E10E948F9282EF93E2E4
:100170000F94582684E595E10E94E24892CE81EEE4
:1001800095E10E948F928DCE20E030E0A901609130
:100190005A0270915B0280915C0290915D020F9413
:1001A000246AAB01BC0188E50E94FA326C8F7D8F16
:1001B0008E8F9F8F20E030E0A90160915E027091E8
:1001C0005F0280916002909161020F94246AAB01FA
:1001D000BC0189E50E94FA329B01AC0129833A8374
:1001E0004B835C836C8D7D8D8E8D9F8D0E94EB2E5D
:1001F000882309F456CE80E00E94AB330E9452C49B
:1002000061E085E40E94F23121E0482FBE016F5F7A
:100210007F4FCE014C960F9402406B017C01AC01E4
:100220009B010F94166D81115CC04C8C5D8C6E8CA3
:100230007F8C20E030E0A901C301B2010F94CD65AD
:1002400027E137EB41E558EB87FD04C027E137EBA9
:1002500041E558E3C301B2010F94246AAB01BC012C
:1002600082E096E10E94005449805A806B807C8035
:1002700020E030E0A901C301B2010F94CD6527E170
:1002800037EB41E558EB87FD04C027E137EB41E54B
:1002900058E3C301B2010F94246AAB01BC018DEF96
:1002A00095E10E94005420E030E0A901C701B601A9
:1002B0000F94CD6527E137EB41E558EB87FD04C08E
:1002C00027E137EB41E558E3C701B6010F94246AF3
:1002D000AB01BC0188EF95E10E9400548AE00E94C6
:1002E000E43F0E9439C40E94F5DCDBCD90934F05BA
:1002F000D8CDF0E8CF2EF2E0DF2EAAE5EA2EA2E07C
:10030000FA2E1CA2212C10E0F60181916F010E94AF
:100310009F2F082F882349F10E94D0322B013C01E6
:10032000F70120813181428153810F94236A4B016F
:100330005C012DEB37E346E855EB0F94846C87FDA9
:100340000AC02DEB37E346E855E3C501B4010F942D
:10035000CD65181654F4133011F4202E0CA1F701BA
:1003600040825182628273820CA31F5FF4E0EF0E21
:10037000F11C143049F62CA1222329F00E9473C5E8
:100380000E94F5DC8ECD2220D9F386E692E00E9411
:1003900087BEF6CF009171051091720509371105DE
:1003A00011F40C94578C0CF001C20E34110509F4B1
:1003B00001C70CF033C10A31110509F478C50CF0FE
:1003C000BFC00431110509F406C50CF092C001311B
:1003D000110509F4F6C40CF06EC00230110508F0E6
:1003E00032CC60906F057090700580E50E949F2F61
:1003F000182FC12CD12C7601882359F00E94C032CD
:100400006B017C0111E0C114D104E104F10409F491
:1004100010E083E50E949F2F882311F40C947592BD
:100420000E94D03220E030E04AE754E40F94336673
:100430000F94976B6B017C0111110C947992C1148C
:10044000D104E104F10411F00C9479926114710467
:1004500011F40C947992F3018081882311F40C94A7
:1004600079920E9476BEC3010F94852810915005A1
:1004700083E08093500581E080936F06C114D1041E
:10048000E104F10409F48EC40F94054CC60ED71E86
:10049000E81EF91E0F94054C6C197D098E099F0901
:1004A00097FF88C480916F06882309F483C480E095
:1004B0000E94895CEFCF0231110509F0C4CB83E5BE
:1004C0000E949F2F882311F40C94A98A0E94D03295
:1004D00020E030E04AE754E40F9433660F94976BC2
:1004E00060930102709302028093030290930402CE
:1004F000D8CC0731110509F496C484F405311105EF
:1005000009F48EC40631110509F09DCB0E9430A577
:1005100080919B17877F80939B17C3CC083111056F
:1005200009F494C40931110509F08DCB80919B1712
:1005300082FF03C08B7F80939B170E940D7CB1CC00
:100540000032110509F48BC5E4F50D31110509F4EC
:1005500020C58CF40B31110509F4C8C40C31110508
:1005600009F071CB40E060E080916F0590917005DB
:100570000E9406AB96CC0E31110509F411C50F315E
:10058000110509F060CB0E940BCE6C8F7D8F8E8F92
:100590009F8FBE016F5F7F4FCE014C960E94B63891
:1005A000CE0101960F9485280E947A47BE016F5FA5
:1005B0007F4F8BEA96E10E941B468AE00E94E43F4F
:1005C00070CC0B34110509F4EDC5ECF40A321105B9
:1005D00009F48BC50934110509F035CB80E50E947B
:1005E000562F882309F45DCC80919B1782FD59CC4E
:1005F0000E94C23190E08536910514F084E690E0C7
:10060000809361064ECC0C34110509F4CFC50D342E
:10061000110509F018CB0E943DCE43CC0C361105D4
:1006200009F43FCC0CF061C00535110509F4D6C7BB
:1006300034F50235110509F483C7C4F401351105F9
:1006400009F001CB0E9490AC0E943DCE0E94EBC00D
:100650000E94A93E68EE73E080E090E00E94793E3F
:1006600060E08FE897E10E942CD91BCC033511057F
:1006700009F46AC70435110509F421CFE4CA093623
:10068000110509F4E8C6F4F40C35110509F4C1C7E5
:100690000836110509F0D7CA8091641183FD01CC99
:1006A0000E94BF4A87FDFDCB83E50E949F2F8823D0
:1006B00009F4F7CB0E94D0320F94906BCB010E94CB
:1006C0008DF5EFCB0A36110509F416C70B36110567
:1006D00009F0B9CA60E080E50E94D6318111E1CB12
:1006E0001092031410926506DCCB0237110511F449
:1006F0000C94AA8BA4F50F36110509F434C6CCF47A
:100700000D36110509F4E8C50E36110509F09BCA2E
:100710008EE40E949F2F882309F4C3CB0E9491315D
:100720006093721370937313809374139093751383
:10073000B8CB0037110509F4B4CB0137110509F026
:1007400082CA83E50E949F2F882309F453C60E9422
:10075000C2318D3308F049C680930002A2CB063720
:10076000110511F40C941A8C84F40337110511F45B
:100770000C94B08B0537110509F065CA80916F059F
:10078000909170050F9485288CCB0737110511F4D3
:100790000C944D8C0837110509F055CA81E08093FF
:1007A0003809809337090E946CC67BCB023981E0FF
:1007B000180711F40C94E68F0CF071C1033D11057C
:1007C00011F40C94488D0CF0DDC00B39110509F4BF
:1007D0006CC62CF50D37110509F4AEC63CF40A378A
:1007E000110509F030CA0E94D6525BCB0C381105B6
:1007F00009F410C60139110509F025CA70E060E05E
:1008000083E50E94B3318C01823010F40C945F8C2C
:100810000E942E468BEB99E10E946F4242CB0B3C2B
:10082000110511F40C94AC8C64F50E3B110509F420
:100830000EC6093C110509F006CA0E94BF4A87FD91
:1008400030CB00E812E08BEBE82E83E1F82EF801C4
:1008500081918F010E94562F882349F00E94D03247
:100860000F94976BF7016083718382839383F4E025
:10087000EF0EF11C22E00438120749F70E9404BE73
:1008800010CB0C3C110511F40C94CF8C0D3C1105D0
:1008900009F0D9C980916B05827149F480916D0589
:1008A0008C7829F480916E05837009F4FACA82E489
:1008B0000E94562F882351F00E94C0326093CB13C0
:1008C0007093CC138093CD139093CE1383E50E9445
:1008D000562F882351F00E94D0326093FB137093FF
:1008E000FC138093FD139093FE1384E50E94562F12
:1008F000882351F00E94D0326093FF13709300144C
:10090000809301149093021488E50E94562F882347
:1009100051F00E94D0326093D90B7093DA0B809320
:10092000DB0B9093DC0B89E50E94562F882351F056
:100930000E94D0326093DD0B7093DE0B8093DF0B4F
:100940009093E00B8AE50E94562F882351F00E9475
:10095000D0326093E10B7093E20B8093E30B9093A2
:10096000E40B85E40E94562F882309F49ACA0E945A
:10097000D0326093E50B7093E60B8093E70B909376
:10098000E80B8FCA0D32F1E01F0711F40C94A58E0D
:100990000CF061C0023E110511F40C94E18DE4F5F8
:1009A0000C3D110511F40C94B88D0D3D110509F0A5
:1009B0004AC90E94BF4AD82E87FD73CA83E50E94A8
:1009C0009F2FED2C0D2C000CFF088701000F111F2D
:1009D000882311F40C94C78D0E94AF31F801E25FB7
:1009E000FD4F918380838701000F111F000F111F9E
:1009F00002591D4FBC01990F880B990B0F94D465B8
:100A00002AE037ED43E25CE30F943366F80160833C
:100A100071838283938345CA023281E0180711F4FF
:100A20000C94208E0C32114009F00DC964E071E085
:100A300083E50E94A1318C0168EE73E080E50E949D
:100A4000A131893823E1920710F088E893E1B801D9
:100A50000E94FFD826CA0033F1E01F0711F40C945E
:100A6000278F6CF40E3281E0180711F40C949B8FE1
:100A70000F32114009F0E7C80E94115412CA003920
:100A8000F1E01F0711F40C94E28F0139114009F0D5
:100A9000DAC881E00E947BC60E94F5DC02CA0B35F1
:100AA00082E0180711F40C9450900CF0C2C0063F7D
:100AB000F1E01F0711F40C94F98F0CF08AC0093A89
:100AC00081E0180711F40C94F18F0CF075C00A390D
:100AD000F1E01F0709F4E5C9043A114009F0B3C871
:100AE00083E50E94562F1091B70B882341F00E9496
:100AF000E231182F811103C080E00E94AB33809156
:100B00005A0290915B02A0915C02B0915D028983D0
:100B10009A83AB83BC8380915E0290915F02A09127
:100B20006002B09161028D839E83AF83B88780910C
:100B3000620290916302A0916402B091650289877C
:100B40009A87AB87BC8786E50E94562F882321F0C1
:100B500089EC9AE10F948F60812F0E94AB331123AF
:100B600051F08091B70B811106C00E942E468AEA8F
:100B70009AE10E946F420E947A478CE99AE10E94B2
:100B80006F428091B70B882311F40C94ED8F89E9A3
:100B90009AE10E946F428AE00E94E43F4CE050E0FC
:100BA0006AE572E0CE0101960F947F6D892B09F4FE
:100BB00078C90E94F5DC75C9043F81E0180711F47B
:100BC0000C94F58F053F114009F03DC80E9469EA79
:100BD00068C90C30F2E01F0711F40C940590DCF4A6
:100BE000073F81E0180711F40C94FD8F083F114076
:100BF00009F029C881E0809370060E94F2E3109208
:100C00007006882309F44DC90E947A4786EE9AE15E
:100C10000E946F4246C90933F2E01F0711F40C9499
:100C200036910835124011F00C94237E0E940193F6
:100C300038C90F3883E0180711F40C943A910CF07E
:100C400084C00335F3E01F0711F40C94109054F4A2
:100C50000A5213400A30110510F00C94237E0E94B2
:100C600035941FC9043883E0180711F40C94CD9013
:100C70000A38134011F00C94237E60E089E40E944E
:100C8000D631D82E90E8692E92E0792E11E000E05E
:100C900070E060E0F30181913F010E94B3317C017B
:100CA0000097C1F0023011F40C941891033011F444
:100CB0000C942491013011F40C940C91D11009C0C2
:100CC00090939F1580939E15BC0188E695E10F9443
:100CD000535110E00F5F0430D9F6112309F4E1C835
:100CE0000E943E4060919E1570919F1587E49BE1A4
:100CF0000E9411468AE00E94E43F0E943B406091BE
:100D00005F157091601589E59BE10E9411468AE0AC
:100D10000E94E43F0E943840609120157091211597
:100D20008BE69BE10E9411468AE00E94E43F0E940C
:100D300035406091E1147091E2148DE79BE10E94CF
:100D400011468AE00E94E43FACC80239F3E01F0775
:100D500011F40C94DE9174F4003983E0180711F457
:100D60000C9470910139134011F00C94237E0E9471
:100D7000E84A97C8003AF3E01F0709F4A6C1073E06
:100D8000134011F00C94237E81E08093380210927E
:100D9000BA1360E083E50E94F231811182C80E949B
:100DA000C65A7FC880916F06882321F080E00E9498
:100DB000895CF8CF0E947ED910926F06109350057F
:100DC00070C860E08DE196E10E942CD917981698C2
:100DD0001598149866C885E396E10E946F421092B8
:100DE0002C0780E994E10E9458A28BE1E0E9F4E14C
:100DF000DE01119601900D928A95E1F750E040E0F6
:100E0000BE016F5F7F4F90E080E00E941BA9CE0182
:100E100001960E9453A686E296E10E946F4241C865
:100E20000E9441A53EC880916F0590917005FC011C
:100E30002191222331F02032D9F7DF0111971C9242
:100E4000F7CF40E061E00E9406AB2BC88091BE0660
:100E50008823E9F080E090E0A0EAB1E488A399A3B8
:100E6000AAA3BBA31C8E1D8E1E8E1F8E19821A82F2
:100E70001B821C8220E0AE01405E5F4FBE01645EBB
:100E80007F4FCE0101960E94FE790C94517F0E9403
:100E90009239882321F00E94719E0E94C6CE8AE476
:100EA0009CE30F9458260E947ED90C94517F809128
:100EB0009B1783FD02C00C94517F83E50E949F2FF6
:100EC000882311F40C94517F0E949131AB01BC0135
:100ED00040939717509398176093991770939A17A8
:100EE00087E394E10E94C4A10C94517F83E40E94A3
:100EF000562F882319F180E596E10E946F42809178
:100F00003A14882391F0BE016F5F7F4F87E394E12D
:100F10000E948AA48E010F5F1F4FF80181918F01FB
:100F2000882339F00E94E43FF8CF86E496E10E94DE
:100F30006F428AE00E94E43F0C94517F80919B179E
:100F400082FF21C08FE596E10E946F426091971762
:100F5000709198178091991790919A174AE00E9482
:100F6000B4498FE20E94E43F609193177091941707
:100F700080919517909196174AE00E94B4490E947B
:100F8000C05A0C94517F81E796E10E946F420C9405
:100F9000517F80919B178E7F80939B170C94517F7C
:100FA00080919B1783FD02C00C94517F0F94E83F02
:100FB00080919B1783FD02C00C94517F60916F0557
:100FC00070917005CE014C960F9441298C010097C9
:100FD00011F40C94517F6C8D7D8D19821C8222E05E
:100FE000AC01CE0101960E9422A8811119C0F12CFA
:100FF000CE0101960E9453A6B801FF2031F18DE980
:1010000096E10E941B468AE00E94E43F10929717E7
:10101000109298171092991710929A170C94517F6A
:10102000CE0101960F94AD28882309F361E0CE012B
:1010300001960E9470A40097D1F225EEFC01208356
:101040001C820E94799FF82ED3CF85E896E10E94FA
:101050001B4682E896E10E946F420C94517F80917A
:101060009B1782FD0E9476BE80919B1783FD02C074
:101070000C94517F60E080E50E94F231182F482FD8
:1010800061E080916F05909170050E9406AB83E549
:101090000E949F2F882381F00E949131AB01BC01F7
:1010A00040939717509398176093991770939A17D6
:1010B00087E394E10E94C4A10E94719E11110C94D7
:1010C000517F0E94C6CE0C94517F20916F053091C4
:1010D000700590919B17926090939B1740E060E0A1
:1010E000C9010E9406AB0C94517F83E50E949F2F9B
:1010F000882311F40C94517F0E94C231F82E80E5B0
:101100000E949F2F811108C081E0F11001C080E092
:101110000E94AE3E0C94517F6DE070E080E50E942D
:10112000B3318C0197FF02C00C94517FE82E60E030
:1011300089E40E94F231811120C077ECC72E76E15C
:10114000D72EE6EE6E2EE6E17E2E41E050E0B601AF
:10115000CE0101960F9406658981E81208C00E94AD
:101160002E4688EB96E10E946F420C94517FFFEF70
:10117000CF1ADF0A6C147D0441F761E0802F0F94D1
:10118000CA4A6F2D802F0F9496496F2D70E0802FE3
:101190000F94FB4A28E0E2120C94517FF092031462
:1011A0000C94517F0E94C6CE0C94517F0E94FECEBB
:1011B0000C94517F70E060E083E50E94B3318E347F
:1011C000910531F40E94D5BD0E947ED90C94517FC7
:1011D00084E497E10E946F42609127097091280989
:1011E0008BE397E10E9411466091290970912A09C9
:1011F0008EE297E10E9411466091270970912809BB
:101200008091290990912A09681B790B8091940695
:10121000815021E030E0823010F030E020E0621BAD
:10122000730B83E297E10E9411468AE00E94E43F3B
:101230008BE197E10E946F4280912B0990912C09DC
:10124000A0912D09B0912E098C8F9D8FAE8FBF8FED
:10125000BE016F5F7F4FCE014C960E94B638BE0133
:101260006F5F7F4F8EE097E10E941B4680912F09B0
:1012700090913009A0913109B09132098C8F9D8FE6
:10128000AE8FBF8FBE016F5F7F4FCE014C960E9425
:10129000B638BE016F5F7F4F8EEF96E10E941B460E
:1012A00020E030E04AE754E460913309709134095A
:1012B00080913509909136090F941E6BAB01BC01EA
:1012C00086EE96E10E9400548DE60E94E43F8AE09B
:1012D0000E94E43F0C94517F8091641183FF02C00F
:1012E0000C94517F0E94BF4A082F87FF02C00C94C4
:1012F000517F83E50E949F2F182F882319F10E94A8
:10130000D0320F94906BCB010E948DF56091281420
:1013100070912914072E000C880B990B0F94D4653B
:1013200020912414309125144091261450912714B3
:101330000F94846C18166CF48EE597E160E00E94BF
:101340002CD90BC082E50E949F2F8111D8CF0C941D
:10135000517F8CE497E1112389F3612F802F0E9444
:1013600085DB0C94517F83E50E94562F882331F052
:1013700060E083E50E94D631809364110E947A4731
:101380008EE797E10E946F4280916411882351F1AA
:1013900010E000E020E08091641190E0B0E0A0E077
:1013A000002E04C0B695A795979587950A94D2F715
:1013B00080FF12C0FF24F394F20E222319F08CE276
:1013C0000E94E43FF801EE0FFF1FEC58F84E8591A4
:1013D00094910E946F422F2D0F5F1F4F0530110512
:1013E000D1F6A7CD80E797E1A2CD8CE380930002F0
:1013F0000C94517F0E947A474091000250E070E0C7
:1014000060E085E897E10E94184A8AE00E94E43F84
:101410000C94517F8091641183FF02C00C94517F22
:1014200083E50E949F2F882311F40C94517F0E9422
:10143000D0320F94906B6C3871050CF48B011093C3
:10144000AA060093A9060E9487960C94517F0E94D9
:1014500049640C94517F0E94BF4A182F87FD0AC02F
:101460008CE897E10E946F42812F0E9416DB8AE090
:101470000E94E43F30925005A5960FB6F894DEBF67
:101480000FBECDBFDF91CF911F910F91FF90EF90D5
:10149000DF90CF90BF90AF909F908F907F906F9094
:1014A0005F904F903F902F90089583E50E949F2F6B
:1014B000882311F40C94517F0E94C231182F8D3370
:1014C00008F01CE3109346050F94054C6B017C015A
:1014D000212F30E0A8EEB3E00F94146AC60ED71E99
:1014E000E81EF91EC0924205D0924305E0924405E1
:1014F000F09245050C94517F60E080E50E94D63162
:1015000081110C94517F81E40E94562F6091031445
:1015100070E0811102C06FEF70E083E50E94A1319D
:101520008F3F910519F010F08FEF90E08093031436
:10153000809365060C94517F0E940D7C0C94517F22
:1015400010924A050C94517F81E080934A050C94D7
:10155000517F88E50E94562F811113C089E50E94B2
:10156000562F81110EC08AE50E94562F811109C0A5
:1015700085E40E94562F811104C00E94EBC00C9498
:10158000517F0E9476BE88E50E94562F882331F055
:10159000179A8091AF0B8E7F8093AF0B89E50E94E5
:1015A000562F882331F0169A8091AF0B8D7F809350
:1015B000AF0B8AE50E94562F882331F0159A80914F
:1015C000AF0B8B7F8093AF0B85E40E94562F88234F
:1015D00011F40C94517F149A0C94517F83E50E946E
:1015E000562F882311F40C94517F0E94D03220E0B2
:1015F00030E04AE754E40F9433660F94976B60939E
:101600004B0570934C0580934D0590934E050C94BB
:10161000517F0E94BF4A87FF02C00C94517F809186
:101620006B0584FD09C080916D0587FD05C0809123
:101630006E05837009F489C040E8C42E42E0D42EC0
:101640005BEBE52E53E1F52E10E0F60181916F0181
:101650000E949F2F882309F465C0133009F06DC0E4
:101660000E94D0322B013C0120E030E040EA51E4FE
:101670000F94CD6587FF4EC0A30192016091DB13EB
:101680007091DC138091DD139091DE130F941E6B2B
:101690004B015C01AC019B016091E50B7091E60B85
:1016A0008091E70B9091E80B0F9433666093E50B04
:1016B0007093E60B8093E70B9093E80BA5019401E0
:1016C0006091EB137091EC138091ED139091EE13F8
:1016D0000F9433666093EB137093EC138093ED13C8
:1016E0009093EE136091D10B7091D20B8091D30B3C
:1016F0009091D40B0F94D265A50194010F94336699
:101700000F94976B6093D10B7093D20B8093D30B94
:101710009093D40B4092DB135092DC136092DD1354
:101720007092DE131F5FF4E0EF0EF11C143009F02D
:101730008CCF0E9452BE0C94517F0E94D032F70190
:10174000648B758B868B978BEDCF81E00F94C02ACD
:101750000C94517F0E9476BE0E94F5DC0C94517F60
:1017600087EC98E10E946F4260E087EB98E10E946D
:10177000E05A60E082EA98E10E94E05A61E08BE979
:1017800098E10E94E05A60E080E998E10E94E05A06
:1017900061E080E898E10E94E05A60E087E798E124
:1017A0000E94E05A61E08DE698E10E94E05A61E013
:1017B00083E698E10E94E05A61E08BE598E10E949F
:1017C000E05A61E08DE498E10E94E05A61E08FE325
:1017D00098E10E94E05A60E080E398E10E94E05ABC
:1017E00060E082E298E10E94E05A60E08CE098E1DB
:1017F0000E94E05A61E08BEF97E10E94E05A60E0BE
:101800008CEE97E10E94E05A60E087ED97E10E943C
:10181000E05A61E084EC97E10E94E05A60E087EBD7
:1018200097E10E94E05A60E083EA97E10E94E05A63
:101830000C94517F00916F051091700583E0F12C9D
:1018400040E08150E1F0F8019081292F2B7F213475
:10185000C1F721812133A9F7913421F0953421F486
:1018600041E002C0FF24F39498012E5F3F4F8901AD
:101870002F5F3F4FF80190819032C9F3E2CF4111C1
:101880000E947A47FF2021F087EB99E10E946F4286
:10189000C8010E94245B0C94517F81E00E94AE3EFF
:1018A0000E943BC680E00E94AE3E0C94517F109295
:1018B0003809109237090E946CC60C94517F88E455
:1018C0000E949F2F8823A9F00E94AF31F801FF27C3
:1018D000EE0FFF1FE158F94F833221E0920714F019
:1018E00082E291E08837910514F488E790E09183D3
:1018F000808386E40E949F2F882379F00E94AF3175
:1019000097FD28C08F3F910519F014F08FEF90E0FC
:10191000F801FF27E758F94F808382E40E949F2F48
:10192000882311F40C94517F0E94AF31F801FF27F6
:10193000EE0FFF1FE558F94F8D38910514F08CE834
:1019400090E08530910514F485E090E091838083E8
:101950000C94517F80E0DCCF0E94BF4A87FF02C019
:101960000C94517F10E8E12E12E0F12E10E000E01F
:10197000F70181917F010E94562F882349F00E9430
:10198000D032F801E554FC4E64A375A386A397A357
:101990000C5F1F4F0031110559F70C94517F809156
:1019A0006C0587FD2DC080916D058E7049F54091C5
:1019B000EF135091F0136091F1137091F21383EED5
:1019C00099E10E9400544091F3135091F4136091F7
:1019D000F5137091F61380EE99E10E940054409146
:1019E000F7135091F8136091F9137091FA138DED7C
:1019F00099E10E9400548AE00E94E43F0C94517FD8
:101A000083E50E949F2F882391F00E94D03260933B
:101A1000EF137093F0138093F1139093F21360938C
:101A2000F7137093F8138093F9139093FA1380E5EA
:101A30000E949F2F882351F00E94D0326093EF13B1
:101A40007093F0138093F1139093F21382E50E9448
:101A50009F2F882351F00E94D0326093F31370932C
:101A6000F4138093F5139093F61384E50E949F2F4F
:101A7000882311F40C94517F0E94D0326093F713A5
:101A80007093F8138093F9139093FA130C94517F89
:101A90000E947A4783E19AE10E946F4283E50E94A7
:101AA000562F882321F00E94E23180933D028091DD
:101AB0003D02882309F459C089E99AE10E946F42E6
:101AC0008BE09AE10E946F424091140250911502FE
:101AD000609116027091170289E09AE10E94005409
:101AE00040911C0250911D0260911E0270911F02D4
:101AF00086E09AE10E940054409124025091250210
:101B0000609126027091270283E09AE10E940054BE
:101B10008BEF99E10E946F42409118025091190297
:101B200060911A0270911B0289EF99E10E940054A2
:101B30004091200250912102609122027091230273
:101B400086EF99E10E9400544091280250912902A9
:101B500060912A0270912B0283EF99E10E94005458
:101B60008AE00E94E43F0C94517F85E99AE1A6CF78
:101B700083E50E949F2F882311F40C94517F0E94CB
:101B8000AF3190931302809312020C94517F0E9404
:101B90007A4785E40E94E43F80E38D0D0E94E43F94
:101BA000F801E25FFD4F6081718183E29AE10E945A
:101BB000B24A85E20E94E43F8AE00E94E43F0C942E
:101BC000517F80E50E94562F882311F40C94517F99
:101BD00070E060E080E50E94B331E82E6FEF7FEFA8
:101BE00083E50E94B3318C010196039710F00C94A9
:101BF000517FE7FE02C00C94517F0E9476BE0E2CEE
:101C0000000CFF080F3F100789F001301105A9F003
